:020000040800F2
:10000000002000100989020841D501083D39020885
:100010003DD5010839D5010835D50108000000009B
:1000200000000000000000000000000031D50108C1
:100030002DD501080000000029D50108152201086E
:1000400071890208718902087189020871890208A0
:100050007189020871890208611001088D11010877
:100060005111010815110108D9100108F5D800082F
:10007000E5D80008D5D80008C5D80008B5D80008CC
:10008000A1D800088DD8000871890208718902087A
:10009000EDD8010871890208718902089D100108D4
:1000A00075170108D117010865170108F517010830
:1000B000C5170108B5170108A517010871890208BD
:1000C0007189020871890208718902087189020820
:1000D00071890208C50201081D230108A122010837
:1000E000251001087189020819D5010871890208D3
:1000F000851701087189020895170108718902089E
:1001000000000000000000000000000071890208EB
:1001100071890208718902087189020871890208CF
:1001200079D8000865D8000851D800083DD80008E3
:1001300029D80008718902080000000000000000B2
:1001400071890208718902087189020800000000A3
:10015000000000000000000000000000000000009F
:100160000000000000000000718902087189020887
:10017000718902080000000000000000000000007B
:08018000000000007189020873
:100188002DE9F04FB0F908502DED048B0D81EDB23B
:10019800382D8FB00C4600F0E284804634D9802D8B
:1001A80000F0DA8078D8522D00F0008140F25084B7
:1001B800542D00F0C7846E2D40F016817D4B0A68DF
:1001C8001B887D4DFF2BA8BFFF23511C2160137096
:1001D800A96881F3100189B220460CF087FE774B9D
:1001E800204619880CF082FE296801F30F0189B2B4
:1001F800204601250CF07AFE2B46284663810FB075
:10020800BDEC048BBDE8F08F042D00F0CF8440F2E4
:10021800D583202D57D040F20584242D00F09084FA
:10022800282D40F0E1800B68DFF8B081644E591C3E
:10023800022221601A70236806275A1C22601F7048
:1002480023680A22591C21601A70236801255A194B
:1002580022601D70B8F8001020460CF047FEB8F870
:10026800021020460CF042FE23685A1922601F70C3
:1002780023685022591921601A70236800225919DD
:1002880021601A70318820460CF030FE71882046B3
:100298000CF02CFE2B46B0E7822D35D0C0F0F7834A
:1002A800A02D00F0E183FE2D40F09E80454D05F124
:1002B800080635F8021B20460CF018FEB542F8D1A6
:1002C80001252B4699E70B683F4D591C6A78216038
:1002D8001A7023682A78591C21601A702368AA7832
:1002E800591C21601A70E98820460CF0FFFD23682C
:1002F8002A79591C21601A7022686979531C0125D2
:1003080023602B46117078E70B68304A2A4D117824
:100318002D4A581C20601970D18820460CF0E6FD43
:10032800244B22681B88FF2B02F10101A8BFFF2381
:1003380021601370A96881F3100189B220460CF07E
:10034800D5FD296801F30F0189B220460CF0CEFDD6
:100358001F4B22681978D1E7DFF884801D4F1E4EA5
:10036800DFF880A008F10D090A2516E0322D00F00B
:100378003D83A5F13C00C0B2132840F23D83002321
:100388002268511C216015702268C84502F10101DC
:100398002160137094D018F8015B0A2DE6D1BAF8E1
:1003A8000030FF2BA8BFFF23DBB2E9E70A68002172
:1003B800A4E700BF303E0020BC5B00205035002081
:1003C800C82800205C3D0020E05E0020423E00205E
:1003D800405D002067666666E0280020A46400206F
:1003E80099B1020810290020A5F10A03E72B00F2B1
:1003F800EA80DFE813F0E506E800E800E800E80036
:10040800E800E800E800E800E800E800E800E800A4
:10041800E800E800E800E800E800E800E800E80094
:10042800E800E800E800B406E800E800E800A306F1
:10043800E800E800E8009E06E8005D06E800E8003D
:10044800E800E800E8002606E8000006E800ED05F8
:10045800E800E800E8004A045A07E8005007E80006
:10046800E8004707E800E800E800E800E8003D0485
:10047800E800E800E800E8002B07E8000907E800C2
:10048800F7069008E800E800E800E800E800E8005F
:10049800E8003B08E8001008E800E107E800A808C1
:1004A800E8007F08E800E800E800E800960763072E
:1004B800E405BC05AA05E800E80091058505E80003
:1004C8004B052E05E800E800E800E8002205E800F2
:1004D800E8000005E800E800E800EF04D604C504D9
:1004E800E800E800E800E8008A04E800E800E8001E
:1004F800E800E800E800E800E800E800E800E800B4
:10050800E800E800E800E800E800E800E8009607EE
:10051800E800E800E800E800E800E800E800E80093
:10052800E800E800E800E800E800E800E800E80083
:10053800E800E800E800E800E800E800E800E80073
:10054800E800E800E800E800E800E800E800E80063
:10055800E800E800E800E800E800E800E800E80053
:10056800E800E800E800E800E800E800E800E80043
:10057800E800E800E800E800E800E800E800E80033
:10058800E800E800E800E800E800E800E800E80023
:10059800E800E800E800E800E800E800E800E80013
:1005A800E800E800E800E800E800E800E800E80003
:1005B800E800E800E800E800E800E800E800E800F3
:1005C800E8007D045204742DD8F8003000F026832A
:1005D800772D00F01383292D00F03283392D01F097
:1005E800E485212D01F0BA85D8F804600B3DF61A90
:1005F800EF2D01F2C08301A252F825F0691B000813
:100608007F1D00087F1D00087F1D00087F1D000852
:100618007F1D00087F1D00087F1D00087F1D000842
:100628007F1D00087F1D00087F1D00087F1D000832
:100638007F1D00087F1D00087F1D00087F1D000822
:100648007F1D00087F1D00087F1D00087F1D000812
:100658007F1D00087F1D00087F1D0008FB1A000889
:100668007F1D0008E11A00087F1D0008BF1A000856
:100678007F1D00087F1D00087F1D0008AB1A0008B9
:100688007F1D00083F1E00087F1D00087F1D000811
:100698007F1D00087F1D00087F1D00082F1E000811
:1006A8007F1D0008D11D00087F1D00083B1D0008A4
:1006B8007F1D00087F1D00087F1D00087F1D0008A2
:1006C800C90200087F1D00081B1D00087F1D0008C7
:1006D8007F1D0008FF1C00087F1D00087F1D000803
:1006E8007F1D00087F1D00087F1D00087F1D000872
:1006F8007F1D00087F1D00087F1D00087F1D000862
:10070800B31C00087F1D0008651C00087F1D000839
:100718007F1D00087B1F00087F1D00087F1D000843
:100728007F1D00087F1D00087F1D00087F1D000831
:100738007F1D0008D51900087F1D0008F51E000858
:100748007F1D0008571900087F1D0008F7180008CA
:100758007F1D0008C91800087F1D00087F1D0008BC
:100768007F1D00087F1D00087F1D00087F1D0008F1
:100778007F1D00087F1D00087F1D00087F1D0008E1
:100788007F1D00087F1D00087F1D00087F1D0008D1
:100798007F1D00087F1D00087F1D00087F1D0008C1
:1007A8007F1D00087F1D00087F1D00087F1D0008B1
:1007B8007F1D00087F1D00087F1D00087F1D0008A1
:1007C8007F1D00087F1D00087F1D00087F1D000891
:1007D8007F1D00087F1D00087F1D00087F1D000881
:1007E8007F1D00087F1D00087F1D00087F1D000871
:1007F8007F1D00087F1D00087F1D00087F1D000861
:100808007F1D00087F1D00087F1D00087F1D000850
:100818007F1D00087F1D00087F1D00087F1D000840
:100828007F1D00087F1D00087F1D00087F1D000830
:100838007F1D00087F1D00087F1D00087F1D000820
:100848007F1D00087F1D00087F1D00087F1D000810
:100858007F1D00087F1D00087F1D00087F1D000800
:100868007F1D00087F1D00087F1D00087F1D0008F0
:100878007F1D00087F1D00087F1D00087F1D0008E0
:100888007F1D00087F1D00087F1D00087F1D0008D0
:100898007F1D00087F1D00087F1D00087F1D0008C0
:1008A8007F1D00087F1D00087F1D00087F1D0008B0
:1008B8007F1D00087F1D00087F1D00087F1D0008A0
:1008C8007F1D00087F1D00087F1D00087F1D000890
:1008D8007F1D00087F1D00087F1D00087F1D000880
:1008E8007F1D00087F1D00087F1D00087F1D000870
:1008F8006F1800087F1D0008311800087F1D0008C8
:10090800BB1B0008A11B0008491C00087F1D00082C
:10091800171800087F1D0008ED1700087F1D000844
:100928008D1700087F1D0008651700087F1D000847
:100938007F1D0008431700084716000833160008F3
:10094800051600087F1D0008E31500087F1D000834
:100958007F1D00087F1D00087F1D00087F1D0008FF
:100968007F1D00087F1D00087F1D00087F1D0008EF
:100978007F1D00087F1D00087F1D00087F1D0008DF
:100988007F1D00087F1D00087F1D00080F17000845
:100998007F1D00087F1D0008A51600087F1D0008A0
:1009A8007F1D00087F1D00087F1D00087F1D0008AF
:1009B8007F1D00087F1D000829170008022D00F080
:1009C800148100F20081012D7FF40EAD0B68002226
:1009D800591C21601A7023685A1C22601D702268F5
:1009E8002421531C23602B46117006E43388FF2B07
:1009F800A8BFFF23DBB2C3E417F0F0FD00283FF4E3
:100A0800BEAC03780A2B00F21981B0F9023087FBDB
:100A18000312DB17C3EBA2039BB2FF2BA8BFFF2374
:100A2800DBB2ADE4052D7FF4DFAC0B22BF492046D5
:100A38000CF02CFA0822BE4920460CF027FA0125B2
:100A48000722BC4920460CF021FA2B46FFF7D5BBFC
:100A5800442D7FF4C9AC002A3FF432ACB64B136086
:100A680001252B46FFF7C9BBB44B084619680CF0A3
:100A780025FAB34B204619680CF020FAB14B1968D7
:100A8800204601250CF01AFA2B46FFF7B6BBDFF813
:100A9800EC92AD4F09F10E064FF00A081DE0B8F1CF
:100AA800500F32D0B8F1320F33D0A8F13C00C0B2A9
:100AB800132831D90025294623685A1C226020466C
:100AC80083F800800CF012FA294620460CF00EFA42
:100AD800B1453FF4F5AB19F8018BB8F10A0FDED137
:100AE8009A4B9D68196805EB85054FF6FF736D00F5
:100AF8009D42A8BF1D469942A8BF194625EAE5753B
:100B080021EAE171ADB289B2D6E7914A95681168D8
:100B1800E9E797E82200E6E717F060FD0028C9D06A
:100B280003780A2BC6D8B0F90430B0F9061003EBE5
:100B3800830383F3500521EAE171ADB289B2BBE7C3
:100B4800844B9CE70B6800215A1C226019702268AC
:100B58000125531923602B461170FFF74EBB0A6815
:100B68007D4B0125511C2160157022680521501903
:100B78002060117022680A215019206011702268C3
:100B880000215019206011702268197850192060CE
:100B9800117022685978501920601170226899786C
:100BA800531923602B461170FFF727BB2A466B4960
:100BB80020460CF06BF9002120460CF097F92268CA
:100BC8000021FFF79BBB0B680222591C21601A7099
:100BD800236801255A1922601D70226800215319C3
:100BE80023602B461170FFF708BB04225C4920469E
:100BF80001250CF04BF92B46FFF7FFBAD8F8042073
:100C08009A421EBF5A1CC8F800201978554A08BFD6
:100C18000021204622F020FEFFF752BBD8F804201E
:100C28009A421EBF5A1CC8F8002019784E4A08BFBD
:100C38000021204622F010FEFFF742BB0023EFE61A
:100C48005A1CC8F800201B780A2B01F01383502B7C
:100C580041F0918040460CF00DF9444E30804046FA
:100C68000CF008F94FF0FF3570802B46FFF7C5BA36
:100C7800236800255A1C2260294620461D700CF066
:100C88001DF9294620460CF019F9002120460125B6
:100C98000CF014F92B46FFF7B0BA354B03F1700589
:100CA80022681978501C2060117022685978501CED
:100CB8002060117022689978501C20601170226899
:100CC800D978501C2060117022681979501C206056
:100CD800117022685979501C206011702268997926
:100CE8000733501C9D4220601170D9D1FFF7E8BA34
:100CF800204D2046A9890CF0F9F86989204601257C
:100D08000CF0F4F82B46FFF778BA1B4D2046A98A59
:100D18000CF0ECF8E98A20460CF0E8F8298B20461C
:100D280001250CF0E3F82B46FFF767BA3CD7020819
:100D380048D7020854D7020825370208ACF7FF1F26
:100D4800B0F7FF1FB4F7FF1FD82800208C28002019
:100D5800CC280020DC640020DB5E002034D70208A9
:100D68002CD702083D360208FD360208C8280020A4
:100D78007C460020B4640020683E002089B1020847
:100D88002368B24AB2491078B24A5D1C25601870CF
:100D980023689278581C20601A7022688978FFF7B7
:100DA800ADBA2268AC4BAD491878551C2560107057
:100DB80022685878551C2560107022689B78501C52
:100DC80020601370C988204601250CF08FF82B4647
:100DD800FFF713BAA14D204629880CF087F86988D7
:100DE80020460CF083F8A988204601250CF07EF8EF
:100DF8002B46FFF702BA9A4D05F16006A9882046EE
:100E08000CF074F8E98820460CF070F8298920461F
:100E18000CF06CF82368AA7A591C21601A702368B0
:100E2800EA7A591C21601A7055F80C1B20460CF000
:100E380045F8B542E2D1FFF743BA8A4952232268FE
:100E4800501C2060137011F8013F002BF7D1FFF7F9
:100E580037BA854D00232268286803EB4301561CE6
:100E6800405C266010702A6820680A44461C527844
:100E7800266002702A6820680A4401339278411C6F
:100E88000A2B21600270E6D1FFF71ABA774D236862
:100E98002A68591C127821601A702B682268997880
:100EA800531C2360002311702A6821681A440133F7
:100EB8005279481C032B20600A70F5D123682A68F0
:100EC800591C127A21601A7023682A68591CD27832
:100ED80021601A7023682A68591C127921601A70D7
:100EE8002B68204659890CF001F823682A68591C98
:100EF800527A21601A702B6822685978FFF7FEB978
:100F0800002120460BF0DAFF0125002120460BF0D6
:100F1800EDFF2B46FFF771B9554D204629880BF098
:100F2800E5FF698820460BF0E1FFB5F90430514927
:100F3800DA1781FB0313C2EBA30399B220460125FC
:100F48000BF0D4FF2B46FFF758B94B4E3378002BE4
:100F58003FF4B6A9494F002537F8021F20460BF089
:100F6800C5FF337801359D42F6DBFFF7A9B9444D3B
:100F7800444EDFF83481DFF83491DFED438ADFED4A
:100F8800439A9FED439A05F1200708E0204604356F
:100F98000BF0ACFFBD4206F118063FF491A9717C35
:100FA8000029F3D095ED008AB0EE480A27F004FF37
:100FB80098F80030002B41F01D8181B2E6E710223D
:100FC8003449204601250BF061FF2B46FFF715B980
:100FD800314D324E05F1300795F902100023F256D3
:100FE8008A4200F0E3870C33482BF8D10835BD421C
:100FF800F2D1FFF765B92A4B03F15A0522685979EE
:10100800501C2060117022681978501C20601170E3
:1010180022685978501C2060117022689978501CF9
:10102800206011702268D978501C206011702268E5
:1010380019790633501C9D4220601170DED1FFF7EC
:101048003FB9184B2268597DFFF758B9084A002064
:10105800CC640020B4640020AC640020E03C002094
:101068003C48002058B10208F05E0020207500209E
:10107800B060002067666666B86000207E71002058
:1010880064350020DC5600200000404200407444D3
:1010980000E08244543500202C740020AC65002008
:1010A800705D0020FC420020903E0020504300204C
:1010B800B04D23682A7A591C21601A70A98B2046E2
:1010C8000BF014FF298B20460BF010FF698B20468C
:1010D8000BF00CFF2368EA7C591C21601A70E98C1C
:1010E80020460BF003FF298D20460BF0FFFE2368F6
:1010F800AA7F591C21601A70236895F82020591C72
:1011080021601A70A98C20460BF0F0FE2368EA7A59
:10111800591C21601A70E96820460BF0CFFE23683D
:101128002A7C591C21601A70226895F82110FFF753
:10113800E5B8914B22681978FFF7E0B88F4D204643
:1011480029880BF0D3FEA98820460BF0CFFE298909
:10115800204601250BF0CAFE2B46FFF74EB8884DF6
:10116800884F05F1500600212878874A0B4607E08A
:101178000133242B02F10C0200F0158712F80C1C25
:101188008842F5D103EB4303226807EB8303511C24
:1011980093F864302160137023686A78591C2160C1
:1011A8001A702368AA78591C21601A702368EA7893
:1011B8000435591CAE4221601A70D4D1FFF780B8AB
:1011C800724826F0DFFE00287FF77AA86F4B1D18BB
:1011D800226813F8011B501C9D4220601170F7D142
:1011E800FFF76EB8236800255A1C22601D7023681B
:1011F8005A1C22601D7023685A1C226029461D70E3
:1012080020460BF05BFE40E5614E3378002B3FF43F
:1012180057A8604F0025B846236817F81520591CB1
:1012280021601A7098F8011001EB810101EB81012E
:1012380001F2EE2189B220460BF058FE33780135D1
:101248009D4208F10208E7DBFFF73AB82368524DE0
:10125800591C2A7821601A7023686A78591C216001
:101268001A70698820460BF041FE23682A79591CB8
:1012780021601A70E98820460BF038FE2268297A26
:10128800FFF73CB808223B49204601250BF0FEFD3C
:101298002B46FEF7B2BF2268404B501C997820605D
:1012A800117022685978FFF729B82268012153186C
:1012B80023600D460B461170FEF79FBF384E338AE8
:1012C800B3F5007F06F1340594BF012704274036A3
:1012D80055F8041B91FBF7F1204689B20BF006FE86
:1012E800AE42F5D12F4D304F05F10C06B5EC010A91
:1012F800D7ED087A80EE270A27F05EFD81B22046F6
:101308000BF0F4FDB542F1D1284D05F10C0655F866
:10131800041B204689B20BF0E9FDB542F7D1FEF770
:10132800CFBF0DF1140900220592DFF888A0204BE9
:1013380003920492C9F80420904601214FF6FF7BDE
:1013480007E008F10108B8F10B0F00F04D861AF913
:10135800011F4E1CF5D04BFA08F2D007F1D51A88B8
:1013680042FA08F2D207ECD5484601930BF0E2FFA7
:10137800019BE6E7FC420020B0350020545D0020C8
:10138800B435002058B10208C0B102082C60002012
:10139800B860002050490020F43C0020D8640020A8
:1013A8006C600020445200201C4A0020143D00209C
:1013B800F81C0020A8B10208AE4D23686A79AE4E29
:1013C800591C21601A7033682046198C0BF08EFD69
:1013D80033682046598C0BF089FD698920460BF04B
:1013E80085FDA98920460BF081FD33682046998C3C
:1013F8000BF07CFD33682046D98C0BF077FDE9892A
:1014080020460BF073FD298A204601250BF06EFD5E
:101418002B46FEF7F2BE974EF378002B00F0DD86E0
:1014280023680822591C21601A7023680122991820
:1014380021601A702368914D591C2A7921601A700D
:101448002368AA78591C21601A70298820460BF055
:101458004DFD698A20460BF049FD2368F279591C35
:1014680021601A702268E978FEF748BF20F0B8F9C1
:10147800FF28064600F0E6860EA9002501F82E5D35
:101488000DF109008DF8095023F0F6F80EA800F8C0
:101498002D5D23F0E5F80EA800F82C5D23F0D4F8B4
:1014A8000EA820F8245D20F07BF923685A1C2260DE
:1014B8001E7023689DF80920591C21601A70236842
:1014C8009DF80A20591C21601A7023689DF80B208A
:1014D800591C21601A7023689DF80C20591C216042
:1014E8001A70BDF81410204601250BF0FFFC2B469E
:1014F800FEF783BE2368624A6249D078624A5D1C5F
:101508002560187023681278581C20601A702268A9
:10151800C978FEF7F3BE22685C4B0125511C216097
:10152800157022689978501920601170226819780E
:1015380050192060117022685978531923602B467E
:101548001170FEF75ABE002120460BF0CFFC002197
:1015580020460BF0CBFC002120460BF0C7FC22688C
:10156800454D0023511C2160137022682968501CC6
:1015780091F82F102060117022682968501C91F88A
:101588003A102060117022682968501C91F83B10AD
:10159800206011702268511C216013702268511C50
:1015A800216013702268511C216013702B6820463B
:1015B800D98F0BF09BFC2B682046998F0BF096FC7B
:1015C80023682A68591C92F8312021601A702B6808
:1015D800226893F83210FEF791BE40460BF04AFCA1
:1015E800264EB08240460BF045FCF08240460BF098
:1015F80041FC012530832B46FEF7FFBD1A46591CD6
:10160800C8F800101B4912F8020B0870C8F800202F
:101618001B495A788A70DA1CC8F80020194A9B7846
:10162800937001252B46FEF7E8BD134B184918683F
:101638004A22012529F0B3FC2B46FEF7DEBD1946E8
:101648005A1CC8F80020134A11F8020B1070C8F889
:10165800001059785170D91CC8F800109B78937005
:1016680040460BF007FC0C4B0125D8802B46FEF7B3
:10167800C4BD00BF084A0020F05E0020683E00207C
:10168800B4640020CC640020C46400205D600020A5
:10169800BCBB0208AC640020E03C00205A1CC8F81F
:1016A80000201A780F2A00F26683991CC8F80010E7
:1016B800C2EBC202B74958788854D81CC8F8000051
:1016C8000A4499785170191DC8F80010D97891709A
:1016D800591DC8F800101979D170991DC8F8001063
:1016E80059791171D91DC8F800109979517103F110
:1016F8000801C8F80010DB799371012519F0FAFC8C
:101708002B46FEF77ABD40460BF0B4FBA24EB081E3
:1017180040460BF0AFFB012570812B46FEF76DBDEF
:101728009E4B1B78DB0700F12683012522F038F950
:1017380022F0D6F92B46FEF760BD40460BF09AFB27
:10174800974E308040460BF095FB708040460BF07A
:1017580091FB0125B0802B46FEF74FBD914F3B789A
:10176800002B3EF4ADAD904E002540460BF082FBB9
:1017780015F068F93B78A6EC010A01359D42F4DBC7
:10178800FEF79EBD0F2E40F0F6825A1CC8F80020C6
:101798001D78072D00F2EF82844F40460C260BF08F
:1017A80069FB06FB05F6BD19A88040460BF062FBF5
:1017B800E88040460BF05EFBD8F8003028811A46D6
:1017C800591CC8F8001012F8021BA972C8F80020AA
:1017D8005B78EB7240460BF035FB0125B8512B4680
:1017E800FEF70BBD5A1CC8F800201878060600F151
:1017F800BB856A4B1B78DD073EF562AD032828BF21
:101808000020012522F0B0F82B46FEF7F6BC634B0A
:101818001B78D8073EF554AD012522F03DFB22F098
:101828005FF92B46FEF7E9BC614A1068DA1C0146ED
:101838002133951EC8F8005012F8035C0D70551E30
:10184800C8F8005012F8025C4D70C8F8002012F871
:10185800015C8D700332934201F10301E9D119F063
:101868002BFEFEF72DBDC6F34706122E00F283822B
:10187800B6B10EAB0DF1120903EB46054F46263DF6
:1018880040460BF0F7FA27F8020FBD42F8D1494B52
:1018980039F8022F23F8022F4F45F9D1112E09D814
:1018A800454A7300023B13440021223223F8021FE9
:1018B8009A42FBD1414A01231D461370FEF79DBC95
:1018C8001A46591CC8F80010334912F8020BC870A0
:1018D800C8F800203A495A780A70DA1CC8F800207B
:1018E800384A9B78D37001252B46FEF786BC4046C4
:1018F8000BF0C0FA40460BF0BDFA40460BF0BAFABE
:10190800D8F800302A4D9A1C2F68C8F800205A7859
:1019180087F82F20DA1CC8F800209A7887F83A2030
:101928001A1DC8F80020DA7887F83B200733C8F872
:10193800003040460BF09EFAF88740462F680BF0BF
:1019480099FA112EB88700F2FD84286887E75A1C97
:10195800C8F80020164D1C4F1B78D5F800907B71F5
:1019680040460BF087FAA9F820004046D5F80090C9
:101978000BF080FA052EA9F8220000F2118522F05A
:1019880019F81AF017FD2868012514F093FE2B4664
:10199800FEF733BC7C460020B4640020855B002041
:1019A800E03C0020493D0020E83B00203C48002066
:1019B800F05E0020C6430020C8430020EC4300200E
:1019C800C4640020CC640020084A002040460BF084
:1019D80051FA05461FF004FFFF283EF471ACB5F537
:1019E8007A7F80F097840DF13809002309F8243DA7
:1019F800EE08494603A88DF80C30013622F03CFE6B
:101A08009DF80C30F6B205F00705B34205F1010563
:101A180003D19DF81430AB4203D0294630461FF05D
:101A2800CBFED8F80030D8F80420D21A012A7EF765
:101A380047AC5A1C0EA8C8F8002000221D7800F8F0
:101A48002C2D22F00DFE9DF80C30AB420AD0CC4B69
:101A58001B683BB19A79AA4204D31B681B690BB176
:101A680028469847D8F800305A1CC8F8002048463D
:101A780000221D788DF8142022F0E6FD9DF8143020
:101A8800AB423EF41DACBE4B1B68002B3EF418ACB9
:101A98001B685B69002B3EF413AC28469847FEF799
:101AA8000FBC5A1CC8F80020B64A1B7813700125D1
:101AB8002B46FEF7A2BB40460BF0DCF9B24E306075
:101AC80040460BF0D7F9706040460BF0D3F901257A
:101AD800B0602B46FEF791BBAC4E00233360404606
:101AE8000BF0B0F933680125034333602B46FEF74A
:101AF80084BB5A1CC8F800201878132800F23B81D0
:101B08009A1CC8F800205D78A14A002105E001313F
:101B1800242902F10C0200F02E81167AAE42F6D189
:101B28009C4D9D4A0C2606FB0151DD1C91F85C106A
:101B380002F82010C8F8005002EB80029978517022
:101B4800191DC8F80010D8789070581DC8F8000002
:101B580092491B790868D37012F074FCFEF7B0BB89
:101B68008F4B102E4FF0000228BF10261A605A60C3
:101B78009A60DA601A74002E3EF4A2ABD8F80020FE
:101B880016440132C8F8002012F8011C03F8011BA2
:101B98009642F6D1FEF794BB824B1B78D9073EF5E7
:101BA8008FAB814B4FF4C87201251A802B46FEF784
:101BB80024BB092E40F2DF807C4F1A46591C3D6831
:101BC800C8F8001012F8021B2970C8F800205A78CB
:101BD800AA70DA1CC8F800209A78642A03F1040174
:101BE800A8BF64226A71C8F80010DA78642A03F181
:101BF8000501A8BF6422AA71C8F800101A79EA7111
:101C08009A1DC8F800205A79642A28BF6422D91D71
:101C18002A72C8F800109A79EA7003F10802C8F825
:101C28000020DB792B7140460BF024F90A2E6881DD
:101C380040F0A583012525F0E1FE2B46FEF7DDBA2D
:101C4800584B1B78DA073EF53BAB594A1378012508
:101C580043F0040313702B46FEF7CFBA5A1CC8F89A
:101C680000201E78112E00F286809A1CC8F80020E9
:101C7800504D5B7805F8163040460BF0FBF840F6FF
:101C8800CA039842A8BF184640F2EE23984205EBD3
:101C98004601B8BF18460125A0F2EE222B461920AE
:101CA80092FBF0F24A70FEF7A8BA1A46591C424D48
:101CB800C8F8001012F8021B2970C8F800205B78D9
:101CC8006B7040460BF0D6F8D8F8003068805A1C84
:101CD800C8F800201B782B7140460BF0CBF8D8F8D9
:101CE8000030E8805A1CC8F800201B782B720125A8
:101CF8002B46FEF782BA314A03F108010133C8F8CE
:101D0800003013F8010C02F8010F9942F6D1FEF7E2
:101D1800D7BA591C1A46C8F80010294912F8020BFC
:101D28008870C8F800205B784B7001252B46FEF7B9
:101D380064BA0722B6FBF2F2C2EBC201711A1AD1D9
:101D4800D2B2571EFFB2002A3EF4BAAADFF8749046
:101D580001378A465A1CC8F8002093F90010194B1D
:101D6800002593F902208A4200F0AA820135062D47
:101D780003F10803F5D14FF0FF352B46FEF73DBAC6
:101D8800A8650020B0350020545D0020DC640020E8
:101D9800B4B1020858B10208B4350020F05E002042
:101DA8002C600020855B00203C75002020750020F9
:101DB8001036002050490020F43C0020FB4200204F
:101DC800D86400202C7400205A1CC8F800201A7807
:101DD8000E2AD0D8991CC8F800105D78032DCAD8EF
:101DE800CF48062101FB02F14218DE1C5571C8F8E4
:101DF80000609D784554191DC8F80010D9785170B5
:101E0800591DC8F8001019799170991DC8F800106B
:101E18005979D170D91DC8F800109B791371012523
:101E28002B46FEF7EAB95A1CC8F80020BD4A1B78B1
:101E38005375FEF745BA5A1CC8F80020B94D1B78EF
:101E48002B7240460BF016F8A88340460BF012F8A8
:101E5800288340460BF00EF8D8F8003068835A1CE7
:101E6800C8F800201B78EB74082E7EF629AA404695
:101E78000BF000F8E88440460AF0FCFF0C2E288599
:101E88007EF61EAAD8F800301A46591CC8F8001069
:101E980012F8021BA977C8F800205B7885F8203073
:101EA80040460AF0E7FF102EA8847EF609AAD8F863
:101EB80000305A1CC8F800201B78EB7240460AF024
:101EC800C1FFD8F80030E8605A1CC8F800201A781A
:101ED8002A74162E7EF6F4A99A1CC8F800205B789E
:101EE80085F8213001252B46FEF787B91A46591C7B
:101EF800C8F800108C4E12F8021BB170C8F8002008
:101F08008A495A780A70DA1CC8F80020884D9A78ED
:101F18002A711A1DC8F80020DB78092BA8BF0923ED
:101F28004046AB700AF0A6FFD8F80030D8F8042075
:101F38002880D11A012907DD40460AF09BFFD8F80E
:101F48000030D8F8042068829A4240F04C8221F090
:101F580031FDD8F80030D8F804209A423EF4B0A9F0
:101F68005A1CC8F800201B78EB7001252B46FEF799
:101F780044B9704A1278012A3EF6A2A919465A1C99
:101F8800C8F800206C4A11F8020B9070C8F80010CD
:101F980059781170D91CC8F800109B785370012526
:101FA8002B46FEF72AB900231B7AFFDE23685A1C4A
:101FB80022601970298820460AF098FF2368EA7879
:101FC800591C21601A7023682A79591C21601A70DB
:101FD8002368AA79591C21601A7023686A79591CE8
:101FE80021601A70FFF702B8DFF86CB14FF00008F3
:101FF8004FF0080A08F10108B8F1240F1BD0C8F106
:1020080020020AFA02F22BFA08F6A8F12003164376
:102018002AFA03F31E4306F0010200231343E9D012
:102028005FFA88F012F008FA0028E3D041464846E3
:102038000BF080F9DEE7414B1B78DF0700F10A81DE
:1020480000263F4FB04602E00136242E0ED031461E
:1020580038460BF07FF90028F6D0314648460BF099
:1020680079F9002856D108F10108EDE7354B364ECD
:10207800B3F8501020460AF039FF344B198820462F
:1020880089B20AF033FF324B1A68530103F020017A
:10209800C2F340030B43C2F3800143EA4103C2F396
:1020A800C00143EA8103C2F3401143EAC10102F0CF
:1020B8001002114320460AF019FF03A90422204602
:1020C8000AF0E4FE23683178224A581C206019700F
:1020D80011886429A8BF642120460AF007FF962DBD
:1020E80000F0BD80002120460AF000FF2168B8F109
:1020F800190348BFA8F11203A3F3C4034A1C2260C2
:1021080020460B701A4604A901250AF0BFFE2B468B
:10211800FEF773B8414603A80BF00CF9A3E700BF1C
:10212800705D0020FC420020084A0020A8640020BE
:10213800683E0020686000205D600020855B00200C
:10214800DC1B0020B814002028600020B8620020A2
:1021580050520020445D002090E33FF41A46591C79
:10216800C8F80010A44D12F8021B6970C8F80020C6
:102178005A782A70DA1CC8F800209B78AB70404661
:102188000AF078FED8F80030E880591C1A46C8F8DA
:10219800001012F8021B2971C8F800205B786B71D7
:1021A8004FF0FF352B46FEF728B85A1CC8F8002018
:1021B8001A780A2A7FF4DFAD9A1CC8F800208F4AE3
:1021C80059781170D91CC8F8001099785170191DE8
:1021D800C8F80010DB789370CDE52368B178884A99
:1021E800581C2060197023681278591C21601A70D5
:1021F800FFF720B9D9F8003013F48053B4EEE88A19
:102208003ED0F1EE10FA11DBB4EEC98AF1EE10FA05
:1022180039D8DFED7C7A9FED7C7A77EEC87AB4EE18
:10222800C78AF1EE10FAB0EE678A2CD94FF47A71AA
:10223800B5EE408AF1EE10FA40F2DC5308BF1946B9
:10224800FEF7A4BE22680125531923602B4610709F
:10225800FDF7D3BF059B43F001030593F0E6236820
:102268000322591C21601A7023687278591C216056
:102278001A703BE740460AF0FDFD644EFEF7EEBCDF
:10228800F1EE10FA42DBF7EE007A78EE677AB6EEF6
:10229800007AF0EE696AE7EE876A40F2E932FDEE0D
:1022A800E67A17EE901AB1F5FA6FA8BF4FF4FA6103
:1022B8009142B8BF114689B2002B3EF467AEB7E72A
:1022C80009EBC5064046B1700AF0D4FDD8F80020E5
:1022D80029F835001346511CC8F8001013F8021BE2
:1022E800F170C8F8003053783371D31CC8F8003047
:1022F8009378B371131DC8F800300AF1010AD27837
:10230800727157457FF426ADFDF7DABF4FF47A7145
:10231800FEF73CBE0DF1140948461FF041FABDF81E
:102328001430AB423FF47DAB394B1B68002B3FF4B4
:1023380078AB1B689B69002B3FF473AB2846984722
:10234800FFF76FBBD8F800302968581C1A46C8F840
:10235800000012F8020B81F83100C8F800205B7801
:1023680081F83230FFF7F1BA00F07F00032828BF68
:102378000020012524F0D2F82B46FDF73EBFD8F8FF
:1023880000303A68591CC8F80010197851720B2EA1
:102398003FF450AC991CC8F800105B78537049E4BE
:1023A80040460AF067FD788140460AF063FDB8812F
:1023B8004046D5F800900AF05DFDA9F82400404693
:1023C800D5F800900AF056FD0D2EA9F826007FF6E4
:1023D800D6AA40460AF04EFDF88140460AF04AFD6A
:1023E8003882FFF7CCBA5A1CC8F800201B78003393
:1023F80018BF0123F371AAE5E05E0020DB5E002030
:10240800A864002000C0884400C08244A46400205E
:10241800A86500202DE9F04FDFF810B12DED0C8BE9
:102428009BF800309FB0012B089002F035853A4C9C
:1024380094F80021002A41F09784072B374D02F0C9
:10244800B184002306936B683448984700286FD0FE
:10245800B5F8A880002285F84920B8F1000F40F0AF
:102468009882B5F92460E96AB5F926002A6BB5F9AE
:102478002830711AA9632A490591821A686BEA63A0
:102488000E461B1A95F84A1026482B6413F0AAFC2E
:10249800336813F0005302F0A384D5ED0F5AD5ED3D
:1024A8000E7A214A94ED666AD4ED676A94ED687AEB
:1024B800D4F8A4311268B8EEE58AD5ED105AF8EED2
:1024C800E77AF8EEE58A013377EE867A38EE268ADF
:1024D80078EE878A9342C4ED667A84ED678AC4ED04
:1024E800688AC4F8A43101F0BF879BF80080B8F16E
:1024F800140F03F09C840023D4F8AC610793062ED4
:1025080002F24885DFE816F0C2199019E614781B24
:10251800E21BEE1A861A00BFE41B00201C4A0020AA
:1025280050430020544A002054520020593D0020B6
:102538009BF80090B9F1070F00F0E58294F8BC31E0
:102548000A93002B40F0EB82D54B5B79002B40F0CF
:102558001B8201239BF8002084F8BC31072A02F073
:10256800DD8500230D93CF4BD4ED719A93ED007A5E
:10257800CD4ADFF8ACA3CD4B1268DFF8A8830993E6
:10258800F7EE007A37EEE98A069228EE078AC84AFB
:102598000593B4EEE78A53460025F1EE10FAD4ED20
:1025A800708ADFF88493DFEDC3AA9FEDC39A9FED8D
:1025B800C3BADFEDC3CA9FEDC3AADFEDC3BAC34FE9
:1025C8000792C24688BFB0EE678A2E469846C04B2F
:1025D8002B44D3ED007ABF4BF5EE407A2B44F1EE55
:1025E80010FA93ED00CA17D0BB4B2B4493ED007A39
:1025F8007CEE476AB0EEE66AF4EEC67AF1EE10FABF
:1026080008D5F5EEC06AF1EE10FACCBF37EE87CAEE
:1026180037EE67CA83ED00CAB4F814E11EF0030F61
:1026280000F08582022E05F084840699AB4B91F860
:10263800322007EE102A91F831202B44D3ED006A9E
:102648005342B8EEC77A07EE903A27EE267AF8EEAC
:10265800E77AB4EEE77AF1EE10FA0AD407EE902A98
:10266800F8EE677AF4EEC77AF1EE10FA88BFF0EE6A
:10267800477A9B4B0B939B4A03EB460332F91610A0
:10268800B3F90A30C81A07EE100AB8EEC77A1EF076
:10269800010FE7EE497A00F0BB82DFF890E29EED89
:1026A80000CA27EE8CCA94F8D4E1BEF1000F1FD0FF
:1026B800DFF878E2D4F8D8019EED00CADFF870E2BE
:1026C8005B1A07EE903A089BDEF800102CEE09CA58
:1026D800F8EEE77A1B1A8B422CEE27CA01F3178310
:1026E800F7EE007AF4EEE79AF1EE10FA01F1DA82E9
:1026F8007D4B2B44D3ED007A059BD3ED01DA68EED0
:10270800A77A3CEE6DDA67EE8D7AC8ED007A079B02
:10271800D9ED006A93ED007A744BD7ED007A26EE76
:10272800877A2B4467EE086A93ED007A26EE877A5B
:10273800F0EE676AE7EE0D6AB0EE667A94ED716ABC
:10274800F7EE006AB4EEE66AF1EE10FAACBF0123C8
:10275800002343B1F0EEE77AF0EEC76AF4EEE76AD9
:10276800F1EE10FA01D587ED007A022E05F0A88364
:102778005F4A604B52F826001B68B0EE6D0A984716
:102788005D4A5E4B52F826001B689847069B93F8F3
:102798003A30632B04D8B4F81431002B01F0C98205
:1027A800F0EE6C7A564B99ED007A37EEC00A2B445E
:1027B800D3ED007A83ED000A069B30EE670A93F8A2
:1027C800482080EE07CADAB1F7EE007AF4EEE79A0D
:1027D800F1EE10FA14DB4B4BD3ED007AB0EECC7A65
:1027E800B4EEE77AF1EE10FA0ADD474BD3ED007A42
:1027F800B0EECDDAB4EEE7DAF1EE10FA01F3B88311
:10280800424B94F8E4212B44D3ED007A68EEA77A82
:1028180027EE8CCA8AED00CA2AB9C8ED00CAC7EDEE
:1028280000CACAED00CA059B043504330C2D06F115
:1028380001060AF1040A08F1040807F104070593E0
:102848007FF4C5AE9BF80030072B02F0B983012B4B
:1028580002F05484002309932D4B05931A46124B1A
:1028680012681B680792114693F82F2011F48053C1
:102878000B9300F05982274B08931B78DFF8B4A01C
:1028880013F0010F244B0693198B244B9AED037A0E
:10289800DB8808BFA4F8EC11C81A07EE900A4BE0D1
:1028A800084A0020BC470020F05E0020405200206B
:1028B8000000002000009642CDCCCC3DAE47813FC1
:1028C800000000000000C8420000344338350020F2
:1028D800B0470020E81C0020AC1D0020541D00203B
:1028E800B4640020B06000206C47002078470020C6
:1028F80008370020043700206C3700206837002094
:10290800C01D0020D0470020CC470020844700206D
:1029180050430020855B0020FC420020E03C002062
:102928002C350020443500206847002098470020B7
:10293800C0470020443E0020F8EEE77AB4EEE77A7C
:10294800F1EE10FA42F25883CD1806EE905AF8EEDE
:10295800E66AB4EEE67AF1EE10FA81F25A85B4F836
:10296800EC31984284F29080994B9A49D3ED003A21
:1029780091ED004A984B84ED7C4AC4ED7D3AD3ED45
:10298800006ADFED967AEBE1954B1B78013BDBB2F1
:10299800E0E5944B9449099391F801A01B68934F83
:1029A8009BF80090B7F906004FF47A71B1FBF3F386
:1029B800C3EB431603EB8603DE00B6B2B04503F063
:1029C8002183E96FB5F924E02B6E4A1C07EE90EAE3
:1029D8007344012AEA672B66F8EEE77A03F01C8352
:1029E800D5ED1B5AD5ED1D6A07EE102A37EEE56ABC
:1029F800B8EEC75AB8F1010F86EE057A37EE257A98
:102A080077EEC77A85ED1C7AE6EE276A85ED1B7AA4
:102A1800F0EE667AC5ED1E6AC5ED1D6A04F0A38066
:102A2800D5F89010B5F926E06B6E4A1C07EE90EACF
:102A38007344012AC5F890206B66F8EEE77A03F034
:102A48000483D5ED205AD5ED226A07EE102A37EE19
:102A5800E56AB8EEC75AB8F1010F86EE057A37EE87
:102A6800257A77EEC77A85ED217AE6EE276A85ED35
:102A7800207AF0EE667AC5ED236AC5ED226A04F085
:102A8800A880D5F8A410B5F928E0AB6E4A1C07EE6B
:102A980090EA7344012AC5F8A420AB66F8EEE77AF9
:102AA80003F0ED82D5ED255AD5ED276A07EE102AF9
:102AB80037EEE56AB8EEC75AB8F1010F86EE057A27
:102AC80037EE257A77EEC77A85ED267AE6EE276A1D
:102AD80085ED257AF0EE667AC5ED286AC5ED276A98
:102AE80004F06A80F880B5F8A8309BF80090013BA4
:102AF800A5F8A83009990023B9F1070F4B608B603E
:102B0800CB607FF41BAD0FF097FA069B374FC01AC6
:102B180094F8BC3138800A93002B3FF415AD013B83
:102B280084F8BC311FB0BDEC0C8BBDE8F08F94F875
:102B3800D43163B1022E05F0EB812D4B0B932D4A56
:102B480003EB460332F91610B3F90A30B0E52A4B05
:102B58002B4493ED000A059BD3ED01DA28EE800A99
:102B68003CEE6DDA022E20EE0D0A88ED000A7FF4A5
:102B7800CEAD224A224B10681B689847079B99EDF7
:102B8800007AD3ED006A1F4BD7ED007A1A781E4BF6
:102B980083ED020A1D4B26EE877A2B4427EE087A2E
:102BA80093ED006A27EE067AF0EE676AE7EE0D6AA3
:102BB800012AB0EE667A02D0192A7FF4BFADB4EECE
:102BC800EADAF1EE10FACCBF01230023C1E500BF19
:102BD800D83C002098640020F03C00200000000051
:102BE800A864002040520020084A00205C3D0020D4
:102BF800B4640020B06000206C470020CC3B00206B
:102C0800E03B0020644700202C3500207847002056
:102C1800B2F900C0D4ED5F6A94ED607AB2F90200AF
:102C28000C908CEAEC70B4EEE67AA0EBEC70F1EE66
:102C380010FA0E900C984BBFB7EE007AF7EE006AC8
:102C480077EE665A76EEC75A0028B8BF40420F9012
:102C58000E9886460F98864541F34881BCF1000FCF
:102C6800D6BFCCF1000007EE10CA07EE100ADFF855
:102C7800A8E0B8EEC77A9EF800E027EE097ABEF120
:102C8800000F01F04581DFF894E09EED005AB5EEA3
:102C9800C05AF1EE10FA42F31181DFF884E0DEED5C
:102CA800004AF5EEC04AF1EE10FA42F3078134EE1D
:102CB800C77AB7EE006AC7EE246A75EEC65AF4EE14
:102CC800C66A65EE8A5AF1EE10FA85EE857A88BFF3
:102CD800F0EE466AF5EEC06AF1EE10FA37EE067AC3
:102CE800B8BFF0EE6C6A66EE876AF4EEC66AF1EE7B
:102CF80010FA88BFF0EE466AF5EEC06AF1EE10FAF7
:102D0800B8BFF0EE6C6ADFF81CE09EED007A67EE63
:102D1800877AA7EEA6CAC6E4A4470020A0470020E9
:102D2800A84700209C470020E74B06935B8BDFF801
:102D3800D4A3E6499AED037A91ED004A07EE903A5A
:102D4800E34B84ED7C4AD3ED003AE24BC4ED7D3A87
:102D5800F8EEE77AD3ED006ADF4B089377EE677AEF
:102D6800C7EEA62ADD49DE4B91ED008ADD49DFED8D
:102D7800DE6A91ED005ADD499FEDDD6AD1ED005A1A
:102D880093ED007AF7EE007AF4EEE72A38EE058A3A
:102D9800F1EE10FA88BFF0EE672A38EE258AF4EED5
:102DA800E62AF1EE10FA28EE066AB8BFF0EE662AB7
:102DB800F1EE476A34EE635AB4EEE66AF1EE10FAC1
:102DC800C4ED7E2A84ED805A00F19185B4EEC76A7D
:102DD800F1EE10FA88BFB0EE476AC04BDFEDC47A57
:102DE800D3ED018ABF4BD3ED014AC04B78EEA48ADC
:102DF800D3ED015A78EEA58A68EEA77AF4EEE76A71
:102E0800F1EE10FA08DCB4EEE77AF1EE10FA8CBFB6
:102E1800F0EE676AF0EE476AB04BDFEDB57A93EDF6
:102E2800029AB04BD3ED025AB24B39EE259A93ED84
:102E3800007A69EE277AF1EE475AF4EEE57AF1EE78
:102E480010FA08D4F4EEC77AF1EE10FA8CBFF0EE5F
:102E5800475AF0EE675A002A41F09183F7EE007A5C
:102E6800A54B5A7894F80432002AA44ABFEE003AD7
:102E7800B7EE007A92F8008014BFB0EE472AB0EEA1
:102E8800432A002B14BFF0EE434AF0EE474AB8F14C
:102E9800000F03F06F81F4EEC77AF1EE10FA65EED9
:102EA800825A974B41F32A8493ED027A93ED011AE3
:102EB800D3ED031A9FED8C2A26EE877A27EEA43AE3
:102EC800A1EE067AA1EEA57A27EE037AB4EEC27ACD
:102ED800F1EE10FAB4BFF0EE427AF0EE477A8DEDDB
:102EE800127A88BFB0EE427AB8F1010F00F0C981BA
:102EF800D3ED064AD3ED051A93ED072A66EEA44AE8
:102F0800E1EE864AE2EE254A64EE834AF4EEC74AC9
:102F1800F1EE10FAF4EEE74A8CBFB0EE472AB0EEB5
:102F2800642AF1EE10FA98BFB0EE427AA8BFF0EE2C
:102F3800647AB8F1020FCDED134A00F0A281D3ED07
:102F48000A4AD3ED091A93ED0B2A66EEA44AE1EE7C
:102F5800864AE2EE254A64EE834AF4EEC74AF1EE69
:102F680010FAF4EEE74A8CBFB0EE472AB0EE642AB6
:102F7800F1EE10FA98BFB0EE427AA8BFF0EE647A8C
:102F8800B8F1030FCDED144A00F07B81D3ED0E4A62
:102F9800D3ED0D1A93ED0F2A66EEA44AE1EE864AA8
:102FA800E2EE254A64EE834AF4EEC74AF1EE10FADF
:102FB800F4EEE74A8CBFB0EE472AB0EE642AF1EE91
:102FC80010FA98BFB0EE427AA8BFF0EE647AB8F172
:102FD800040FCDED154A00F05481D3ED124AD3ED1C
:102FE800111A93ED132A66EEA44AE1EE864AE2EE40
:102FF800254A64EE834AB4EEE47AF1EE10FAF4EE70
:10300800E47A8CBFB0EE642AB0EE472AF1EE10FAEB
:1030180058BFB0EE427AB8BFF0EE647AB8F1050F47
:10302800CDED164A00F02D81D3ED164AD3ED151AD1
:1030380093ED172A66EEA44AE6EE214AE5EE824AA7
:1030480064EE834AF4EEC74AF1EE10FAF4EEE74A6A
:103058008CBFB0EE472AB0EE642AF1EE10FA98BFA2
:10306800B0EE427AA8BFF0EE647AB8F1060FCDED63
:10307800174A00F00681D3ED1A4AD3ED191A93EDD9
:103088001B2A66EEA44AE6EE214AE5EE824A64EE81
:10309800834AF4EEC74AF1EE10FAF4EEE74A8CBF21
:1030A800B0EE472AB0EE642AF1EE10FA98BFB0EEFF
:1030B800427AA8BFF0EE647AB8F1070FCDED184A4E
:1030C80000F0DF8020E000BFFC4200209864002070
:1030D8001C630020E83C0020855B00202C35002084
:1030E800D447002038350020000000004435002077
:1030F8006F12833AD8470020B0350020493D0020A0
:10310800183C0020443E0020D3ED1E4AD3ED1D1A82
:1031180093ED1F2A66EEA44AE6EE214AE5EE824ABE
:1031280064EE834AF4EEC74AF1EE10FAF4EEE74A89
:103138008CBFB0EE472AB0EE642AF1EE10FA98BFC1
:10314800B0EE427AA8BFF0EE647AB8F1080FCDED80
:10315800194A00F09680D3ED224AD3ED211A93ED57
:10316800232A66EEA44AE1EE864AE2EE254A64EE98
:10317800834AF4EEC74AF1EE10FAF4EEE74A8CBF40
:10318800B0EE472AB0EE642AF1EE10FAD8BFB0EEDE
:10319800427AA8BFF0EE647AB8F1090FCDED1A4A69
:1031A8006FD0D3ED264AD3ED251A93ED272A66EE84
:1031B800A44AE1EE864AE2EE254A64EE834AB4EE7A
:1031C800E47AF1EE10FAF4EEE74A8CBFB0EE642A26
:1031D800B0EE472AF1EE10FA98BFB0EE427AA8BFD7
:1031E800F0EE647AB8F10A0FCDED1B4A49D0D3ED61
:1031F8002A4AD3ED291A93ED2B2A66EEA44AE6EE65
:10320800214AE5EE824A64EE834AB4EEE47AF1EEAE
:1032180010FAF4EEE47A8CBFB0EE642AB0EE472AD6
:10322800F1EE10FACDED1C4A58BFB0EE427AA8BFB5
:10323800F0EE674AB8F10B0F03F03F84D3ED2E7A16
:10324800D3ED2D1A93ED2F2A66EEA77AE1EE867A52
:10325800E2EE257A67EE837AB4EEE77AF1EE10FAB9
:10326800F4EEE74A8CBFF0EE676AF0EE476AF1EEDB
:1032780010FACDED1D7AA8BFB0EE667AA8BFF0EEC1
:10328800647A77EEC77AF7EE006AF4EEE67AF1EE42
:1032980010FAC4ED717A43F3E18386EEA77AB8F1A8
:1032A800010FDDED127A67EE877ACDED127A5FD0E5
:1032B800DDED137A67EE877AB8F1020FCDED137A58
:1032C80056D0DDED147A67EE877AB8F1030FCDEDAD
:1032D800147A4DD0DDED157A67EE877AB8F1040FD0
:1032E800CDED157A44D0DDED167A67EE877AB8F120
:1032F800050FCDED167A3BD0DDED177A67EE877AAC
:10330800B8F1060FCDED177A32D0DDED187A67EEF9
:10331800877AB8F1070FCDED187A29D0DDED197A43
:1033280067EE877AB8F1080FCDED197A20D0DDED78
:103338001A7A67EE877AB8F1090FCDED1A7A17D0A5
:10334800DDED1B7A67EE877AB8F10A0FCDED1B7AAF
:103358000ED0DDED1C7A67EE877AB8F10B0FCDED54
:103368001C7A05D0DDED1D7A27EE877A8DED1D7A62
:10337800E34B1A6812F0805200F0B2854FF07C538C
:10338800C4F8F831B8F1000F02F0EE86089BDD4E64
:103398001F78DD48DD49DE4D96ED006A94F8FC3172
:1033A800069EC0780978B5F90650D4ED7E6A768B0A
:1033B80007F0010C079F07F0100E07F48007002B99
:1033C80040F0AA82BEF1000F00F03286BCF1000F77
:1033D80043F0FE80002843F08F83CE4BDDED127A58
:1033E80093ED007ACC49E7EE267ABDEEC47A17EE63
:1033F800102AB0EE637AA5EE277A1546F0EE477AE2
:10340800FDEEE77ABDEEE37A17EE906A17EE100A42
:10341800B242A8BF3546B042C8BF054607EE905A2B
:10342800F8EEE77AB8F1010FC1ED007A00F05881A3
:1034380093ED047ADDED137AE7EE267AB0EE637A3F
:10344800A5EE277AFDEEC77A17EE906A17EE905A26
:103458009642A8BF15468642B8BF054607EE905A61
:10346800F8EEE77AB8F1020FC1ED017A00F0388181
:1034780093ED087ADDED147AE7EE267AB0EE637AFA
:10348800A5EE277AFDEEC77A17EE906A17EE905AE6
:103498009642A8BF15468642B8BF054607EE905A21
:1034A800F8EEE77AB8F1030FC1ED027A00F018815F
:1034B80093ED0C7ADDED157AE7EE267AB0EE637AB5
:1034C800A5EE277AFDEEC77A17EE906A17EE905AA6
:1034D8009642A8BF15468642B8BF054607EE905AE1
:1034E800F8EEE77AB8F1040FC1ED037A00F0F8803E
:1034F80093ED107ADDED167AE7EE267AB0EE637A70
:10350800A5EE277AFDEEC77A17EE906A17EE905A65
:103518009642A8BF15468642B8BF054607EE905AA0
:10352800F8EEE77AB8F1050FC1ED047A00F0D8801B
:1035380093ED147ADDED177AE7EE267AB0EE637A2A
:10354800A5EE277AFDEEC77A17EE906A17EE905A25
:103558009642A8BF15468642B8BF054607EE905A60
:10356800F8EEE77AB8F1060FC1ED057A00F0B880F9
:1035780093ED187ADDED187AE7EE267AB0EE637AE5
:10358800A5EE277AFDEEC77A17EE906A17EE905AE5
:103598009642A8BF15468642B8BF054607EE905A20
:1035A800F8EEE77AB8F1070FC1ED067A00F09880D7
:1035B80093ED1C7ADDED197AE7EE267AB0EE637AA0
:1035C800A5EE277AFDEEC77A17EE906A17EE905AA5
:1035D8009642A8BF15468642B8BF054607EE905AE0
:1035E800F8EEE77AB8F1080FC1ED077A78D093EDD5
:1035F800207ADDED1A7AE7EE267AB0EE637AA5EE48
:10360800277AFDEEC77A17EE906A17EE905A96421F
:10361800A8BF15468642B8BF054607EE905AF8EE91
:10362800E77AB8F1090FC1ED087A59D093ED247AF9
:10363800DDED1B7AE7EE267AB0EE637AA5EE277AFF
:10364800FDEEC77A17EE906A17EE905A9642A8BF19
:1036580015468642B8BF054607EE905AF8EEE77A57
:10366800B8F10A0FC1ED097A3AD093ED287ADDED69
:103678001C7AE7EE267AB0EE637AA5EE277AFDEE9D
:10368800C77A17EE906A17EE905A9642A8BF154669
:103698008642B8BF054607EE905AF8EEE77AB8F1C9
:1036A8000B0FC1ED0A7A1BD093ED2C7ADDED1D7A54
:1036B800E6EE877AE5EE273AFDEEE37A17EE903AE2
:1036C8009A42A8BF1A469842D8BF104607EE900AF9
:1036D800F8EEE77AC1ED0B7AB8F1000F00F0AC8292
:1036E8004FEA88020D490C4827F059FC0C4B1B681F
:1036F800002B00F0A6820B4B1B78192B1FD813E068
:103708008C640020E43B0020085D0020903E0020EF
:1037180080710020183C002064350020E83B002020
:1037280060470020644700200122734902FA03F32E
:103738001940002943F076821D0302F16A836F4E17
:103748006F4F079B99061CD5FB7AFF2B04D06D4A57
:1037580012789A4202F25883B7F90880FB7DA6F8DE
:103768000080FF2B04D0674A12789A4202F24783FE
:10377800B7F914507580082010F05EFE002842F05A
:103788002C80B7F90600B6F900C0B6F902E0B7F91F
:103798001210B7F91E20B6F90450B7F90430B6F97B
:1037A80006806045A8BF60467145A8BF7146AA4219
:1037B800A8BF2A469C45A8BF03463380B7F91030F6
:1037C800B6F908007345C8BF1946B7F92A307180A1
:1037D800B7F91C10B7F934E04345A8BF4346A942DE
:1037E800CCBF0D461546B7F93620B580B7F9285035
:1037F800B6F90A108242A8BF0246A845ACBF98464F
:10380800A846B7F94230B6F90C50A6F806808B42A4
:10381800A8BF0B468645CCBF70461046B7F94E2068
:103828003081B7F94000B6F90EE0AA42A8BF2A468F
:103838008842C8BF0346B7F95A00B7F94C107381DC
:103848007045B7F95830304FA8BF70469E45A8BF9D
:103858000346A942D8BF1146B181F381BB892BB376
:10386800DFF8AC80DFF8ACA0DFF8949008F1100521
:10387800B8F9023000EE103A5046B8EEC00A08F027
:103888003DFE25F099FAB9F90430B9F9062000B2DD
:1038980098420AF12C0A09F10C0903DB824213460B
:1038A800A8BF034628F8023FA845E1D1174B1B786B
:1038B800013B182B00F2A686DFE813F09206A40657
:1038C800A4067B0FA406A406A406EB12A406A4066D
:1038D800A406A406A406DB12A406A406A406A4064D
:1038E800C9127B0FF812A406A406DB129206B0EEEA
:1038F800666AFFF772BA00BF3241300354350020C0
:103908003C480020B8600020FC5700206447002095
:10391800523500201C450020BEF1000F40F01485F0
:10392800D94BDDED127A93ED007A002941F0288415
:10393800E7EE267AD549B1EE455AB0EE447AA5EEBF
:10394800277AF0EE477ABDEEC47A002843F08083E8
:10395800FDEEE77A17EE100A17EE906AFDEEE37AAD
:10396800B04217EE902A17EE105AA8BF3546B24259
:10397800C8BF154607EE905AF8EEE77AB8F1010F7E
:10398800C1ED007A00F0548193ED047ADDED137AED
:10399800E7EE267AB0EE447AA5EE277AFDEEC77AEE
:1039A80017EE906A17EE905A8642A8BF05469642CF
:1039B800B8BF154607EE905AF8EEE77AB8F1020F4D
:1039C800C1ED017A00F0348193ED087ADDED147AC7
:1039D800E7EE267AB0EE447AA5EE277AFDEEC77AAE
:1039E80017EE906A17EE905A8642A8BF054696428F
:1039F800B8BF154607EE905AF8EEE77AB8F1030F0C
:103A0800C1ED027A00F0148193ED0C7ADDED157AA0
:103A1800E7EE267AB0EE447AA5EE277AFDEEC77A6D
:103A280017EE906A17EE905A8642A8BF054696424E
:103A3800B8BF154607EE905AF8EEE77AB8F1040FCA
:103A4800C1ED037A00F0F48093ED107ADDED167A7B
:103A5800E7EE267AB0EE447AA5EE277AFDEEC77A2D
:103A680017EE906A17EE905A8642A8BF054696420E
:103A7800B8BF154607EE905AF8EEE77AB8F1050F89
:103A8800C1ED047A00F0D48093ED147ADDED177A55
:103A9800E7EE267AB0EE447AA5EE277AFDEEC77AED
:103AA80017EE906A17EE905A8642A8BF05469642CE
:103AB800B8BF154607EE905AF8EEE77AB8F1060F48
:103AC800C1ED057A00F0B48093ED187ADDED187A2F
:103AD800E7EE267AB0EE447AA5EE277AFDEEC77AAD
:103AE80017EE906A17EE905A8642A8BF054696428E
:103AF800B8BF154607EE905AF8EEE77AB8F1070F07
:103B0800C1ED067A00F0948093ED1C7ADDED197A08
:103B1800E7EE267AB0EE447AA5EE277AFDEEC77A6C
:103B280017EE906A17EE905A8642A8BF054696424D
:103B3800B8BF154607EE905AF8EEE77AB8F1080FC5
:103B4800C1ED077A74D093ED207ADDED1A7AE7EEAD
:103B5800267AB0EE447AA5EE277AFDEEC77A17EEFC
:103B6800906A17EE905A8642A8BF05469642B8BF9B
:103B7800154607EE905AF8EEE77AB8F1090FC1ED4D
:103B8800087A55D093ED247ADDED1B7AE7EE267A94
:103B9800B0EE447AA5EE277AFDEEC77A17EE906A62
:103BA80017EE905A8642A8BF05469642B8BF1546FA
:103BB80007EE905AF8EEE77AB8F10A0FC1ED097AE4
:103BC80036D093ED287ADDED1C7AE7EE267AB0EE52
:103BD800447AA5EE277AFDEEC77A17EE906A17EEBB
:103BE800905A8642A8BF05469642B8BF154607EECA
:103BF800905AF8EEE77AB8F10B0FC1ED0A7A17D0B0
:103C080093ED2C7ADDED1D7AE6EE877AA5EE274A4C
:103C1800FDEEC47A17EE903A9842A8BF18469A4229
:103C2800D8BF024607EE902AF8EEE77AC1ED0B7A84
:103C3800BCF1000F3FF450AD154B1B68002B7FF40F
:103C48005AAD144B1B7893B1134B187860B10F4ED3
:103C5800124F0025E8B23B68B6EC010A98470E4BB4
:103C6800187801358542F5DB0D4B1B6898479BF8A2
:103C78000030072B01F02681012384F800311FB0A2
:103C8800BDEC0C8BBDE8F08F183C0020643500209B
:103C980060470020F8420020493D0020843E002073
:103CA8008C3E00200B9BB2F900E0B3F90A30CB49F7
:103CB800AEEB0300096880EAE073A3EBE0738B4284
:103CC800BEF616ADB2F902300B9AB2F90C209A1A68
:103CD80082EAE273A3EBE27399427EF709AD099990
:103CE800BF4BD1ED017A93ED007AF0EEE77AF4EE6E
:103CF800C77AF1EE10FA7EF5FBACD1ED027AF0EE60
:103D0800E77AB4EEE77AF1EE10FA7EF7F1ACB54B4C
:103D18001A88002384F8D431002A40F09B83B24AE1
:103D2800B24B1178186881F001010DF053F9FEF7D4
:103D3800DFBCAF4BAF4A2B44D3ED006A92ED007A5B
:103D4800AD4B26EE877AF7EE006AB4EEE67AD3ED4D
:103D5800007AF1EE10FA88BFB0EE667A27EE277A7D
:103D680067EE0C7AFEF71EBD072B02F0728600265E
:103D7800A24B05931B68A24D5A0501F1B581A14BD1
:103D88001B78002B40F00A819F4B069394F8127120
:103D980027B1B4F814319B0742F0DC83069A94F8F3
:103DA8001C31D27F002B41F03E810699897F002982
:103DB80000F07186022902F0D081032901F0EE8417
:103DC800924949880232D2B2002B02F0B68100290A
:103DD80002F0B3818E480068B1FBF0F10FFA81F868
:103DE800A4F84C81002A03F04B8607EE908AF8EE7F
:103DF800E77AF7EE006A86EEA77ADFF824A2012AAE
:103E0800D4ED586ADAED007A77EEE67A67EE877ACB
:103E1800C4ED547A21D0DAED017AD4ED596A77EEFF
:103E2800E67A022A67EE877AC4ED557A15D0DAED7C
:103E3800027AD4ED5A6A77EEE67A032A67EE877A31
:103E4800C4ED567A09D0DAED037AD4ED5B6A77EEE1
:103E5800E67A67EE877AC4ED577A9BF8001009294D
:103E680003F05786B8F1000F40F31D8692B3D4EDE6
:103E7800587A94ED547A77EE877A012AC4ED587A05
:103E8800CAED007A21D0D4ED597A94ED557A77EEBF
:103E9800877A022AC4ED597ACAED017A15D0D4ED91
:103EA8005A7A94ED567A77EE877A032AC4ED5A7ACD
:103EB800CAED027A09D0D4ED5B7A94ED577A77EEA1
:103EC800877AC4ED5B7ACAED037A013A022AB8BF51
:103ED8000222D2B2002B0CBF1346022300F0E4BD2D
:103EE800079B5E023FF54AAAFFF74CBA0C98DFF829
:103EF80034E10028D8BF404207EE100A9EF800E0DF
:103F0800B8EEC77A27EE097ABEF1000F7EF4BBAE91
:103F1800DFF814E1DEED006AF4EECB6AF1EE10FA98
:103F280041F16480B7EE005A35EE665A9FED396A62
:103F3800DFF8F8E03BEEC77A25EE065A9EED006AF8
:103F4800E7EE056A26EE867AB5EEC07AF1EE10FA4B
:103F580040F2B487CAEE076AB7EE006A35EEC67A51
:103F6800F0EE465AE7EE265AF0EE656AFEF7BDBE59
:103F780001230899C4F8D811022A84F8D4317EF4B0
:103F88003FAC184A1288002A43F0A285164A174BFC
:103F9800117818680DF01EF8FEF732BC1A4A1E4B4D
:103FA80006921146B3F906204B8B9A423FF7EEAEC4
:103FB8001A4B1B78012B02F0AB80192B02F0A8805A
:103FC8000E2B3FF4E3AE082B3FF4E0AEDFF850A031
:103FD8000023CAF80830C4F80C31D7E6C4470020DB
:103FE800C8470020C8620020CA620020CC620020B6
:103FF800601D002094470020904700205043002077
:104008001C4A002068000020FC420020B860002004
:1040180098350020610BB63B80710020B035002038
:10402800443E0020A4470020AC470020A0470020C1
:10403800C34BDDED127A93ED007A002842F08683B7
:10404800E7EE267ABF49BDEEC47A17EE102AB0EE25
:10405800637AA5EE277A1546F0EE477AFDEEE77A01
:10406800BDEEE37A17EE906A17EE100AB242A8BFC7
:104078003546B042C8BF054607EE905AF8EEE77AD3
:10408800B8F1010FC1ED007A3FF4D2AD93ED047A97
:10409800DDED137AE7EE267AB0EE637AA5EE277A9D
:1040A800FDEEC77A17EE906A17EE905A9642A8BFAF
:1040B80015468642B8BF054607EE905AF8EEE77AED
:1040C800B8F1020FC1ED017A3FF4B2AD93ED087A71
:1040D800DDED147AE7EE267AB0EE637AA5EE277A5C
:1040E800FDEEC77A17EE906A17EE905A9642A8BF6F
:1040F80015468642B8BF054607EE905AF8EEE77AAD
:10410800B8F1030FC1ED027A3FF492AD93ED0C7A4A
:10411800DDED157AE7EE267AB0EE637AA5EE277A1A
:10412800FDEEC77A17EE906A17EE905A9642A8BF2E
:1041380015468642B8BF054607EE905AF8EEE77A6C
:10414800B8F1040FC1ED037A3FF472AD93ED107A24
:10415800DDED167AE7EE267AB0EE637AA5EE277AD9
:10416800FDEEC77A17EE906A17EE905A9642A8BFEE
:1041780015468642B8BF054607EE905AF8EEE77A2C
:10418800B8F1050FC1ED047A3FF452AD93ED147AFE
:10419800DDED177AE7EE267AB0EE637AA5EE277A98
:1041A800FDEEC77A17EE906A17EE905A9642A8BFAE
:1041B80015468642B8BF054607EE905AF8EEE77AEC
:1041C800B8F1060FC1ED057A3FF432AD93ED187AD8
:1041D800DDED187AE7EE267AB0EE637AA5EE277A57
:1041E800FDEEC77A17EE906A17EE905A9642A8BF6E
:1041F80015468642B8BF054607EE905AF8EEE77AAC
:10420800B8F1070FC1ED067A3FF412AD93ED1C7AB1
:10421800DDED197AE7EE267AB0EE637AA5EE277A15
:10422800FDEEC77A17EE906A17EE905A9642A8BF2D
:1042380015468642B8BF054607EE905AF8EEE77A6B
:10424800B8F1080FC1ED077A3FF4F2AC93ED207A8C
:10425800DDED1A7AE7EE267AB0EE637AA5EE277AD4
:10426800FDEEC77A17EE906A17EE905A9642A8BFED
:1042780015468642B8BF054607EE905AF8EEE77A2B
:10428800B8F1090FC1ED087A3FF4D2AC93ED247A66
:10429800DDED1B7AE7EE267AB0EE637AA5EE277A93
:1042A800FDEEC77A17EE906A17EE905A9642A8BFAD
:1042B80015468642B8BF054607EE905AF8EEE77AEB
:1042C800B8F10A0FC1ED097A3FF4B2AC93ED287A40
:1042D800DDED1C7AE7EE267AB0EE637AA5EE277A52
:1042E800FDEEC77A17EE906A17EE905A9642A8BF6D
:1042F80015468642B8BF054607EE905AF8EEE77AAB
:10430800B8F10B0FC1ED0A7A3FF492AC93ED2C7A19
:10431800DDED1D7AE6EE877AE5EE273AFDEEE37AE3
:1043280017EE903A9A42A8BF1A469842D8BF10464C
:1043380007EE900AF8EEE77AC1ED0B7A78E400BF51
:10434800183C002064350020BCF1000F42F08A813F
:10435800002941F0B481FDEEE37A0DF1480E17EE25
:10436800906AFDEEC47A0EEB880317EE907AFDEEA4
:10437800C67A80F00102D049DFF87893CDF8308012
:1043880017EE905ACDF838A0B1EE455A4FFA80FC96
:1043980098460D9492460B4693ED007AFEEC017A0E
:1043A800E6EE877A3A461031B0EE447AA5EE277ADF
:1043B800FDEEC77A17EE903A9F42A8BF1A469D4273
:1043C800CCBF002400F00104002C14BF14462C4676
:1043D8009E42CCBF00230AF0010307EE904A002B4F
:1043E80014BF13463346B8EEE77A07EE903AF8EE74
:1043F800E77ABCF1000F18BFF0EE477AC645E9EC42
:10440800017AC8D1DDF830800D9CDDF838A0FFF7BF
:1044180063B907EE901AF8EEE77AA848A84DD0EDF0
:10442800003A95ED004AA74884ED7C4A06EE903A9A
:1044380077EE677ABCEEC77AF8EEE66A17EE103ABE
:1044480077EEE67AC4ED7D3AA4F8EC31D0ED006A57
:10445800FEF786BC9C494A69002A3EF449A90A68C5
:1044680013604B74FEF744B907EE103A9BF800301E
:10447800964FC4F8A481B8EEC77AF7EE006A132BFA
:1044880086EE879AB7F90400B4F8A86195ED080A92
:1044980001F01C858E4B8F4A93ED001A93ED093A73
:1044A80093ED162A93ED1F6AD3ED0B1A93ED144A78
:1044B800D3ED015AD3ED0A3A93ED0C7A93ED155AE0
:1044C800D3ED172AD3ED206AD3ED044AD3ED030ABE
:1044D80069EE277A69EE288A29EE088AA7EE813ADA
:1044E80002EB860E0021A2EE286AC4F89811C4F8DF
:1044F8009C11A8EE214AE7EEA53AA8EE075A93EDDB
:104508001A7AD3ED0F5A93ED021AD3ED0E1A8EEDE7
:10451800003AE2EEA86A64EEC34A27EE467A93EDC3
:104528000D2AD3ED192A8EED204AE3EE603A65EEA6
:10453800C45A93ED183AC3ED093AE7EE814AF0EE12
:10454800477AA1EEC45AE8EE025AE2EEC66AE3EEF2
:10455800287AC3ED0A4A83ED145AC3ED155A8EED35
:10456800406AC3ED1F6AC3ED207AC4F8A011731C1A
:1045780003F01F03A4F8A831B880FDF7B6BF564B67
:104588001A79002A3EF46AAC544A1278002A3EF49A
:1045980065AC1B789FED522A07EE103A514B07EE97
:1045A800902A1B88F8EEE77A04EE903AB8EE477A3C
:1045B800F8EE644A27EE277AB7EE003AC7EE247A77
:1045C800F4EEC27AF1EE10FA88BFF0EE427AF4EE19
:1045D800C37AF1EE10FAB8BFF0EE437AFEF740BCAA
:1045E800BB7B002B43F01181089B1B7813F0010360
:1045F80043F00B813C4A1268002A03F0D183136010
:1046080001230A93059B1B689A0639D4374A127806
:10461800052A35D0DD027FF514ABFE7B112E3FF65F
:1046280010AB334BDDF828901D4633F9163000EEF9
:10463800103A4846B8EEC00A06F1010806F10E071E
:1046480021F012FF4B465FFA88F89E1BFFB2A9467D
:1046580000E0A84608F1010508EB0600B8F1120FC2
:10466800EDB2C0B23FF4EDAA39F9183000EE103AB5
:10467800B8EEC00A21F0F8FEBD42EAD1FFF7E1BA70
:104688000A9A13460233551CDBB21046EDB20A9360
:10469800B6F9003000EE103AB8EEC00A21F0E4FE98
:1046A800B6F9023000EE103A2846B8EEC00A21F0FA
:1046B800DBFE059B1B68ADE7183C0020D83C0020BA
:1046C80098640020F03C0020D06200205C3D00206F
:1046D8001455002078520020E05E0020423E002061
:1046E800713DAA3F303E00200C580020644700204E
:1046F80080710020643500200000000093ED027AEC
:1047080093ED012AD3ED037A1FED053A26EE877A59
:10471800A6EE027AA7EEA57A27EE247AB4EEC37A3B
:10472800F1EE10FAB4BFF0EE437AF0EE477A8DED71
:10473800127A88BFB0EE437AB8F1010F3EF4A1AD0A
:1047480093ED063AD3ED051A93ED072A26EE833A40
:10475800A6EE213AA2EE253A23EE243AB4EEC73A61
:10476800F1EE10FAB4EEE73A8CBFB0EE472AB0EE9D
:10477800432AF1EE10FA98BFB0EE427AA8BFF0EEE5
:10478800437AB8F1020F8DED133A3EF47AAD93ED0A
:104798000A3AD3ED091A93ED0B2A26EE833AA6EED0
:1047A800213AA2EE253A23EE243AB4EEC73AF1EEC6
:1047B80010FAB4EEE73A8CBFB0EE472AB0EE432ABF
:1047C800F1EE10FA98BFB0EE427AA8BFF0EE437A45
:1047D800B8F1030F8DED143A3EF453AD93ED0E3A54
:1047E800D3ED0D1A93ED0F2A26EE833AA6EE213A61
:1047F800A2EE253A23EE243AB4EEC73AF1EE10FAC7
:10480800B4EEE73A8CBFB0EE472AB0EE432AF1EE99
:1048180010FA98BFB0EE427AA8BFF0EE437AB8F12A
:10482800040F8DED153A3EF42CAD93ED123AD3ED0D
:10483800111A93ED132A26EE833AA6EE213AA2EE38
:10484800253A23EE243AB4EEC73AF1EE10FAB4EE64
:10485800E73A8CBFB0EE472AB0EE432AF1EE10FAE1
:1048680098BFB0EE427AA8BFF0EE437AB8F1050FD0
:104878008DED163A3EF405AD93ED163AD3ED151AC3
:1048880093ED172A26EE833AA6EE213AA2EE253AB0
:1048980023EE243AB4EEC73AF1EE10FAB4EEE73A52
:1048A8008CBFB0EE472AB0EE432AF1EE10FA98BF5B
:1048B800B0EE427AA8BFF0EE437AB8F1060F8DED5C
:1048C800173A3EF4DEAC93ED1A3AD3ED191A93ED8C
:1048D8001B2A26EE833AA6EE213AA2EE253A23EECB
:1048E800243AB4EEC73AF1EE10FAB4EEE73A8CBFC8
:1048F800B0EE472AB0EE432AF1EE10FA98BFB0EEB8
:10490800427AA8BFF0EE437AB8F1070F8DED183A56
:104918003EF4B7AC93ED1E3AD3ED1D1A93ED1F2A62
:1049280026EE833AA1EE863AA2EE253A23EE243A01
:10493800B4EEC73AF1EE10FAB4EEE73A8CBFB0EE37
:10494800472AB0EE432AF1EE10FA98BFB0EE427A49
:10495800A8BFF0EE437AB8F1080F8DED193A3EF48E
:1049680090AC93ED223AD3ED211A93ED232A26EE4B
:10497800833AA1EE863AA2EE253A23EE243AB4EE23
:10498800C73AF1EE10FAB4EEE73A8CBFB0EE472A18
:10499800B0EE432AF1EE10FA98BFB0EE427AA8BF03
:1049A800F0EE437AB8F1090F8DED1A3A3EF469AC8E
:1049B80093ED262AD3ED251A93ED273A26EE822A7F
:1049C800A1EE862AA3EE252A22EE242AB4EEC72ACF
:1049D800F1EE10FAB4EEE72A8CBFB0EE473AB0EE2B
:1049E800423AF1EE10FA8DED1B2A98BFB0EE437AE9
:1049F800B8BFB0EE672AB8F10A0F02F01783D3EDFB
:104A08002A7AD3ED291A93ED2B3A66EEA77AE1EECE
:104A1800867AE3EE257A67EEA47AF4EEC77AF1EEA9
:104A280010FAF4EEC27A8CBFB0EE473AB0EE673AAD
:104A3800F1EE10FA98BFB0EE437AA8BFB0EE672A3D
:104A4800B8F10B0FCDED1C7A02F0F082D3ED2E7A7F
:104A5800D3ED2D1A93ED2F3A66EEA77AE6EE217A7A
:104A6800E5EE837A67EEA47AB4EEE77AF1EE10FA0F
:104A7800B4EEE72A8CBFF0EE676AF0EE476AF1EE13
:104A880010FACDED1D7A58BFB0EE667AA8BFF0EEE9
:104A9800427AFEF7F6BBA4F84C118846002B00F0CA
:104AA8006E81DFF838A30223C14ADFEDC26A1168BC
:104AB8009BF800E00A78887807EE902AF8EEE77A03
:104AC800B0EE007A67EEA67AF4EEC77AF1EE10FA45
:104AD80040F3898237EEC77ADFEDB76AB0EE676ACE
:104AE800A7EE266AB0EE467A9FEDB46ADAED006A60
:104AF80066EE866AB0EEE66AC4ED5C6A84ED5F6ACB
:104B080098B105EE900AB8EEE55ADFEDAA5A66EEBE
:104B1800A64A25EE255AF7EE005A75EEC55A64EEF8
:104B2800864AE5EE245A66EEA56ADFEDA55A4A796B
:104B380027EE257A27EE267ACAB1DFED9E6ADFEDE9
:104B4800A15A26EE266A06EE902AF8EEE66A66EE86
:104B5800866AF4EEE56AF1EE10FA00F39E85F7EE48
:104B6800005A75EEE66A85EEA66A27EE067ABEF169
:104B78000C0F9FED958ADFED956A00F06285B4EE23
:104B8800C87AF1EE10FA98BFB0EE478AB4EEE68A1A
:104B9800F1EE10FAB8BFB0EE668A84ED418A002BB8
:104BA80000F0E080B0EE007AF4EEC77AF1EE10FA89
:104BB80005DD37EEC77ADFED806AE7EE267A9AEDF3
:104BC800017ADFED7E6A27EE267AB0EEC76A84EDB9
:104BD8005D7A84ED606A98B106EE900ADFED755A49
:104BE800F8EEE66A27EE075A66EEA56AF7EE005A6F
:104BF80075EEE65A25EE065AE6EE855A27EE257A30
:104C0800DFED6F6A8A7967EEA67A67EE877AAAB1CE
:104C180007EE102AB8EEC77ADFED665ADFED696A4B
:104C280027EE067A27EE257AB4EEE67AF1EE10FA48
:104C380040F33785DFED666A67EEA67ABEF10C0FA2
:104C480000F0E084DFED606A9FED607AF4EEE67ACA
:104C5800F1EE10FA88BFF0EE667AF4EEC77AF1EE5C
:104C680010FAB8BFF0EE477A012BC4ED427A79DD2D
:104C78004B78DFED506A07EE903AF8EEE77AB0EE3F
:104C8800007A67EEA67A4B7AF4EEC77AF1EE10FA5C
:104C980005DD37EEC77ADFED486AE7EE267A9AED4A
:104CA800027ADFED466A27EE267AB0EEC76A84ED0F
:104CB8005E7A84ED616A9BB106EE903ADFED3D5A6B
:104CC800F8EEE66A27EE075A66EEA56AF7EE005A8E
:104CD80075EEE65A25EE065AE6EE855A27EE257A4F
:104CE800DFED376ACB7967EEA67A67EE877A0BB382
:104CF80007EE103AB8EEC77ADFED2E5ADFED316ACB
:104D080027EE067A27EE257AB4EEE67AF1EE10FA67
:104D18000CDCB5EEC07AF1EE10FA01F10082B7EEC4
:104D2800006A36EE477AC6EE076A01E0DFED286AC8
:104D380067EEA67ABEF10C0F00F09E84DFED226AC2
:104D48009FED227AF4EEE67AF1EE10FA88BFF0EEE3
:104D5800667AF4EEC77AF1EE10FAB8BFF0EE477A49
:104D6800C4ED437ABEF1090F00F04284069B93F824
:104D78002170002F40F0F683002384F81C31154B76
:104D88001B7823B9144FBB78002B41F00C829BF899
:104D98000030072B00F078840022072B84F80021CC
:104DA8007DF44FAB0DF048F90690FDF74CBB00BF02
:104DB800207500200AD7233CD7A368416F12033B14
:104DC80000004843A4707D3F00C0F94400C0F9C406
:104DD8000000C842CD5B00205D600020443E0020FA
:104DE800D14A099292460026D04FDFF85083B14647
:104DF800B7EC018AD5ED087AB8EEC88A28EE278A7A
:104E0800B9F1000F03F040807BBB9BF80030082B02
:104E18003BD006F5D260B0EE480A2844D5F88C3667
:104E2800984706F5E360D5F81437284498479BF867
:104E38000030032BB0EE408A22D0D5F8AC30D7F83A
:104E48004406B0EE480A98470AEB890309F10109BC
:104E5800B9F1030F06F12C0683ED010A3DF468ABA6
:104E6800059B1B6803F00053C2E706F5F460B0EE3B
:104E7800480A2844D5F89C379847B0EE408AC4E7DA
:104E880023F09AFF28F81900D7E7B0EE480A23F074
:104E980093FF28F81900BCE7A54BA64C1A68A64B47
:104EA800A64F94F80001D2691B883A807B800028BD
:104EB8007EF45DAF0690A24DFDF7C5BADFEDA16A9D
:104EC800FDF721BF0DF0B8F8099A9C4B801AD880DD
:104ED800FEF7D2BEDFF89892D4ED017A94ED006A1D
:104EE800B9F80000D9F8143077EEA77AF0EE006A26
:104EF800B0EE677AA6EE267A013804EBC002D6EE49
:104F0800267A083A1033F6EE003A27EE237A67EE4F
:104F1800A37A84ED207AC4ED217A864C274604F1E1
:104F2800800192ED027A92ED036AD7ED036AD7ED1C
:104F3800027A53ED014A13ED025A37EE674A76EECC
:104F4800C65A77EE277AE4EE845A0138A2F10802AD
:104F5800E5EE047A07F1080703F1080336EE267A2E
:104F680001F10801E4EE877AE5EE475A67EEA37A85
:104F780025EEA37AC1ED007A81ED017AD1D1B8F19D
:104F8800140F07D10DF058F8079B6C4FC01A7880A2
:104F9800D4F8AC61644B09936B4A059BDDF824A0F7
:104FA8001B68013682FB06129119F217C2EBA102A7
:104FB800C2EBC202B61AC4F8AC6103F0005312E7A0
:104FC8000DF03AF89BF800300D9A5C4F801A012BCF
:104FD800788000F09480072B7DF43CAC0DF02CF821
:104FE8000990FDF739BCB0EE677A7DE5DFF884E11A
:104FF8009EED007AFEF7A8BF54495548554BD1EDB0
:10500800003A90ED004A54491B7884ED7C4AC4ED7F
:105018007D3AD1ED006A13B1012384F8FC31D4ED57
:105028007E7AFDF79DBE4D494D48D1F8EC100068D9
:1050380044F62067B942A8BF3946B1F57A7FB8BFB0
:105048004FF47A7110F0100F059889B2A4F81E1168
:10505800006801F01485C00440F1E0834148D0F8AD
:1050680000E0BEF836707F08DFF80CA1DFF80CC14D
:10507800D4F82001DAED037AACFB011C4FEA9C1C42
:10508800642191FBFCF11429BDEEE77A04EB40089A
:10509800A8BF142101308842C4F8200117EE109AE5
:1050A800A4BF0020C4F8200104EB4000A8F8249114
:1050B800B0F9241107EE101AB8EEC77A77EEC77A5E
:1050C800FDEEE77ACDED077ABDF91C0080EAE071C4
:1050D800A1EBE071B94202F39C84234908464FF0E2
:1050E8007E510160FEF761BEAB68002B3EF447AE0F
:1050F80005F1440128469847FEF741BE0F4F0CF0D2
:105108009BFF1A4AD4F8E83112680990C31A9A1A10
:10511800C4F8E801BB80FA80FDF79EBB0CF08CFF59
:105128000D90FDF720BA00BF40520020544A0020DD
:105138003C5D0020E41B0020445D00205C3D002015
:105148001C4A002000000000932449921C630020A0
:10515800DC3C0020903E0020EC3C0020B8140020ED
:105168008C640020F05E00200000002098350020AC
:1051780060520020A0470020443E0020D34D62101A
:10518800E7EE267AEE49B1EE455AB0EE447AA5EE3E
:10519800277AF0EE477ABDEEC47A00283EF4D8AB01
:1051A800F4EEE37AF1EE10FAB8BFF0EE467AFDEECF
:1051B800E77A17EE105A17EE906AFDEEC67AB542F6
:1051C80017EE902A17EE100AA8BF3046B242C8BFA1
:1051D800104607EE900AF8EEE77AB8F1010FC1ED34
:1051E800007A3EF425AD93ED047ADDED137AE7EE0F
:1051F800267AB0EE447AA5EE277AB4EEE37AF1EE99
:1052080010FAF0EE477AB8BFF0EE467AFDEEE77A8C
:1052180017EE906A17EE900AAE42A8BF284696424B
:10522800B8BF104607EE900AF8EEE77AB8F1020F19
:10523800C1ED017A3EF4FCAC93ED087ADDED147A09
:10524800E7EE267AB0EE447AA5EE277AB4EEE37A52
:10525800F1EE10FAF0EE477AB8BFF0EE467AFDEEBE
:10526800E77A17EE906A17EE900AAE42A8BF284672
:105278009642B8BF104607EE900AF8EEE77AB8F102
:10528800030FC1ED027A3EF4D3AC93ED0C7ADDED59
:10529800157AE7EE267AB0EE447AA5EE277AB4EED0
:1052A800E37AF1EE10FAF0EE477AB8BFF0EE467AFC
:1052B800FDEEE77A17EE906A17EE900AAE42A8BFA5
:1052C80028469642B8BF104607EE900AF8EEE77AED
:1052D800B8F1040FC1ED037A3EF4AAAC93ED107A4D
:1052E800DDED167AE7EE267AB0EE447AA5EE277A57
:1052F800B4EEE37AF1EE10FAF0EE477AB8BFF0EECA
:10530800467AFDEEE77A17EE906A17EE900AAE42FB
:10531800A8BF28469642B8BF104607EE900AF8EE96
:10532800E77AB8F1050FC1ED047A3EF481AC93ED4C
:10533800147ADDED177AE7EE267AB0EE447AA5EE18
:10534800277AB4EEE37AF1EE10FAF0EE477AB8BFB6
:10535800F0EE467AFDEEE77A17EE906A17EE900ABD
:10536800AE42A8BF28469642B8BF104607EE900A3C
:10537800F8EEE77AB8F1060FC1ED057A3EF458ACBD
:1053880093ED187ADDED187AE7EE267AB0EE447AD6
:10539800A5EE277AB4EEE37AF1EE10FAF0EE477A4A
:1053A800B8BFF0EE467AFDEEE77A17EE906A17EE90
:1053B800900AAE42A8BF28469642B8BF104607EEEC
:1053C800900AF8EEE77AB8F1070FC1ED067A3EF4D5
:1053D8002FAC93ED1C7ADDED197AE7EE267AB0EE64
:1053E800447AA5EE277AB4EEE37AF1EE10FAF0EEFD
:1053F800477AB8BFF0EE467AFDEEE77A17EE906A84
:1054080017EE900AAE42A8BF28469642B8BF10468B
:1054180007EE900AF8EEE77AB8F1080FC1ED077ABF
:105428003EF406AC93ED207ADDED1A7AE7EE267AA3
:10543800B0EE447AA5EE277AB4EEE37AF1EE10FAEC
:10544800F0EE477AB8BFF0EE467AFDEEE77A17EE4F
:10545800906A17EE900AAE42A8BF28469642B8BF97
:10546800104607EE900AF8EEE77AB8F1090FC1ED99
:10547800087A3EF4DDAB93ED247ADDED1B7AE7EE96
:10548800267AB0EE447AA5EE277AB4EEE37AF1EE06
:1054980010FAF0EE477AB8BFF0EE467AFDEEE77AFA
:1054A80017EE906A17EE900AAE42A8BF28469642B9
:1054B800B8BF104607EE900AF8EEE77AB8F10A0F7F
:1054C800C1ED097A3EF4B4AB93ED287ADDED1C7A90
:1054D800E7EE267AB0EE447AA5EE277AB4EEE37AC0
:1054E800F1EE10FAF0EE477AB8BFF0EE467AFDEE2C
:1054F800E77A17EE906A17EE900AAE42A8BF2846E0
:105508009642B8BF104607EE900AF8EEE77AB8F16F
:105518000B0FC1ED0A7A3EF48BAB93ED2C7ADDEDDF
:105528001D7AE6EE877AA5EE274AF4EEC43AF1EE44
:1055380010FAC8BFB0EE464AFDEEC47A02E000BFDA
:105548006435002017EE903A9D42A8BF1D469A4246
:10555800D8BF2A4607EE902AF8EEE77AC1ED0B7A13
:10556800FEF766BB1E21BB4807F0F4FE00283FF497
:1055780003ACB4F8143159063FF5FEAB94F8883102
:10558800BB4242F0E582B44BD4ED637A93ED010A55
:10559800D4ED435A9FEDB16ADFEDB16A27EEE57AA3
:1055A80067EE887AA0EE087AE5EE807AB4EEC67ADD
:1055B800F1EE10FA88BFB0EE467AB4EEE67AF1EE74
:1055C80010FAF4EEC67AB8BFB0EE667AF1EE10FAC9
:1055D80088BFF0EE467AF4EEE67AF1EE10FAB8BF3C
:1055E800F0EE667A84ED417AC4ED437AFFF7C4BBE6
:1055F800FDEEC87A9B4F17EE903AA7F80480FB801F
:10560800FFF7B4BB9FED957ADFED956A954FF4EE01
:10561800C77AF1EE10FA98BFB0EE677AFDEEE77A36
:10562800B4EEE67AF1EE10FA17EE902AB8BFB0EEB3
:10563800667A012B84ED427A7A803FF719ABFFF73F
:1056480095BBB4EEC87AF1EE10FA98BFB0EE478A6F
:10565800BDEEC77AB4EEE68A824FF1EE10FA17EE85
:10566800102AB8BFB0EE668A84ED418A3A80002BD2
:105678007FF498AAFFF77ABBBDEEE77A794F17EE69
:10568800103ABB80FFF75ABB0CF0D6FC754F9BF85D
:105698000030801BB880FFF77FBB9FED736AFFF770
:1056A80064BAB5EEC07AF1EE10FA00F13C85B7EEB7
:1056B800006A36EE477AC6EE076AFFF7BDBAFDEE16
:1056C800E37A12A917EE906AFDEEC47A01EB88031B
:1056D80017EE907AFDEEC67A80F00102DFF8A0910D
:1056E800DFF8A0E1CDF8308017EE905A0D94B1EEB6
:1056F800455A4FFA80FC1C46CDF838A090464B46D8
:1057080093ED007AF1EC017AE6EE877A00F0010376
:1057180009F11009B0EE447AA5EE277AF4EEC73AFB
:10572800F1EE10FAD8BF0023002BF0EE477A18BF2D
:10573800B0EE467ABDEEC77AFDEEE77A17EE102A8C
:1057480017EE90AABA4217EE103AA8BF3B46954208
:10575800CCBF002200F00102002A08BF2B465745A3
:1057680007EE103A3A46A8BF52465645CCBF00232A
:1057780008F00103002B08BF324607EE902AB8EE66
:10578800C77AF8EEE77ABCF1000F18BFF0EE477A57
:10579800A142EEEC017AB2D1FEF734BE069991F837
:1057A8002010C1EB411001EB8001C90089B2FEF75E
:1057B80009BB2E4BB6F908101A6802B111609B6933
:1057C800B6F90A2003B11A60059B1B689A0601F115
:1057D8009F8702220A92FEF71DBF94F82832012BF8
:1057E80002F03980224B97F916005A8897F90AE097
:1057F8001B88204910FB03F31EFB02F281FB020CFD
:1058080081FB0301D217DB17C2EB2C12C3EB211368
:1058180042441D4432807580FDF7B3BF1648D0F866
:1058280000E0BEF936701FE4DFF85C901348D9F841
:105838000820B9F80C1022F045FB9BF80080B8F15D
:10584800140F02F02582D4F8AC610136C4F8AC61BB
:10585800FFF742BB8C6400200000002000C0F94420
:1058680000C0F9C45C3D00200000C8420C5800206C
:10587800B06000201F85EB51F05E0020E41B002083
:10588800183C00206435002060520020DFF8649343
:10589800B9F80070D9F804E04FEA570C4FEA8C02C7
:1058A80004EB8708FF0804EB020300F09F80103226
:1058B8000137C54803EB0717424410330EF11006B1
:1058C80008F1100151ED032A51ED043A10ED043AA4
:1058D80010ED032A51ED026A11ED016A10ED020A7A
:1058E80010ED018A12ED044A12ED035A53ED044AF1
:1058F80053ED035A13ED027A53ED017A52ED020A81
:1059080012ED011A73EE238A72EE221A40ED048A10
:1059180040ED031A70EE268A78EE061A40ED028AE8
:1059280040ED011A74EE848A75EE851A43ED048AF7
:1059380043ED031A77EE208A77EE811A43ED028A47
:1059480043ED011A73EE633A75EE655A16ED035A84
:1059580032EE623A74EE644A65EE631A16ED044A52
:1059680023EE052A64EE652AE3EE041A1033BB42DF
:1059780024EE843AA3EE842A00F1100006F1100602
:10598800A5EE853A01F1100102F11002E4EE852A34
:1059980041ED071A01ED082A02ED073A42ED082AFF
:1059A80056ED055A16ED065A70EE666A38EE466AE6
:1059B80030EEC77A71EE677A26EE253A65EEE63A5A
:1059C80025EE674A67EE054AE6EE053AA6EE853A01
:1059D800A7EE254AE7EEA54A01ED063A41ED053A5C
:1059E80002ED064A42ED054A7FF46CAF1FFA8CF6C9
:1059F8007246314675481FF0EDFA3146D9F8042051
:105A080040461FF0E7FA9BF80030142B7FF4C0AA39
:105A1800FFF7B8BA6E4BD4F8B0C10993B4F8A8919F
:105A2800C9F120035FFA83FA6A4B09EB4C1703EBC1
:105A380087075FEA9A0302F0FA8001331801664982
:105A4800614A07EB000E07F1100313ED024A13ED4C
:105A5800035A13ED016A13ED047A51ED024A51ED30
:105A6800035A51ED016A51ED047A64EE244A65EE59
:105A7800255A66EE266A67EE277A1033734542ED9B
:105A8800024A42ED035A42ED016A42ED047A01F1FD
:105A9800100102F11002D8D15049A0F110021744A8
:105AA80001EB020E22441AF0030309D0B7EC017A85
:105AB800FEEC017A67EE277A013BE2EC017AF5D138
:105AC800B9F1000F41F02E86B8F1140F7FF464AAE3
:105AD8000CF0B2FA079B424FD4F8AC61C01A788038
:105AE800FFF75ABAD4F8B091394A3E4B099203EB02
:105AF800C90312680A929DED0A7A9B88DFED3A7A0B
:105B08003A4AF8EE478A09EE103A643BC82BA8BF18
:105B1800C82368EEA78AF8EE497A782BB8BF7823AD
:105B280068EEA78A07EE903A2C27B0EE680A07FBC2
:105B38000927B8EEE78A23F08BF9B8EEC99AF0EE98
:105B4800409AB0EE680A23F0E5F838EE097A79EE63
:105B5800487A28EE098A67EE877AB7EE006A88EEF7
:105B6800277AB8F1140FF8EE007A77EE076A60EE3C
:105B7800277A89EEA67A77EE065A36EE477AC6EE87
:105B8800256A67EEA67A27EE267AC7ED006A87EDC2
:105B9800047AC7ED026AC7ED017AC7ED037A02F00D
:105BA8004B80134B9BF8008009F1010983FB093CEA
:105BB800ACEBE97C0CEB4C0C0136A9EB0C0CC4F8F3
:105BC800AC61C4F8B0C129E7F41B0020E41B002035
:105BD800405200207852002008540020F85300203A
:105BE8005C3D00207854002027D4D236BC510020D8
:105BF8005655555560520020DFF8BC9399F800209F
:105C08005FEA920C02F0DA80DFF8DCE30CF10100C5
:105C180040010EEB00070EF12003AEF1700113ED09
:105C2800076A53ED056A13ED037A53ED017A53EDD4
:105C3800025A13ED084A53ED064A13ED045A26EEAC
:105C4800066A66EEA66A27EE077A67EEA77AA4EEDA
:105C5800046A2033BB42E4EEA46A01F11001A5EE08
:105C6800057AE5EEA57AF1EEC65AB1EEE66AF1EEEE
:105C7800C76AB1EEE77A41ED085A01ED076A41EDCE
:105C8800066A01ED057ACAD12038864404EB0C1166
:105C980012F0030318BF0EF1080E0FD05EED017A63
:105CA8001EED027A67EEA77A013BE7EE077A0EF15E
:105CB800080EB1EEE77AA1EC017AEFD1B8F1140F32
:105CC80001F0D8870136C4F8AC6101E0BA4B1A7804
:105CD800D4F8B0E1B9489FEDCA7A4FEACE07C319A4
:105CE80083ED007A002A7BD0B549B0EE476AF0EE22
:105CF800476A0023F1EC017A013367EEA77A05EED3
:105D0800903AB4EEE77AF1EE10FAF8EEE55AB8BF39
:105D1800B0EE677A9A4276EEA76AA7EEA56AE9D14D
:105D2800F5EEC06AC319F1EE10FA83ED007A57DD7B
:105D3800C6EE265AA34BA44A1288F7EE007A75EEEF
:105D4800E75AD3ED007A65EEA77AFDEEE77A17EE0B
:105D5800903A812B41F371819342A8BF134607EE15
:105D6800903AF8EEE77A994B2C2101FB0E3393ED2C
:105D7800097AD3ED003A93ED0A6A93ED014AD3ED1F
:105D8800046AD3ED034A93ED025AA3EEA77AA4EE70
:105D9800276A66EEC76AA7EE646ABDEEC77AE5EEC3
:105DA800276A17EE101A812983ED096AC3ED0A6A7A
:105DB80041F340818A42A8BF0A4607EE902AF8EECE
:105DC800E77AFCEEE77ACDED097ABDF82430C219FE
:105DD8009380BEF1000F03D1B8F1130F01F08B8649
:105DE800B8F1150F7FF4CBA83844794F838827F88A
:105DF8001E30784BD4F8AC610993FFF7CDB8764ADA
:105E080032F91350FDF7B6BC734A32F91380FDF727
:105E1800A5BC714B714E1A68596832609A68DB6884
:105E2800F36071606E4FB260079BFDF78BBC0CF09E
:105E380003F99BF800800790B8F1140F05BF644F71
:105E4800D4F8AC61D4F8AC613E80FCF758BBDFF8FD
:105E58009C81002538F9023F00EE103AE8B2B8EE0E
:105E6800C00A013520F000FB082DF3D10A95FEF792
:105E7800C9BBDFF87C81002538F9023F00EE103AF3
:105E8800E8B2B8EEC00A013520F0EEFA062DF3D1DB
:105E9800ECE7544BB6F906101A6802B111609B6919
:105EA800B6F90820002B7FF48EAC8DE4DFF844812E
:105EB800002538F9023B00EE103AE8B2B8EEC00A05
:105EC800013520F0D1FA042DF3D1CFE7DFF828818E
:105ED800DFF8289198ED004A98ED097AD8ED014A43
:105EE80098ED0A6AD8ED046A98ED035AD8ED025A7B
:105EF80069EE277A09EB8603A4EE277AA4EEA76A4F
:105F080066EEC76AA5EE476AE5EEA76A20EE070ABD
:105F180088ED096AC8ED0A6A83ED007A29EE088AD5
:105F280022F04AFF69EE288AD8ED145AD8ED1F6A84
:105F380098ED0B1AD8ED161A98ED155A98ED207AA7
:105F480098ED0C2AD8ED172A98ED0F6AD8ED1A7A31
:105F580098ED0E3AD8ED0D3A98ED194AD8ED184A51
:105F6800E8EE015A002209EB8603E8EEA16A00B2C6
:105F7800C4F89821A8EE025AC4F89C21C4F8A021BC
:105F8800A8EEA27A26EE656A67EEE67AA5EEC35A0F
:105F9800A8EE236AA6EEC47AE8EEA47A88ED145A2D
:105FA800C3ED205A88ED156AC3ED406A88ED1F7A63
:105FB800C8ED207AFEF7DBBA5A5200207854002048
:105FC800E41B00205C52002058520020905400200E
:105FD8005C3D002040520020807100205435002094
:105FE8003C4800200C580020641C0020523500203A
:105FF800563500205A3500201455002078520020CC
:1060080000000000B5F92430EA6207EE903A012258
:10601800F8EEE77A2B66EA670023B8F1010FC5EDC1
:106028001C7AC5ED1B7A6B6701F02E85B0457CF4B0
:10603800F7ACB5F926306B6607EE903A00220123DB
:10604800F8EEE77A2A63C5F890300023B8F1010F1B
:10605800C5ED217AC5ED207AC5F8883001F047856D
:10606800B0457CF40EADB5F92830AB6607EE903A32
:1060780000220123F8EEE77A6A63C5F8A43000230A
:10608800B8F1010FC5ED267AC5ED257AC5F89C3023
:106098007CF428AD1FED268AB9F1030F47D0BAF179
:1060A800000F09D007EE90AAF8EEE77AF4EEC87A66
:1060B800F1EE10FA01F18786C74AAB6E126894F8C0
:1060C800B411F88003EB560393FBF6F600236E63D6
:1060D80093621363D36221B1C04B1B88002B7CF4FD
:1060E80002ADBF4B1B6813F4003304D0BD4B1B79C2
:1060F800002B41F0F385BC491A46C85C012803F11E
:106108000C0301F0ED820132152AF6D1FCF7EBBC45
:10611800B64B9B7B002B3DF459AFFDF737BEF7EE2E
:10612800006AFEF705BEF7EE006AFEF785BDB0EE21
:10613800480A22F041FE00B2B1E7B4F84C8108F1F8
:10614800FF380FFA88F8B8F1000FA4F84C817EF7F1
:10615800A5ACDFF8C8A2FDF789BEB4F81E1101F599
:106168007A7189B2FDF72EBE089B1F7807F0010CE3
:10617800FDF75EBD9E4BDFED9F7A1A68C4ED717A1C
:1061880012F0805200F09D84B7EE007A77EE677ABD
:10619800F4EEE27AF1EE10FA88BFF0EE627AC4ED1E
:1061A8007E7AFDF7EFB8DFF8788298F80020013A98
:1061B8000A2A1DD8DFE812F0B401C2017C0160018F
:1061C8001C001C004A013601EA00D4000B008A4A70
:1061D8008A4952680968C8328A4203D316F00CF813
:1061E80030B1BB78032B01F08186012388F8003099
:1061F800FB78002B3EF4CBAD059B1B68DB0441F11B
:10620800B9857F4B9B8807EE903AF8EEE77A7D4A8E
:1062180092ED012AD2ED022A92ED033AD2ED043A28
:1062280092ED054AD2ED064A92ED075AD2ED085A88
:1062380092ED096AD2ED0A6A92ED0B7AB4EE672AFA
:10624800F1EE10FAF4EE672A14BF01230023F1EEF1
:1062580010FAB4EE673A18BF43F00103F1EE10FAF2
:10626800F4EE673A18BF43F00103F1EE10FAB4EE0A
:10627800674A18BF43F00103F1EE10FAF4EE674ADB
:1062880018BF43F00103F1EE10FAB4EE675A18BFD5
:1062980043F00103F1EE10FAF4EE675A18BF43F029
:1062A8000103F1EE10FAB4EE676A18BF43F0010378
:1062B800F1EE10FAF4EE676A18BF43F00103F1EE4D
:1062C80010FAB4EE677A18BF43F00103F1EE10FA42
:1062D80018BF43F00103002B41F0E48492ED007AEB
:1062E800B4EE677AF1EE10FA41F0DC84DFF80C9135
:1062F800D4F89421D9F800309A4201F2DA8498F857
:106308000030012B3EF443AD94F89021002A3EF46E
:106318003EAD0B2B18D801229A4040F6030112EA31
:10632800010718D112F4C06F0ED0093B012B0BD80E
:10633800452015F085FFFF2015F082FF324815F043
:106348006BFF384615F07CFF2B4BD9F800205A60BC
:106358000B2388F80030002384F89031FEF717BD2E
:106368002A4B1B78002B01F073841A200EF064F876
:10637800002841F06D8494F89031002B41F0688436
:10638800092388F800301CF0BFFB31E71A200EF013
:1063980053F80028F7D01E4B1B88002BF3D11D4B58
:1063A8004520D3F8009015F04BFF0E2015F048FF5C
:1063B80048461CF0EDF8DDF8209048461CF0E8F857
:1063C800154A4FF480510A234846118088F8003056
:1063D8001CF0F0F8D7E700BF3C5D00207A490020A8
:1063E800685D0020E05E00205CD00208FC570020B9
:1063F8008C640020000000809C640020F062002073
:10640800E03C0020E83B0020F8D8020804360020D1
:10641800006300201063002094640020443E0020A4
:106428006860002015F0C6FE1CF088FB00283FF4C9
:10643800DFAE15F0E1FE00283FF4DAAEB44A4FF4BF
:1064480080510A23118088F80030D1E615F0B2FE99
:10645800B04B002105208DE80300A3F1080202914A
:1064680053201DF01DF800287FF4C2AEAA4A082365
:10647800106088F80030BBE615F09CFEA74A02922F
:10648800A2F10C03252101930091A2F10A035021E6
:10649800163A49201DF004F800287FF4A9AE9E4B57
:1064A8004FF0FF3107221860596088F800209FE6F6
:1064B800DFF8649215F07EFE994AD9F80430126824
:1064C80064339342BFF494AE402015F057FE002881
:1064D8007FF48EAED9F8003092494FF0400A0FE0B1
:1064E800069115F0ADFE0699D9F800300A68013317
:1064F800013ABAF1010A0A60C9F8003001F02E85A4
:10650800894AD35C1846002BEAD100234FF0FF32AA
:10651800C9F800300423C9F8042088F8003067E679
:10652800824B1B78DA077FF563AE80201EF00EF9E8
:1065380008B109F00DF90FF049FA59E6784B764A97
:106548001B68536077490023136003220B6088F8A7
:1065580000204DE6764BDFED777A93ED080AB4EE2E
:10656800E70AF1EE10FA41F2D98022F0BBFCD4ED33
:10657800467A20EE270A22F01FFCB0F5617F01F36E
:10658800508107EE900AF8EEE76ADFED6B7A66EE67
:10659800A76A07EE907AB8EEE77AFDEEE67A17EE8C
:1065A800903A2033402B41F2A1839FED640A22F0F8
:1065B80003FC00B207EE900AB8EEE77ADFF888A18C
:1065C800DAED037A77EE877ACAED037AFDF7E6BB50
:1065D8000B9B002B01F0C281FDEEC67A12AA17EEC2
:1065E80090EAFDEEC47A564D564E17EE903AFDEEFF
:1065F800E37A02EB880C17EE907A14E0FDEEC77A86
:1066080017EE909A4F4503DC9945C846A8BF9846AF
:1066180007EE908AF8EEE77A6245E6EC017A05F132
:1066280010053DF409AB95ED007AF2EC017AE7EE3E
:10663800267AB846B0EE637AA5EE277AF0EE477A66
:106648000028DBD031B1F4EE473AF1EE10FAC8BFBA
:10665800F0EE467AFDEEE77AF04617EE909ACE45D0
:10666800D2DDD5E70B9B002B01F01781FDEEE37A15
:1066780012AB17EE906AFDEEC47A314A314D17EE2F
:1066880090EAFDEEC67AB1EE455A17EE907A03EB22
:10669800880C14E0FDEEC77A17EE908AB04503DB4C
:1066A800F045A8BFF046C14607EE909AF8EEE77AA3
:1066B8006345E5EC017A02F110023DF4BDAA92EDC2
:1066C800007AF3EC017AE7EE267AB146B0EE447A26
:1066D800A5EE277AF0EE477A0028DBD0B84631B12C
:1066E800B4EE637AF1EE10FA48BFF0EE467AFDEEAA
:1066F800E77A17EE909AB94504DBF14517EE908AD0
:10670800A8BFF04607EE908AF8EEE77AD0E700BF18
:106718009464002088B502089C640020DAB302085B
:10672800F0620020FC49002064B30208855B002069
:10673800A03600208FC2753CD06D393A00000000A9
:10674800183C002064350020443E0020002940F019
:10675800E585E7EE267AE249BDEEC47A17EE105ACF
:10676800B0EE637AA5EE277A2846F0EE477AFDEE7A
:10677800E77ABDEEC67A17EE906A17EE102AB54290
:10678800A8BF3046B242C8BF104607EE900AF8EEDE
:10679800E77AB8F1010FC1ED007A3DF449AA93ED0B
:1067A800047ADDED137AE7EE267AB0EE637AA5EE89
:1067B800277AFDEEC77A17EE906A17EE900AAE4276
:1067C800A8BF28469642B8BF104607EE900AF8EED2
:1067D800E77AB8F1020FC1ED017A3DF429AA93EDE9
:1067E800087ADDED147AE7EE267AB0EE637AA5EE44
:1067F800277AFDEEC77A17EE906A17EE900AAE4236
:10680800A8BF28469642B8BF104607EE900AF8EE91
:10681800E77AB8F1030FC1ED027A3DF409AA93EDC6
:106828000C7ADDED157AE7EE267AB0EE637AA5EEFE
:10683800277AFDEEC77A17EE906A17EE900AAE42F5
:10684800A8BF28469642B8BF104607EE900AF8EE51
:10685800E77AB8F1040FC1ED037A3DF4E9A993EDA5
:10686800107ADDED167AE7EE267AB0EE637AA5EEB9
:10687800277AFDEEC77A17EE906A17EE900AAE42B5
:10688800A8BF28469642B8BF104607EE900AF8EE11
:10689800E77AB8F1050FC1ED047A3DF4C9A993ED83
:1068A800147ADDED177AE7EE267AB0EE637AA5EE74
:1068B800277AFDEEC77A17EE906A17EE900AAE4275
:1068C800A8BF28469642B8BF104607EE900AF8EED1
:1068D800E77AB8F1060FC1ED057A3DF4A9A993ED61
:1068E800187ADDED187AE7EE267AB0EE637AA5EE2F
:1068F800277AFDEEC77A17EE906A17EE900AAE4235
:10690800A8BF28469642B8BF104607EE900AF8EE90
:10691800E77AB8F1070FC1ED067A3DF489A993ED3E
:106928001C7ADDED197AE7EE267AB0EE637AA5EEE9
:10693800277AFDEEC77A17EE906A17EE900AAE42F4
:10694800A8BF28469642B8BF104607EE900AF8EE50
:10695800E77AB8F1080FC1ED077A3DF469A993ED1C
:10696800207ADDED1A7AE7EE267AB0EE637AA5EEA4
:10697800277AFDEEC77A17EE906A17EE900AAE42B4
:10698800A8BF28469642B8BF104607EE900AF8EE10
:10699800E77AB8F1090FC1ED087A3DF449A993EDFA
:1069A800247ADDED1B7AE7EE267AB0EE637AA5EE5F
:1069B800277AFDEEC77A17EE906A17EE900AAE4274
:1069C800A8BF28469642B8BF104607EE900AF8EED0
:1069D800E77AB8F10A0FC1ED097A3DF429A993EDD8
:1069E800287ADDED1C7AE7EE267AB0EE637AA5EE1A
:1069F800277AFDEEC77A17EE906A17EE900AAE4234
:106A0800A8BF28469642B8BF104607EE900AF8EE8F
:106A1800E77AB8F10B0FC1ED0A7A3DF409A993EDB5
:106A28002C7ADDED1D7AE6EE877AE5EE273AFDEE63
:106A3800E37A17EE903A9D42A8BF1D469342A8BF3D
:106A48002A4607EE902AF8EEE77AC1ED0B7AFDF7B1
:106A5800EFB80BF0F1FA0646FDF78AB9214B1A6830
:106A680012F080522DD0B6EE007A67EE877AF4EEF7
:106A7800E27AF1EE10FA3FF792ABFFF785BBC70059
:106A88003EF5E9AAFDF791B917491848184BD1ED19
:106A9800003A90ED004A17491B78C4ED7E7A84EDE0
:106AA8007C4AC4ED7D3AD1ED006A002B3CF458A92C
:106AB800012384F8FC31FCF753B9F0EE647AFCF753
:106AC800E0BB079B13F4800201D00022CBE7B6EEAF
:106AD800007AF4EEC72AF1EE10FAC4DCFCF752BCD7
:106AE800643500208C6400201C630020DC3C0020FE
:106AF800903E0020EC3C0020FDEEC67A12AB17EE6B
:106B0800905AFDEEC47ACE4ACE4817EE90EA03EBCF
:106B18008806D2ED007AB3EC017AA6EEA77A103295
:106B2800F0EE635AE5EE075A07EE905AB0EE657A32
:106B380031B1F4EE653AF1EE10FAC8BFB0EE467A1C
:106B4800BDEEC77A17EE107ABD4204DC7745A8BFC0
:106B5800774607EE907AF8EEE77A9E42E0EC017A03
:106B6800D7D1FCF7B9BD012A40F38E8707EE101A7A
:106B7800B8EEC77AC7EE876AB1EEE68AB9F1030FB5
:106B880014D0BAF1000F09D007EE90AAF8EEE77A10
:106B9800B4EEE78AF1EE10FA01F315812B6E03EBE0
:106BA800560393FBF6F3EB62FFF740BAB0EE480AE0
:106BB80022F002F900B2E4E7012A7FF76BAA07EE98
:106BC800101AB8EEC77AC7EE876AB1EEE68AFFF701
:106BD80063BA012A40F38B8707EE101AB8EEC77A1A
:106BE800C7EE876AB1EEE68AB9F1030F14D0BAF19D
:106BF800000F09D007EE90AAF8EEE77AB4EEE78A1C
:106C0800F1EE10FA01F3DF806B6E03EB560393FB92
:106C1800F6F32B63FFF724BAB0EE480A22F0CCF85B
:106C280000B2E4E7B4F81431D80540F101879AEDD1
:106C3800017A854BDAED006ADAED027A069A0D934D
:106C4800BDEEC77AB3F90670118B17EE103AFDEE58
:106C5800E66AFDEEE77A16EE902AADF84A3017EEAE
:106C6800903AADF84820ADF84C30784A784DB2F9F2
:106C78000230B2F9002073489FED767AD0ED007AA1
:106C880075484FF47A7603F5E16306FB03F302F5E2
:106C9800E16206FB02F285FB03E61E44DB17C3EB49
:106CA800E62C0D9B00781E880C9077EEC77A85FB42
:106CB80002E51544FDEEE77AD217761AC2EBE52213
:106CC80098885D88B3F808E0ADF85060ACF5FA73C1
:106CD8000D9EADF8603017EE903A6D1AA2F5FA7273
:106CE800401AADF86220ADF84E307289B389ADF81C
:106CF8005250F589ADF85400584E0C987F1AAEEBF7
:106D0800010E521A5B1A6D1A0021ADF85670ADF8D3
:106D180058E0ADF85A20ADF85C30ADF85E503160FF
:106D28007160B160F160002801F055804C4B4D4F07
:106D38000697DFF838810E9489461F463CE01EAB63
:106D480003EB440030F9300C3880069B98F902E0D8
:106D58000D441EFB00F053F82550012303FA04F4F8
:106D6800414B83FB003EC017079B2C42C0EB6E10C3
:106D78000CBF01244FF0FF3498420EDB0B9B02FB43
:106D880003F2394B83FB0253D217C2EB6313A3EB15
:106D98000C031BB28342A8BF034636F8112003FB3D
:106DA800042326F811300C9B09F10109994508F1D3
:106DB800070807F1020769DA98F80630002B37D17F
:106DC80098F8001098F905200B924D00069A98F94A
:106DD800043098F803E098F80140681802EB800046
:106DE800C2888088121A92B21F4802FB03F380FB04
:106DF80003C0DB17C3EB60134FEA520CA3EB0C0381
:106E08001BB20793BEF1000F99D01EAB03EB440AE7
:106E1800B7F900003AF930AC504529DA8644704594
:106E280003DCF2455046A8BF704600B238808CE7B4
:106E38001633D8B20DF000FB0028C1D13880B2E774
:106E4800183C00206435002080710020B0600020CC
:106E5800C5B3A2910080BB44EC4600205435002005
:106E6800EC1D00203C4800201F85EB51F046002017
:106E78007FF76BAFA0EB0E0ED64503DB7045A8BFBE
:106E8800704682460FFA8AF038805EE70E9C069FAD
:106E980097F90A0033886B4A6B4910FB03F3F87AB9
:106EA800097882FB0352FF284FEAE373C3EB6212AF
:106EB80000F0A784814240F2A4840D9B33F91000AE
:106EC80097F916507388104430805E4AF87D15FB98
:106ED80003F382FB0352FF284FEAE373C3EB62120A
:106EE80000F08B84814240F288840D9B33F91000B6
:106EF80097F92250B38810447080524A97F82300BB
:106F080015FB03F382FB0352FF284FEAE373C3EB3D
:106F1800621200F06E84814240F26B840D9B33F95B
:106F2800100097F92E50F3881044B080454A97F81E
:106F38002F0015FB03F382FB0352FF284FEAE3738C
:106F4800C3EB621200F05184814240F24E840D9BE3
:106F580033F9100097F93A5033891044F080394AD0
:106F680097F83B0015FB03F382FB0352FF284FEA17
:106F7800E373C3EB621200F03484814240F231843F
:106F88000D9B33F9100097F94650738910443081EE
:106F98002C4A97F8470015FB03F382FB0352FF289E
:106FA8004FEAE373C3EB621200F01784814240F2A8
:106FB80014840D9B33F9100097F95250B38910448B
:106FC8007081204A97F8530015FB03F382FB0352A4
:106FD800FF284FEAE373C3EB621200F0FB838142A0
:106FE80040F2F8830D9B33F9100097F95E50F3894E
:106FF8001044B081134A97F85F0015FB03F382FB36
:107008000352FF284FEAE373C3EB621300F0DF83F8
:10701800884280F0DC830D9A32F9102005990968BE
:1070280007911344F3810B46FCF78CBBF0EE427AD0
:10703800FCF727B98223FEF7CABEDFED047AFEF714
:1070480092BE00BF1F85EB51B860002000000243CC
:10705800FDEEE77A17EE105A17EE906AFDEEC67A43
:10706800B54217EE902A17EE100AA8BF3046B24272
:10707800C8BF104607EE900AF8EEE77AB8F1010F9C
:10708800C1ED007A3CF4D4AD93ED047ADDED137ACA
:10709800E7EE267AB0EE447AA5EE277AFDEEC77AB7
:1070A80017EE906A17EE900AAE42A8BF284696429D
:1070B800B8BF104607EE900AF8EEE77AB8F1020F6B
:1070C800C1ED017A3CF4B4AD93ED087ADDED147AA4
:1070D800E7EE267AB0EE447AA5EE277AFDEEC77A77
:1070E80017EE906A17EE900AAE42A8BF284696425D
:1070F800B8BF104607EE900AF8EEE77AB8F1030F2A
:10710800C1ED027A3CF494AD93ED0C7ADDED157A7D
:10711800E7EE267AB0EE447AA5EE277AFDEEC77A36
:1071280017EE906A17EE900AAE42A8BF284696421C
:10713800B8BF104607EE900AF8EEE77AB8F1040FE8
:10714800C1ED037A3CF474AD93ED107ADDED167A57
:10715800E7EE267AB0EE447AA5EE277AFDEEC77AF6
:1071680017EE906A17EE900AAE42A8BF28469642DC
:10717800B8BF104607EE900AF8EEE77AB8F1050FA7
:10718800C1ED047A3CF454AD93ED147ADDED177A31
:10719800E7EE267AB0EE447AA5EE277AFDEEC77AB6
:1071A80017EE906A17EE900AAE42A8BF284696429C
:1071B800B8BF104607EE900AF8EEE77AB8F1060F66
:1071C800C1ED057A3CF434AD93ED187ADDED187A0B
:1071D800E7EE267AB0EE447AA5EE277AFDEEC77A76
:1071E80017EE906A17EE900AAE42A8BF284696425C
:1071F800B8BF104607EE900AF8EEE77AB8F1070F25
:10720800C1ED067A3CF414AD93ED1C7ADDED197AE4
:10721800E7EE267AB0EE447AA5EE277AFDEEC77A35
:1072280017EE906A17EE900AAE42A8BF284696421B
:10723800B8BF104607EE900AF8EEE77AB8F1080FE3
:10724800C1ED077A3CF4F4AC93ED207ADDED1A7ABF
:10725800E7EE267AB0EE447AA5EE277AFDEEC77AF5
:1072680017EE906A17EE900AAE42A8BF28469642DB
:10727800B8BF104607EE900AF8EEE77AB8F1090FA2
:10728800C1ED087A3CF4D4AC93ED247ADDED1B7A99
:10729800E7EE267AB0EE447AA5EE277AFDEEC77AB5
:1072A80017EE906A17EE900AAE42A8BF284696429B
:1072B800B8BF104607EE900AF8EEE77AB8F10A0F61
:1072C800C1ED097A3CF4B4AC93ED287ADDED1C7A73
:1072D800E7EE267AB0EE447AA5EE277AFDEEC77A75
:1072E80017EE906A17EE900AAE42A8BF284696425B
:1072F800B8BF104607EE900AF8EEE77AB8F10B0F20
:10730800C1ED0A7A3CF494AC93ED2C7ADDED1D7A4C
:10731800E6EE877AA5EE274AFEF70EB9E7EE267A5B
:10732800ED49BDEEC47A17EE105AB0EE637AA5EEB9
:10733800277A2846F0EE477AF4EEE37AF1EE10FA6F
:10734800B8BFF0EE467AFDEEE77ABDEEC67A17EEE4
:10735800906A17EE102AB542A8BF3046B242C8BF9D
:10736800104607EE900AF8EEE77AB8F1010FC1ED82
:10737800007A3CF45DAC93ED047ADDED137AE7EE28
:10738800267AB0EE637AA5EE277AB4EEE37AF1EEC8
:1073980010FAF0EE477AB8BFF0EE467AFDEEE77ADB
:1073A80017EE906A17EE900AAE42A8BF284696429A
:1073B800B8BF104607EE900AF8EEE77AB8F1020F68
:1073C800C1ED017A3CF434AC93ED087ADDED147A22
:1073D800E7EE267AB0EE637AA5EE277AB4EEE37A82
:1073E800F1EE10FAF0EE477AB8BFF0EE467AFDEE0D
:1073F800E77A17EE906A17EE900AAE42A8BF2846C1
:107408009642B8BF104607EE900AF8EEE77AB8F150
:10741800030FC1ED027A3CF40BAC93ED0C7ADDED71
:10742800157AE7EE267AB0EE637AA5EE277AB4EEFF
:10743800E37AF1EE10FAF0EE477AB8BFF0EE467A4A
:10744800FDEEE77A17EE906A17EE900AAE42A8BFF3
:1074580028469642B8BF104607EE900AF8EEE77A3B
:10746800B8F1040FC1ED037A3CF4E2AB93ED107A66
:10747800DDED167AE7EE267AB0EE637AA5EE277A86
:10748800B4EEE37AF1EE10FAF0EE477AB8BFF0EE18
:10749800467AFDEEE77A17EE906A17EE900AAE424A
:1074A800A8BF28469642B8BF104607EE900AF8EEE5
:1074B800E77AB8F1050FC1ED047A3CF4B9AB93ED66
:1074C800147ADDED177AE7EE267AB0EE637AA5EE48
:1074D800277AB4EEE37AF1EE10FAF0EE477AB8BF05
:1074E800F0EE467AFDEEE77A17EE906A17EE900A0C
:1074F800AE42A8BF28469642B8BF104607EE900A8B
:10750800F8EEE77AB8F1060FC1ED057A3CF490ABD6
:1075180093ED187ADDED187AE7EE267AB0EE637A05
:10752800A5EE277AB4EEE37AF1EE10FAF0EE477A98
:10753800B8BFF0EE467AFDEEE77A17EE906A17EEDE
:10754800900AAE42A8BF28469642B8BF104607EE3A
:10755800900AF8EEE77AB8F1070FC1ED067A3CF425
:1075680067AB93ED1C7ADDED197AE7EE267AB0EE7B
:10757800637AA5EE277AB4EEE37AF1EE10FAF0EE2C
:10758800477AB8BFF0EE467AFDEEE77A17EE906AD2
:1075980017EE900AAE42A8BF28469642B8BF1046DA
:1075A80007EE900AF8EEE77AB8F1080FC1ED077A0E
:1075B8003CF43EAB93ED207ADDED1A7AE7EE267ABD
:1075C800B0EE637AA5EE277AB4EEE37AF1EE10FA1C
:1075D800F0EE477AB8BFF0EE467AFDEEE77A17EE9E
:1075E800906A17EE900AAE42A8BF28469642B8BFE6
:1075F800104607EE900AF8EEE77AB8F1090FC1EDE8
:10760800087A3CF415AB93ED247ADDED1B7AE7EEAE
:10761800267AB0EE637AA5EE277AB4EEE37AF1EE35
:1076280010FAF0EE477AB8BFF0EE467AFDEEE77A48
:1076380017EE906A17EE900AAE42A8BF2846964207
:10764800B8BF104607EE900AF8EEE77AB8F10A0FCD
:10765800C1ED097A3CF4ECAA93ED287ADDED1C7AA9
:10766800E7EE267AB0EE637AA5EE277AB4EEE37AEF
:10767800F1EE10FAF0EE477AB8BFF0EE467AFDEE7A
:10768800E77A17EE906A17EE900AAE42A8BF28462E
:107698009642B8BF104607EE900AF8EEE77AB8F1BE
:1076A8000B0FC1ED0A7A3CF4C3AA93ED2C7ADDEDF9
:1076B8001D7AE7EE267AB0EE637AA7EE857AB4EE05
:1076C800E37AF0EE477AF1EE10FAB8BFF0EE467AB8
:1076D800FDEEE77AFDF736BF6435002000000000B4
:1076E800D4F8B86153003EB1981801EB8000767861
:1076F8004078B042BBF4F7A9134401EB830100239F
:10770800C4F8B811A4F82A32C4F82C32FBF7EBB944
:10771800042303250A930220FCF7BABF1FED117A50
:10772800FEF74CBF4FEA8A03CF1804EB030AD84B85
:1077380003EBCC1C5FEA990300F0538301334FEA53
:10774800031E0CEB0E000CF1100307F110010AF1F7
:10775800100213ED024A13ED035A13ED016A13EDFB
:10776800047A51ED024A51ED035A51ED016A51ED87
:10777800047A64EE244A65EE255A66EE266A67EEB8
:10778800277A1033834242ED024A42ED035A42ED12
:10779800016A42ED047A01F1100102F11002D8D118
:1077A800AEF110030CEB0302F918534419F0030966
:1077B8003EF48AA9B2EC017AF1EC017A67EE277AF5
:1077C800B9F10109E3EC017AF4D1FEF77DB9B7F913
:1077D8005C2023E4B7F9500007E4B7F94400FFF749
:1077E800EBBBB7F93800FFF7CEBBB7F92C00FFF7B2
:1077F800B1BBB7F92000FFF794BBB7F91400FFF746
:1078080077BBB7F90800FFF75BBBA24BB6F90A20B4
:107818001B68002B00F0C4821A6001230A93FCF74E
:10782800F1BE07EE907ADFED9C6AB8EEE77A66EE75
:10783800A65A9FED9A5A9FED9A6ADFED9A7AA5EEBD
:10784800856A26EEA55AE5EE867AE5EE276A26EEE3
:10785800870AFEF7ACBE944997F916E00B8897F9AA
:107868000A20B1F9020091491EFB03F3524200FBC2
:1078780002F081FB03E2121181FB00E1DB17C01764
:10788800C0EB2110991AD31A01440344A8EB010153
:107898001D4431807580FBF774BFFDEEC67A12ABCC
:1078A800CDED0C7AFDEEC47A1094CDED0D7AFDEE97
:1078B800E37ACDF844A0DFF810E2DFF8F4C10C9CBD
:1078C800DDF834A00E9517EE909AB1EE455A03EB09
:1078D80088080F979EED007AF3EC017AE6EE877A36
:1078E800B0EE447AA5EE277AF0EE477AE0B9FDEEDD
:1078F800C77A4F4617EE905AA94503DC5545A8BFED
:1079080055462F4607EE907AF8EEE77A002A00F0FF
:107918004B824345ECEC017A0EF1100EDAD1109C43
:10792800DDF844A0FCF788B931B1F4EE473AF1EE3E
:1079380010FAC8BFF0EE467ABDEEE77A07EE904A35
:1079480017EE105AAC4206DC17EE105A5545A8BF80
:10795800554607EE905AF8EEE77AD7E7FDEEE37A58
:107968000DF1480E17EE909AFDEEC47A1094CDED05
:107978000C7AFDEEC67ACDF844A0DFF84CC14C4B2A
:10798800DDF830A0CDED0D7A17EE904A0EEB8808A1
:107998000E950F979CED007AFEEC017AE6EE877A59
:1079A800B0EE637AA5EE277AF0EE477AC0B9FDEE1D
:1079B800C77A4F4617EE905AA94503DC5545A8BF2C
:1079C80055462F4607EE907AF8EEE77A002A00F03F
:1079D800DD81F045E3EC017A0CF1100CDAD19EE779
:1079E80031B1F4EE473AF1EE10FAC8BFF0EE467A3C
:1079F800FDEEE77A254617EE907ABC4204DC57453F
:107A080017EE905AA8BF554607EE905AF8EEE77A57
:107A1800DCE7BEF838109FED277A07EE901AF8EEEB
:107A2800E77A254967EE877AC1ED007AFCF7BDB998
:107A3800DFED227A29EE279A28EE278A68EEA77AC0
:107A4800BDEEC97AFDEEE77A8DED077A17EE903A2A
:107A5800BDEEC87AADF84A3017EE101A0B9BBDF987
:107A68001C20ADF84C20ADF84810002B40F0F580F4
:107A7800134B069A0D93118BB3F90670FFF7F5B8FF
:107A8800DFF848A0FCF7E9B99FED0E8AFFF776B852
:107A9800785200200C58002084F9223F92E741B91F
:107AA8009730083C15A82ABEB06000201F85EB510E
:107AB800643500206F12833A000000203333333FCF
:107AC8008071002000000000183C0020443E002087
:107AD800D04A516900293AF493AECF490888CF4972
:107AE80091FBF0F1106801605374FAF789BE9FEDBD
:107AF800CC8AFFF779B89FEDCB0ACB4B099325EEDB
:107B0800800A21F059F9C94FD4F8AC61F880FDF723
:107B180043BA9AED000A0993079221F04DF9C44936
:107B2800DFF860E3D1F8EC10C04F079A38808EFB7D
:107B3800013EC917C1EBAE1107EE901AF8EEE77ACD
:107B4800099BFDEEE77A17EE901A7980FCF78AB95F
:107B580007EE907AF8EEE78ADFEDB67A9FEDB60A7F
:107B680084F8887168EEA78A38EE800AFDEEC07A3C
:107B780017EE903A2033402B40F230819FEDA80A4F
:107B8800AE4BFDEEE87A83ED010A17EE903A20330A
:107B9800402B00F21D81DFEDAA7AF4EEE78AF1EEC0
:107BA80010FA40F3E581DFEDA76ADFEDA77A01E07F
:107BB800F0EE478AF4EEE78AF1EE10FA38EEE67A4C
:107BC800F6DCDFEDA27AB4EEE77AF1EE10FA40F1D6
:107BD800CC819FED9C6ADFED9E6A01E0B0EE677A8A
:107BE800B4EEE67AF1EE10FA77EE067AF6D49FED67
:107BF800927AF4EEC77AF1EE10FA40F3F6809FED30
:107C0800907A77EE677A27EEA76ADFED925ADFED72
:107C1800926A9FED927AE6EE256A67EE865AA6EE9C
:107C2800267AE5EE877AC4ED637AFDF7B1BC8C4914
:107C38008C4A8E46FDF737BF0AF0FEF9079B7B4F4B
:107C4800D4F8B091D4F8AC61C01A7880FDF7A9BF18
:107C580008981AF0AFFCFEF796BB834B0699B3F968
:107C68000670098B0D938F42BCBF5242ADF84C2071
:107C7800FEF7FBBF0AF0E0F9079B6C4F99F800206C
:107C8800D4F8AC619BF80080C01AB880FEF71AB827
:107C98000AF0D2F9079B654F9BF80080C01A7880DC
:107CA800FDF7D1BD714B1B6803F59C530833C4F82D
:107CB800943198F80030012B7DF469A894F890313C
:107CC800002B7DF464A8BB78032B00F054810DF0E1
:107CD8007DFE012384F89031FDF759B8644B1B7879
:107CE800002B00F08E800023FEF705BADFED547AF2
:107CF800F4EEE76AF1EE10FA40F3EC80DFED515A4A
:107D08009FED516A01E0F0EE676AF4EEC66AF1EEA3
:107D180010FA76EEE57AF6DCDFED4C6AF4EEE67AF8
:107D2800F1EE10FA40F1D380DFED465A9FED486A34
:107D380001E0F0EE667AF4EEC67AF1EE10FA77EE2C
:107D4800A56AF6D4DFED3C7AF4EEE76AF1EE10FAB4
:107D580004DDDFED3B7A77EEE66A68E5DFED457A2C
:107D6800F4EEE76AF1EE10FA44BFDFED387A77EE09
:107D7800E66A5CE5404B1B78002B46D13F4B1B8BDA
:107D880007EE903AF8EEE77AFEF741BA0F9D002D1C
:107D98007FF41FAE0E9DB542B8BFF0EE467A18E6E6
:107DA80001230A93FCF72EBC0F9D002D7FF4B1AD83
:107DB8000E9DB542B8BFF0EE467AAAE5294901F111
:107DC800800EFDF765BFF880A5F8A860FAF792BEA7
:107DD800DFED137A27E72A4FFFF75AB805F096F92F
:107DE800CEE6534639466246E0E49FED227AF4EE49
:107DF800C77AF1EE10FA44BF9FED147A77EE677AEE
:107E080001E706F033FDFAF76EBEDFED057AFEF7FF
:107E1800FEB900BFD0620020E862002020A1070060
:107E2800000000000000C842405200205C3D0020D5
:107E3800B814002035FA8E3CDB0FC93F0000002043
:107E4800DB0F4940DB0FC940E4CB1641DB0F49C0CB
:107E5800E4CB16C192E741B99730083C15A82ABE71
:107E6800F8530020E41B002080710020F0620020FD
:107E7800423E0020DB0FC9BF903E0020683E002034
:107E88003C480020D34D62109BF80010132924D0E1
:107E98004BB106F5F460B0EE480A2844D5F89C3793
:107EA8009847B0EE408A9BF80030132B7CF4AFAFB4
:107EB800B0EE480A20F080FFA8F80200FCF7A9BF3E
:107EC80094F8E431002B7AF4BDACFAF7A6BCF0EED6
:107ED800676A37E7F0EE667A1EE7B0EE480A07935E
:107EE80020F06AFF079BA8F80000D1E7DFF8A4900C
:107EF800D9F8000005F0D4FF224B1B780022022B92
:107F0800C9F800207EF471A907F03AFCFEF76DB9B4
:107F1800099BD3ED03DA1C4B93ED020A1B4B3CEE95
:107F28006DDA28EE800A20EE0D0A83ED020AFAF7D0
:107F380020BE94F8D431002BEAD1134B2B4493ED97
:107F4800000A059BD3ED01DA28EE800A3CEE6DDAD3
:107F580020EE0D0A88ED000AFAF70BBE0C4AD35C36
:107F6800002B7EF445A9FEF7D0BAF0EE477A3EE63C
:107F7800B0EE687A25E680201CF0E8FB00287CF447
:107F880006AFA4E6943500206C4700202C3500206D
:107F980064B30208004A00202DE9F04F2DED028B52
:107FA8008FB0064617F080FB9C4B1F7827B10FB0A7
:107FB800BDEC028BBDE8F08FDFF8C0B2DBF8003013
:107FC8005C05F4D5964B974D1B78002B40F05C81EF
:107FD800954B1B78002B6BD0944C954AD4F86431A0
:107FE800F31A934201F2398094F86C81B8F1000FCA
:107FF80031D1904F386808F0C7F9C0B201280ED9BE
:10800800022841F0B5838C4B1A78002A41F0A385E9
:10801800D4F87021B21AB2F57A6F81F0A686D4F836
:108028007431002B44D094F86C31BBB9834B1B6876
:108038009B7801211E3B00228B4284F86C1184F846
:10804800802141F2E98538680221043017F034FABA
:1080580094F878310FE0D4F874314BB3D4F87C310C
:1080680040F6B732F31A934222D994F87831002BAC
:1080780001F0B3826F4F013BDBB284F87831002BFB
:1080880001F04480D4F8741194F8802111F801EBC0
:1080980094F88131C4F8741172440133386884F853
:1080A8008021714684F8813108F072F9C4F87C6146
:1080B800634B2F681B7853B1DFF8C481D8F80000F0
:1080C80028B1604B1B78013B012B41F22E805E4B9F
:1080D8001B7863B15D4F3B684BB1544CD5F80090A9
:1080E800D4F8B832A9EB0303632B00F21B87584C72
:1080F8002378022B01F05282DFF8888198F800304B
:10810800032B00F0EF87534B1B7873B1524F3B683A
:108118005BB1464C09F090FFD4F8C032009044F6A9
:108128001F62C31A934200F27D814C4B1B78002BCF
:108138004BD14B4B1B7843B13C4CD4F8103403F56E
:10814800C333A0339E4280F04987464B1B78002BEF
:108158003FF42DAF354E444C444D06F2314720686C
:1081680008F012F900283FF422AF206808F008F957
:108178002B7880465A1E33B120682A7008F004F91B
:108188000028F2D113E703223946781E22F012FFA5
:1081980096F8303496F8312486F8338483F47F4394
:1081A80083F0FF039B1A1FFA88F89BB2B8EB132FD2
:1081B800D5D196F83224DBB29A42D0D1781E10F08D
:1081C80085FA2B7818442870C9E7294C2278002AA8
:1081D80040F0E886154CD4F8083403F5C333A033CF
:1081E8009E42A6D3234A94F80C34C4F80864D55C9C
:1081F800E90701F1B083AA0701F16C836B0701F16C
:1082080083821D4A94F80C341178013393FBF1F200
:1082180001FB123384F80C348BE700BFCD5B0020E0
:10822800485C0020F0620020525C00201C1E0020E8
:108238003F0D0300EC5B002008000020F05B0020ED
:10824800545C00205C5C0020645C0020F865002021
:10825800BA4400206C5C0020705C0020D85C0020D0
:10826800E65C0020765C00207C5C0020805C0020BE
:10827800405C0020E05C0020E55C002050430020CA
:10828800E85B0020190100205C4C2A68D4F85C31B6
:10829800D31A7C2B7FF69CAE94F86031DFF87C9182
:1082A8009FED578AC4F85C21013384F860314FF0A0
:1082B8002408404617F0A6F9524BF9EC016A1B8ACC
:1082C80007EE103AF8EEE66AB8EEC77A08F1010848
:1082D800C6EE877A5FFA88F867EE887AFDEEE77A65
:1082E800CDED007ABDF900A05FFA8AF017F066F9C3
:1082F800CAF3072017F062F9B8F1270FD9D1302057
:1083080017F080F9DFF81881002017F057F90020DE
:1083180017F054F9D8F800005E2108F039F894F8FD
:10832800603113F003092DD1D4F85C2141F2883370
:108338009A4201F2FE84142017F064F9324B334A52
:10834800B3F9043082FB03124FEAE379C9EBA209BF
:108358000FFA89F95FFA89F017F030F9C9F30720A5
:1083680017F02CF91C2017F04DF9002017F026F90A
:10837800002017F023F95E21D8F8000008F008F86B
:1083880094F8603113F0070901F05C83282B7FF41F
:108398001FAE00271720D5F8009084F8607117F0F9
:1083A80031F9384617F00AF9194B1A4CA3FB09237F
:1083B8009B0BA4FB03125209C2EB0212A3EB82032C
:1083C800D8B217F0FBF8182017F01CF9124BA3FBD2
:1083D80009239B09A4FB03125209C2EB0212A3EB67
:1083E8008203D8B217F0EAF8384617F0E7F8D8F859
:1083F80000005E2107F0CCFFEAE500BF1C1E00204C
:1084080000007A446C600020B060002067666666F1
:1084180073B2E74589888888D34D6210A060002030
:10842800F45B002094F8C632002B41F04B81E34BFB
:108438001A6802F00803002B48F603414AF60B407D
:108448004BF60F4349F6074804BF0346884612F027
:10845800040F4FF0190118BF9846920684F8C61207
:1084680003D548F4804848F02008D54B1A79C8F35A
:1084780009010191002A41F0DD845B79002B41F06C
:10848800B1849A4664204FF0FF330A464FF0000942
:10849800CDF81880CDF81C800892ADF826A0ADF86C
:1084A80028308DF83600ADF82490CDF82A90CDF814
:1084B8002E90CDF832900DF1180CBCE80F00DFF8C3
:1084C80010E384F85190AEE80F009CE80F00AEE886
:1084D80007002EF8023B71464FF0010C1B0C4FF0C1
:1084E800FE0E1F20C82201F81E3984F84EE084F8D9
:1084F800522084F853C084F84F0094F8D60284F8C8
:10850800500080F0F10383EA0313DAB2130983F011
:10851800E70343EA022383EAC2031BB283EA031296
:10852800D2B2C3F3072383EA121343EA022383EA8E
:10853800C2031BB283F0C80282EA0212D2B2C3F3AA
:10854800072383EA121343EA022383EAC2031BB216
:1085580083EA0C0E8EEA0E1E5FFA8EFEC3F3072224
:1085680082EA1E1242EA0E22604482EACE0E84F8A3
:10857800D602A4F84CE001F11F0011F8013B83EA90
:108588000E0383EA0313DBB21A0982EA1E2242EAC7
:10859800032282EAC3031BB21FFA83FE8142A4F8B6
:1085A8004CE0EAD183F07C0383EA0313DBB21A09B7
:1085B80082EA1E2E8EEA032E8EEAC30E0FFA8EFE74
:1085C8001FFA8EF34FEA132A5FFA8EFEA4F84C3096
:1085D800DFF8009284F874A004F16E0384F873E065
:1085E80004F14E0C0193DCF80C30DCF80000DCF8E8
:1085F8000410DCF80820C846A8E80F00019B0CF11D
:10860800100C9C45C146EED1DCF80000C8F800000B
:10861800DFF8C4819CF8043089F8043008F1270990
:1086280084F825E384F826A318F8011F386807F0B2
:10863800AFFEC145F8D194F8C722002A41F047801F
:1086480060492B6808780A2184F8C712002801F0CD
:108658003781DFF888C10128BCF80010059141F284
:108668005985BCF802100291022801F0FF83BCF87A
:1086780004100391032801F03385BCF8061001911A
:10868800042801F027850528BCF8081001F01D858D
:108698000628BCF80AA001F014850728BCF80CE0ED
:1086A80001F00085BCF80E9094F8D6220693104687
:1086B80080F0300383EA0313DBB20490424A9DF84A
:1086C80010C0128884F850C0180980F07A0040EA77
:1086D800032080EAC3033D48C2EB022280FB02C0AC
:1086E8001044D217C2EB602205988DF82D204FF068
:1086F800000860F30F0803984FF0000C60F30F0CAC
:1087080000201BB261F30F0000216EF30F0183EA12
:10871800031EC3F307230393029B63F31F48019BC4
:10872800CDF81C8063F31F4C039BCDF820C05FFA83
:108738008EFE6AF31F4069F31F4183EA1E134FF050
:10874800000A09900A918DF82CA043EA0E2C0DF12D
:108758001809B9E80F008CEACE0E0FFA8EFE8EF0DB
:10876800C808DFF86CC084F851A088EA08185FFAD6
:1087780088F8CEF3072EACE80F008EEA181E4EEAF2
:10878800082399E8030083EAC8080FFA88F383F0FE
:1087980023024CF8040B82EA0210C0B2C3F307228A
:1087A80082EA1012049B2CF8141942EA0022591C80
:1087B80082EAC0004FF02308162211E05052002030
:1087C800E05E0020B86000205035002003082080BB
:1087D800701E00201C2100201B2100208071002019
:1087E8004FF0FE0EC82384F8D612A4F84C000CEB08
:1087F800020184F8538084F84EE084F84F2084F80E
:1088080052301CF8013B434083EA0313DBB21A09D8
:1088180082EA102242EA032282EAC3031BB298B218
:108828008C45A4F84C00ECD183F0F40383EA0313DD
:10883800DBB24FEA131E8EEA102E8EEA032E8EEA62
:10884800C30EA0460FFA8EFE1FFA8EF958F84E0F87
:10885800DFF81CC4A4F84C904FEA192A5FFA8EFE80
:1088680084F86AE084F86BA0D8F80410D8F80820D7
:10887800D8F80C30ACE80F00D8F81000D8F814106D
:10888800D8F8182004F21D39ACE8070004F2FF28D4
:1088980084F81DA384F81CE318F8011F386807F052
:1088A80077FDC145F8D194F8CEE2BEF1000F40F053
:1088B8001787E84B94F8D6C2B3F90010B3F9022031
:1088C800B3F904309FEDE46A84F851E007EE103AFA
:1088D8002B6806938CF06A0383EA031306EE901A5A
:1088E800D9B20B0983F0D50343EA012383EAC10314
:1088F8001BB283EA03115242C9B207EE902AC3F3AE
:10890800072383EA111343EA0123F8EEE77AF8EE26
:10891800E66AB8EEC77A83EAC1031BB267EE867AC5
:1089280066EE866A27EE067A002083F0C805CDED4C
:10893800087ACDED076A8DED097A0A900B900C90B4
:1089480085EA05150DF11809EDB2C3F30728B9E852
:108958000F0088EA151848EA052888EAC505DFF8EF
:1089680014832DB2A8E80F0085F01E0E99E80700C1
:108978008EEA0E13DBB2C5F3072E8EEA131E4EEAFB
:10898800032E88E807008EEAC30EA8F110051C2004
:10899800C8214FF005091E234FF0FE080CF1010213
:1089A80084F8521084F8CE9284F8533084F84E80BC
:1089B80084F84F00291884F850C0A4F84CE084F8D3
:1089C800D62215F8013B83EA0E0383EA0313DBB2D0
:1089D8001A0982EA1E2242EA032282EAC3031BB270
:1089E8001FFA83FE8D42A4F84CE0EAD183F02703F6
:1089F80083EA0313DBB21A0982EA1E2E8EEA032EDB
:108A08008EEAC30E0FFA8EFE1FFA8EF34FEA132971
:108A18005FFA8EFEDFF85882A4F84C3084F8719023
:108A280084F870E004F14E0C04F16E0ADCF80000E2
:108A3800DCF80410DCF80820DCF80C3045460FC5DB
:108A48000CF1100CD445A846F0D1844DBCF8003088
:108A5800A8F8003005F1240884F822E384F8239369
:108A680015F8011F386807F093FC4545F8D194F8CC
:108A7800CF320193002B40F02F8694F8D682754BA5
:108A8800774AB3F90410B2F90620DFF8ECC1754D46
:108A9800DFF8E09184F8508088F0220383EA03131A
:108AA800DBB2180980F05900B2F5FA6F40EA0320EA
:108AB80080EAC303A8BF4FF4FA621BB2B2F57A7F0B
:108AC80083EA0310B8BF4FF47A72C0B24FF0640E55
:108AD800A2F57A72C3F307230EFB02F283EA10139E
:108AE80085FB02E543EA00238CFB01CED217C917A8
:108AF8004FF0000AC2EBA512C1EBAE0183EAC00336
:108B08001DB2CDF818A00DF1180CADF82A20ADF85B
:108B18002810CDF81CA0CDF820A0CDF824A085F011
:108B2800C80ECDF808C0BCE80F008EEA0E1E5FFA2A
:108B38008EFEC5F3072585EA1E1545EA0E25A9E828
:108B48000F0085EACE0212B282F04A0383EA0313C9
:108B5800DBB2C2F3072181EA1311DCF8002049F8DF
:108B6800102941EA0321052081EAC303142508F1ED
:108B780001029DF8041084F8CF024FF04A0C4FF020
:108B8800FE0EC82084F8511084F8D62209EB05019E
:108B980084F84F50A4F84C304A4684F853C084F8FF
:108BA8004EE084F852001D4612F8010B684080EA36
:108BB8000010C0B2030983EA152343EA002383EABD
:108BC800C00000B285B28A42A4F84C50ECD180F0C3
:108BD800140080EA0010C0B24FEA101E8EEA152E6B
:108BE8008EEA002E8EEAC00E25460FFA8EFE1FFA78
:108BF8008EF855F84E0FDFF878C0A4F84C804FEA8D
:108C0800182A5FFA8EFE84F869A084F868E069681B
:108C1800EB68AA68ACE80F00286969692B8BACE897
:108C2800030004F2FF25ACF80030A84684F81BA323
:108C380084F81AE304F21B3A18F8011F386807F0A1
:108C4800A7FBC245F8D1084B084A1B781278013BAC
:108C580014E000BFB060002088C3E43A1B21002064
:108C680080710020D34D6210B0350020855B002054
:108C78001C210020701E00206766666612F0010045
:108C8800DBB214BFC0224022172B04D8CA490B44B8
:108C980093F824300193C94B19888B071ABF002316
:108CA80042F01002012311F4027F18BF022311F0D1
:108CB800100F18BF062311F0200F18BF102300282B
:108CC80041F04B80032194F8D6E206938EF04603D8
:108CD80083EA0313D8B2030983F0920343EA00231B
:108CE80083EAC0031BB283EA0310C0B2C3F30728A8
:108CF80088EA101848EA002888EAC0080FFA88F8B5
:108D080088F0C80C9DF804008DF81C008CEA0C1C37
:108D180000235FFA8CFC8DF81E200320029A8DF840
:108D28001D30C8F307288DF81F108DF8200088EA39
:108D38001C1807CA48EA0C2888EACC0C0FFA8CFCE5
:108D48008CEA0C18A9E803005FFA88F8CCF307212D
:108D580081EA181141EA082181EAC80894F854C048
:108D680089F800200FFA88F28CEA020C8CEA0C1CB5
:108D78005FFA8CFCC2F3072282EA1C1242EA0C2238
:108D880094F8550094F8561094F8579094F8588031
:108D980084F8533082EACC0212B2504080EA0010C4
:108DA800C0B2C2F3072282EA101242EA002282EA23
:108DB800C00212B2514081EA0111C9B2C2F30722BE
:108DC80082EA111242EA012282EAC10212B289EA57
:108DD800020989EA09195FFA89F9C2F3072282EAC6
:108DE800191242EA092282EAC90212B288EA020882
:108DF80088EA08185FFA88F8C2F3072282EA18128C
:108E080042EA082294F859C094F85A0094F85B1082
:108E180094F85C9084F8513082EAC80212B28CEA65
:108E2800020C8CEA0C1C5FFA8CFCC2F3072282EA63
:108E38001C1242EA0C2282EACC0212B2504080EAAA
:108E48000010C0B2C2F3072282EA101242EA0022DE
:108E580082EAC00212B2514081EA0111C9B2C2F3DA
:108E6800072282EA111242EA012282EAC10213B2FF
:108E780089EA030282EA0212D2B2C3F3072383EA21
:108E8800121343EA022383EAC2031BB283F03202BD
:108E980082EA0212D2B2C3F3072383EA121343EA27
:108EA800022383EAC2031BB29AB24FF0FE0CDFF82A
:108EB800208184F850E00920C8210EF1010EDBB2B0
:108EC80084F84EC04FEA122C84F84F0084F85210F0
:108ED80084F8D6E2A4F84C2084F85EC084F85D30AB
:108EE800D8F80000D8F80410D8F80820B8F80CA072
:108EF80008F2B22EAEE8070008F2C2288EF80290F7
:108F0800AEF800A084F810C384F80F3315F8011FD9
:108F1800386807F03DFAA845F8D1009BC4F8C0327C
:108F2800FFF703B9DFF8ACA0DFF8AC8041200FF001
:108F380071FCBAF9023088FB0320DB17C3EBA000F1
:108F480080B20FF04DFCBAF9003088FB0320DB1724
:108F5800C3EBA00080B20FF043FCBAF9043088FBE1
:108F68000320DB17C3EBA00080B20FF039FC144BD1
:108F78003868197807F00CFA94F8BC3213F0010835
:108F880000F0FD830F4AC4F8B8920133DBB2A2FBAC
:108F98000312D20802EB8202A3EB420384F8BC322C
:108FA800FFF7A5B8084B0949186807F0C5F9002369
:108FB8002370FFF70FB900BFA8B50208F81C0020FE
:108FC8009C720020CDCCCCCCDC5C00201C5C00204A
:108FD8006A1E0020B06000206766666694F8143444
:108FE800BA4AC4F8106402EB8302D26B42B30EADE6
:108FF80004F21B43B64E45F8203D002104F22D43F0
:109008003180079380211523A52784F81A34284630
:1090180084F8191484F8187490472846318803F0A6
:1090280065FF069DAB4804F583616D1A152DA8BF31
:1090380015252A4621F0B3FFA74A94F81434157071
:10904800A64A013382FB0312A2EBE37202EB42024F
:109058009B1A84F81434FFF778B8A14BA14AD4F8C6
:1090680068112868128893F80BE09F4B401A4FF458
:109078007A71D7B201FB0EF1120A9F771F758842E9
:109088004FF00007DA775A759F701F7180F02E83B2
:10909800964A974811689268C4F8646180FB01E7B2
:1090A800C91780FB02E0C1EBA701D217C2EBA002EF
:1090B80008124FEA222C4FF0F40E1977012758773F
:1090C80083F8202030207521782283F821C083F886
:1090D8001AE0DF7683F8220083F8231083F824202F
:1090E800FEF782BF834F386803685B69984700289A
:1090F8003FF409A83868036801219B699847022250
:10910800002388F800202370FEF7FDBF94F8801133
:1091180094F8813138684A1C013384F8802184F836
:10912800813107F035F9FEF7C1BF734CDFF8D091F4
:109138004FF0000A0BE01B2B00F043820D2B00F0D0
:109148000C824FF0010389F80130D8F8000007F0CD
:109158001BF9002837D0D8F8000007F011F983B2BE
:109168007E2B2A6828D099F80120002AEDD194F89E
:1091780082110029DFD07D2B00F0038294F886E16C
:10918800BEF1000F04D080F02003DBB284F8862102
:109198004A1CD2B2092A635484F8822100F0E5817E
:1091A800082AD2D8B4F88421134403EB132303F01C
:1091B800FF03A4F88431C8E784F882A184F883A166
:1091C80089F801A0C1E794F887312BB1637884F856
:1091D8008701302B00F03E8594F883213B4BDFF864
:1091E8002491DFF824C1DFF824A14FF0010E002AF2
:1091F8003EF46DAF2968C91B012900F2A98194F8D2
:109208009C82B8F1000F40F0F38194F8B41233F85F
:10921800110010B984F8B4E2E9E70131B0F5826FC2
:1092280084F8B41200F018811ED9B0F5E26F00F08E
:10923800BC8033D9B0F5046F00F0C580B0F5116F6C
:1092480000F0CD80B0F5E46FD1D12C4AD76B118AEC
:10925800642303FB07F393FBF1F10FF00EFB0023EC
:1092680084F88331FEF733BFB0F5007F00F0D1807A
:109278004ED8B0F5807F00F04281B0F5887FB6D136
:10928800D9F800104907B2D500214FF488700FF0C3
:10929800F4FA002384F88331FEF719BFB0F5C06FE4
:1092A80000F0CA80B0F5E06FA1D1144A506B118A62
:1092B800642303FB00F34FF4E06093FBF1F10FF03C
:1092C800DCFA002384F88331FEF701BFA8B5020851
:1092D800B85B0020083300201D3300205655555533
:1092E800343E0020303E0020845C0020BC5B00201F
:1092F80067666666144500201C1E00206C6000200E
:109308000800002050520020E05E0020423E00206D
:10931800B0F5047F00F00281B0F5806F7FF467AF8D
:1093280094F8B5320133DBB2032B00F22F8142F2FD
:10933800107184F8B53201FB03F1BD4B1B88002B7B
:1093480040F02A810131BB4B1B78D807BA4B1B88E8
:1093580048BF0431DA0748BF0A31980748BF1431BB
:109368001A0648BF2831D80548BF28315A0748BFD0
:109378006431180748BFC8319A0548BF01F5C8715C
:10938800980648BF01F57A71DA0648BF01F5FA6117
:10939800580648BF01F57A614FF480600FF06DFA06
:1093A800002384F88331FEF792BEA44A976B118A92
:1093B800642303FB07F393FBF1F10FF05EFA84F8E3
:1093C8008381FEF784BE9E4BB3F9041001EB810143
:1093D80049000FF052FA84F88381FEF778BE9CF8B2
:1093E800041000293FF403AF9AF8001000293FF455
:1093F800FEAE944B1B8803EB83035B004FF41160B4
:1094080093FBF1F10FF039FA002384F88331FEF76A
:109418005EBE9CF8051000293FF4E9AE8A4B8B49E3
:109428001B6881FB0321DB17C3EBA1010FF025FAB1
:1094380084F88381FEF74BBE9CF8051000293FF4A1
:10944800D6AE814B4FF4C06099680FF016FA00232E
:1094580084F88331FEF73BBED9F8001011F02008DC
:109468007FF4C5AEDBF80010090600F1DD8378490A
:10947800097B00293FF4BBAE94F8B612032900F229
:10948800B585DFE801F032281902724B1B6859795B
:109498009A79DB7901F1407101EB022101EB03417B
:1094A800002384F8B6324FF482600FF0E6F9002307
:1094B80084F88331FEF70BBE674B1A68137A50792C
:1094C80092781B0403EB002313444A1C84F8B62249
:1094D80003EB0161E7E7604B1A68D379107952789A
:1094E8001B0403EB00231344EFE75B4B1A689379E3
:1094F800D07812781B0403EB00231344E5E7D9F86E
:10950800001048077FF573AE00214FF480700FF00C
:10951800B4F9002384F88331FEF7D9BD9CF8041010
:1095280000293FF464AE9AF8000000283FF45FAECB
:10953800474B5B7B002B00F0F983424B198891FB6A
:10954800F0F101EB810149004FF404700FF095F937
:10955800002384F88331FEF7BABD4FF0010284F886
:1095680082212370A4F88411EFE5B4F88421C2F1B4
:10957800FF0293427FF4E5AD4FF0010384F8873191
:10958800DFE54FF0010384F88631DEE5012384F836
:10959800B53242F21071D0E60231D4E608F04CFD43
:1095A8002E4B1A6840F6B833801A984200F27E8132
:1095B8002B4F3B793A2B00F0D48200232370FEF71F
:1095C800A2BDD8F8000006F0DFFE00287FF4B9AD90
:1095D8004FF0010384F88331B7E5C4F8743184F897
:1095E8006C31204F15F098FF94F87831FEF743BDA1
:1095F800D4F88C32DFF8709094F8B2224B4500F022
:10960800D183511C94F8B3E2D4F890C284F8B21212
:1096180002F00F028DF818200DF11902ACEB0301CE
:10962800002940F3EE8406A902910DF11E0720E0FF
:109638007A490020855B0020F81C00206C6000201F
:10964800B0600020303E0020BC5B00206766666684
:10965800343E002020750020F05E0020C044002029
:10966800A8440020EC5B0020A81F0020002840F33D
:109678001A810133C4F88C3213F8011C02F8011B5B
:10968800BA42ACEB030081EA0E0EEFD384F8B3E2E2
:1096980000F0A684501CB84282F800E005D20EAB58
:1096A8009A1A1B3A002121F09FFC029932200FF0F0
:1096B800C9F84FF00008002384F89C8284F88331AD
:1096C800FEF705BD013B84F8C632FEF7B4BF013A88
:1096D80084F8C722FFF7E7B8013B84F8CF321CE4CF
:1096E8000EF1FF3E84F8CEE2FFF7C1B9C04A2968FF
:1096F8001278C4F86811013A012A3FF6C9AC102162
:10970800022299701A71C3E4BA4ABB4B12680793D4
:10971800A3F1240800202121D50003F8240C88F89F
:10972800021040F1F782B5490327B54B1B8858054D
:1097380000F1ED82DA0700F1968303F00203B14AE3
:10974800002B1CBF03271146AF4D3A46284621F08F
:1097580026FC7B190EA80133A91E40F8203D0022E3
:109768005B1A7A5588F8013015F05CFFFEF749BDA1
:1097780015F0C4FEA54B01221A70FEF750BCA04B91
:109788001B88DA0515D4D80600F17883990600F10C
:1097980011845A0600F13B84180700F16A84D9073E
:1097A80000F17C8413F0020F0CBF4FF004084FF057
:1097B8000C08974B974A1B78D27803F001030AB13B
:1097C80043F00203532000930FF024F8924A1288C2
:1097D80002EB820202EB8202900080B20FF000F8E6
:1097E80000200EF0FDFF8D4A8D4912883868C2EBC3
:1097F800C212520081FB023111444FEAE27ACAEBED
:10980800612A5FFA8AFA514606F0C2FD854B38682C
:109818001A78009B48EA0308824B8AEA020A002168
:1098280083F800A006F0B4FD4146386806F0B0FDA4
:109838007C4B7C4A1B78386888EA0303DBB21946FC
:10984800137006F0A5FD94F8BC32002B7FF49AAB98
:109858004F200EF0DFFF1AF0D3FF1AF0D1FF1AF0F5
:10986800CFFF0121386806F093FD6F4A6D4B92F8DF
:1098780000801B786B4A386808F00108414683F07D
:109888000103137006F084FD664B38681B7888EA7C
:109898000308644B414683F8008006F079FD94F88C
:1098A800BC32FFF76FBB84F8B3E2F3E65F4AB2F865
:1098B800BE3200210133A2F8BE322170FEF723BC6C
:1098C80086468246014601900390029005908146A3
:1098D800FEF7EABE484B504907930EAFA3F12100AB
:1098E80047F8200D4FF0080E4FF000080A2003F843
:1098F80022EC03F8230C03F8248C3846098803F07B
:10990800CFFA4B4B4B491B6881FB0321DB17C3EB99
:10991800A101384689B203F0C3FA474BB3F8069061
:1099280005F028FC069B5A1C069283F80080069BCB
:109938004FEA1922591C06911A70069B5A1C069266
:1099480083F80090069B5A1C06921870384615F04A
:1099580069FEFEF753BCDFF8E8809FED388AB8F956
:109968000230254A079207EE903AF8EEE77A0EAFF2
:1099780067EE887AA2F12403FDEEE77AA2F12101CD
:10998800002047F8201D02F8240C0822CDED007AAB
:109998005A701E229A70BDF80010384603F080FAFB
:1099A800B8F9003007EE903AF8EEE77A384667EEF5
:1099B800887AFDEEE77ACDED007ABDF8001003F065
:1099C8006FFAB8F9043007EE903AF8EEE77A3846BD
:1099D80067EE887AFDEEE77ACDED007ABDF80010E3
:1099E80003F05EFA384615F01DFEFEF704BC00BF12
:1099F800405D00208C6400201C5C0020E0D9020837
:109A0800F81C0020F0D90208FB5B002008000020A9
:109A1800855B0020085D0020303E00205035002086
:109A2800030820809C720020103600201C1E002095
:109A3800BC5B002067666666E05E002058A08B412C
:109A4800B0600020022015F0DDFDFF200EF0C6FDFD
:109A58000378FF2B00F0B28290F901004FEAE07919
:109A68005FFA89F9C0B215F0A9FD484615F0A6FDC0
:109A7800032015F0C7FDFF200EF0B0FD0378DFF8D6
:109A88009C93FF2B1BBFB0F908A05FFA8AF74FF031
:109A9800000ACAF3072A384615F090FD504615F01B
:109AA8008DFD99F80430002B40F0EB810DF1180979
:109AB8004946D04815F048FD132015F0A3FDBDF91F
:109AC8001870F8B215F07AFDC7F3072015F076FD87
:109AD8001B2015F097FDBDF91A70F8B215F06EFD50
:109AE800C7F3072015F06AFD232015F08BFD4E20E3
:109AF80015F064FD002015F061FD4946BD4815F0DC
:109B080023FD122015F07EFDBDF91870F8B215F08E
:109B180055FDC7F3072015F051FD1A2015F072FD09
:109B2800BDF91A70F8B215F049FDC7F3072015F012
:109B380045FD222015F066FD452015F03FFD00206B
:109B480015F03CFD5E21D8F8000006F021FC94F8E1
:109B58006031FEF71BBCC4F8706183F80080FEF723
:109B68005EBABB78DBB103F1FF3C5FFA8CFC0CF109
:109B7800010CBC44BE4600221EF8013B534083EA58
:109B88000313DBB2120AD90042EA0322F44581EA40
:109B9800131382EA0302EFD1002A7FF40EAD964B2D
:109BA800964ADFF87CE21968954B1288DFF87482D0
:109BB800D1F830C0CEF818201A68B8F8BE829B6871
:109BC800CEF828200022CEF86800CEF84830CEF82B
:109BD8003820CEF85880BCF1000F00F05682DCF82F
:109BE8000430086C83423BBFCA681B1A1B1A9B18B7
:109BF800002B7EF481AA0B68DFF82C829B6908464B
:109C0800022198470423F87888F8003011F0CCF83E
:109C180003232370FEF772BA0221386806F0ACFB02
:109C280094F87831FEF727BA10230422184606A9BB
:109C38008DF81A808DF81B808DF81C808DF81D809A
:109C48008DF818308DF819200EF0FCFD84F883810A
:109C5800FEF73DBAA3785A09012A40F0998103F02A
:109C68000F0C13F0100300F0AB81DFF8C081E3782C
:109C780094F804E0A4F8AA0208EB03018EEA0300B2
:109C880084F888214346C4F8A082C4F8A412A8F135
:109C9800070284F8B002A4F8A8E294F8B002DFF84A
:109CA800908186460CE012F8011BC4F8A0024245D8
:109CB80081EA0E0E197007D2D4F8A412D4F8A03293
:109CC800994203F10100EED1424584F8B0E200F078
:109CD800EC81127894F8B0329A4200F09C81494B9A
:109CE800C4F88C3200220133B4F8A812C4F89032B8
:109CF80084F8882101234FF6F672A4F8941284F8A8
:109D08008C3184F89C32A4F89622FFF765BA0327B1
:109D18003D4919E5DBF800303C4A3D4903F480032E
:109D2800834216BF114604270327FEE4334B1988E4
:109D380007E4102015F066FC484615F03FFC48463D
:109D480015F03CFC212015F05DFC484615F036FC6A
:109D5800484615F033FCFEF7EEBA2E49C9780029BB
:109D68000CBF04210521FEF7AEBF012238681A7026
:109D780006F006FB8046386806F002FB18F07F0FF5
:109D88007EF44DA98E287EF44AA994F86C31002BF4
:109D98007EF461A9204BC4F874312D2384F87831FE
:109DA800FEF744B9B4F99612D4F890C294F894E244
:109DB800501C02F00F0242F010020029B8BF42F016
:109DC80020028DF81820ACEB090282EA0E0E5FFA29
:109DD8008EFE8DF8192084F8B20284F8B3E20DF1F2
:109DE8001A021BE4064B9246B3F9003064200A4677
:109DF800FEF74CBB8096980014450020303E0020AA
:109E0800BC5B0020A81F0020E4D90208E0D90208A2
:109E1800D8D90208085D0020845C0020E05E00209C
:109E2800A80000201C1E002019010020281E002068
:109E3800241E0020BC495A790B8803EB830303EBEB
:109E480083034FEA830A1FFA8AFA002A40F05F81E7
:109E58004FF0FF331BB2029305F08CF9029B019A75
:109E680040B2FEF713BBB14904276DE4964692460B
:109E78001146019203929146FEF716BC4FF0340842
:109E880097E4DFF8C4A29AF80020002A3FF40EAE47
:109E9800B4F86271A44B00921B883F016421BFB2E1
:109EA80001FB03235100B3FBF1F347EA0327BFB2D9
:109EB800C3F303231F43062015F0A4FBF8B215F0E3
:109EC8007DFB380A15F07AFBB4F86231964A984956
:109ED8001788009A01339BB293FBF2F002FB103310
:109EE800487AA4F86231012800F007814B7B6E2282
:109EF80002FB07F7152297FBF2F7002B40F0F780DB
:109F08003A2015F07FFBBFB24FF0640AB7FBFAF2B4
:109F180093B2D8B20192009315F050FB009B180A37
:109F280015F04CFB3B2015F06DFB019A0AFB1270F3
:109F380080B20A23053090FBF3F0C0B215F03EFB67
:109F4800002015F03BFBDFF8FCA1282015F05AFB98
:109F58000A23DAF8007097FBF3F7F8B215F02EFB36
:109F6800C7F3072015F02AFB042015F04BFBB9F8BE
:109F78000630002B40F08180DAF8087087F310076C
:109F8800F8B215F01BFBC7F3072015F017FB8DE59A
:109F9800684B694AC4F88C32591C012384F888013B
:109FA80084F88C01C4F89012C4F8942284F89C3286
:109FB800FFF712B94FF02408FFF7FBBB484652E5FC
:109FC80094F88821002A3FF407A994F8B1220132B5
:109FD80002F00F02624546D084F88831FFF7FCB8DA
:109FE800029932200EF02EFCFFF765BB4B1CDBB24A
:109FF800042B84F8B6324FEA01617FF454AAFFF7C4
:10A008004FBA06AB02930DF11E07FFF743BB4FF0A3
:10A018001008FFF7CEBB494BD4F8A022C4F8A422FD
:10A028004FF0000E03F52072114603F5C079C4F80D
:10A03800902203F525707246C4F8A032C4F894E261
:10A04800C4F88C9284F888E1F6F79AF8013030D099
:10A05800D4F88C32C4F890320123C4F88C9284F876
:10A068009C32FFF7B9B8D4F8A412D4F8A032344A15
:10A0780013E64FF02008FFF79CBB05F07BF815F0BE
:10A088009DFA002015F09AFA10E5C8690B6A984203
:10A098003BBFCA681218C31AD31AA9E54FF00808BB
:10A0A800FFF787BB9146FEF7FFBA84F8B1C2FFF706
:10A0B80093B8D4F88C320222591CC4F88C121A7046
:10A0C800C6E796469146FEF7EFBA964692469146FF
:10A0D800FEF7EABA9646924611469146FEF7E4BA6A
:10A0E80096469246114601929146FEF7DDBABFB2F6
:10A0F8009AF8003097FBF3F702E7392015F082FA57
:10A10800F8B215F05BFA380A15F058FA1BE70D4B50
:10A118001B689FE696469246114601920392029268
:10A128009146FEF7C1BA00BF303E0020E8D90208C8
:10A13800343E0020A81F00200000F6FF281E002043
:10A148001F1E0020BC5B0020423E00202DE9F04F7E
:10A158002DED028B9B4A9C49137897B004460B90CF
:10A1680000F59C4020300E900860002B00F07E85A2
:10A17800964909688C4240F297809549059109688B
:10A188009448954D954C0491013B137001F480530C
:10A1980003900A93002B40F09580039B5B7D002B76
:10A1A80040F00285049B180400F1EF87049BD90551
:10A1B8000BD50B9A8A4BDFF858B29A429BF80220CB
:10A1C80001F2B381002A41F0B481864B0693864E92
:10A1D800049B13F4805840F00885039BB4F906707B
:10A1E8005B8B9F42B4BF00270127804B1B6813F08D
:10A1F800805374D0069A127812F0010276D003992F
:10A20800DFF81092898C99ED037A07EE901AF8EE30
:10A21800E77AB4EEE77AF1EE10FA81F27C80002F4B
:10A228006BD195F8A410002967D17148714900686D
:10A2380090F830004FF0000EC1F800E0C1F804E0DB
:10A24800C1F808E06C49002858D10870002A59D094
:10A25800049AD00656D5694A1278D10652D4B8F174
:10A26800000F4FD1002B4DD1049B5A024AD496F8C7
:10A2780000E0BEF1000F01F03C87614B9B78002F96
:10A2880041F0BD873BB15F4A5F4B12681B689B1A60
:10A29800002BC1F2CF87102004F006FB012385F8BC
:10A2A800A53096F800E02FE0494B05931B6804930E
:10A2B800484A494D039203F48053484C0A93002BB3
:10A2C8003FF46BAF0021494803F044F800287FF4BD
:10A2D80064AF1CF067FB059B1B6804935DE7049A59
:10A2E800520287D4069A127802F00102002185F8FA
:10A2F800A410DFF82091002F97D03F490120087063
:10A30800002AA5D196F800E0039AB4F90080518B91
:10A31800928BB4F9020095F8A6B08845CCBF4FF0EF
:10A32800800C4FF0000C4CF040039045A8BF6346EA
:10A338009B0843F0800C8842C8BF634643F0400C3A
:10A348009042B8BF63469B08B4F904C0B4F906004C
:10A3580043F080088C45C8BF434643F04008944505
:10A36800B8BF43469B0843F0800C8842C8BF634689
:10A3780043F0400C9042B8BF63469B4500F01086FE
:10A388004FF0000885F8A63085F8A780BEF1000FC9
:10A3980000F06D87059B1B6803F00403002B40F059
:10A3A8007D850DF1500A194E0023CAF8043006F1D4
:10A3B800500B14934FF0190840F6330340F28337DB
:10A3C8002DE000BF3C3600204834002038360020FD
:10A3D80050430020FC4200205022002080710020C1
:10A3E800404B4C00855B0020680000208C640020F6
:10A3F800F05E002038350020C81D002010360020EF
:10A40800D8640020F06200209C740020B43500203D
:10A41800085D0020443E002004365E4524D0B17813
:10A42800F278914218FB0170F6D296F801E00EF12D
:10A43800040E18FB027134F91E209A42A8BF1A466E
:10A44800B2F5617FB8BF4FF461729042E4DA91428D
:10A45800E2DB31782329DFD850460436049302F032
:10A4680069FF5E45049BDAD15C4B9AE803001F78CC
:10A478005B4B83E80300002F00F09B84594B079344
:10A488005748012102F066FF002840F05E82059BD4
:10A498001B68DE0500F15482534B0493534D2B88FF
:10A4A8001EB226F001061FFA86FA5345A5F800A049
:10A4B80000F0EA854E4E4FF002080F2014274FF0A7
:10A4C800FF0B86F80080777086F802B004F0ECF98C
:10A4D80041464348B5F800A002F03CFF002841F08F
:10A4E800B9812AF002039BB253452B800BD0404B15
:10A4F8001421FF2202260F201E7059709A7004F052
:10A50800D3F9B5F800A03B4B3B4A1978506808933B
:10A518001AF0030F08BF81F00201C1F3400109924C
:10A5280006F058FD049B1B6813F00A0F1AD0062189
:10A538002B4802F00FFF002800F085862B8858066C
:10A5480041F1F4800721264802F004FF50B12B4B5B
:10A558002B4AB3F904302B4982FB0302DB17C3EB08
:10A56800A2030B800C211E4802F0F4FE2A88002862
:10A5780000F04F8242F480739A422B8009D01C4B22
:10A5880002261421FF220F201E7059709A7004F0C1
:10A598008BF91D4B1B78082B00F047820E2B00F01F
:10A5A8004482059B1B68590561D5184B1B79002B04
:10A5B80000F0188114210A4802F0CCFE002840F06F
:10A5C800168115F071F8012004F0BEF800284ED06D
:10A5D800DFF83CA000264FF0CC0B1EE0CD5B00203E
:10A5E8008C6400202075002050520020F81C0020A8
:10A5F800945E0020BA620020BC620020B060002097
:10A608006766666698740020B0350020343E0020E6
:10A61800FC650020DEB2022E29D80BFB06F8731C5D
:10A628005AF80870002FF5D1C378D84A90F902007B
:10A6380052F8233001970322009201213A4603F091
:10A6480059FC034606EB460000EB0010049353B197
:10A6580039460AEB8000CC2220F0C6FC049B4AF85D
:10A6680008300136F6B21BF027F90028D3D1069B33
:10A678001E7816F0010600F01182C54B01221A70EF
:10A68800079BB4F906101B68C2485A8901279142F2
:10A69800077080F2E981C04B4FF07E521A60BF4AC2
:10A6A800039BB4F900C01F8B92F9043092F801E0C3
:10A6B8001078002BACEB070314BF01224FF0FF32D8
:10A6C800002B40F3C581B3F5FA7FC0F2C7814FF480
:10A6D800FA731B1A07EE903AF8EEE77A6745C9ED68
:10A6E800007A03DDF1EE677AC9ED007AB4F902C0A9
:10A6F800ACEB0703002B40F38081B3F5FA7FC0F27F
:10A7080082814FF4FA731B1A07EE903AF8EEE77A53
:10A718006745C9ED017A03DDF1EE677AC9ED017A83
:10A72800B4F90400C31B002BD8BF3B1AB3F5FA7F5A
:10A7380080F25E817345D8BF4FF0000E00F35A8156
:10A7480002FB0EF207EE902A059BF8EEE77AB84274
:10A758001A68C9ED027ABCBFF1EE677AC9ED027AD0
:10A7680012F4805200F00B82B1F5FA6FA8BF4FF4D3
:10A77800FA61B1F57A7FB8BF4FF47A71A1F57A71B1
:10A78800874C884884FB013ECB17C3EB6E1303F15B
:10A79800010E6FF0630C30F91EE030F913000CFB6A
:10A7A8000313AEEB000103FB01F384FB0314DB1777
:10A7B800C3EB641303441BB207EE903AB8EEE78A82
:10A7C80089ED038A002A40F08C832B885B0624D409
:10A7D800002E40F0A8801DF0F3FA17B0BDEC028BF4
:10A7E800BDE8F08F069B1B78DA077FF5EAAE3C20C0
:10A7F80019F0ACFF00283FF43AAF04F0A9FF3C2061
:10A8080019F046FF00283FF432AF04F0A1FF3C20C6
:10A8180019F03EFF0028F0D129E7634B634AB3F9EA
:10A8280004306349DFED636A09889FED637A82FB30
:10A838000302DB17C3EBA2035B1A1BB207EE903AC5
:10A84800F8EEE77A67EEA67A77EE876ABDEEE66AF3
:10A8580016EE103A2033402B40F27387BDEEE77AAC
:10A86800DFED626A17EE103A2033402B00F2B6870C
:10A878009FED527AF4EEC77AF1EE10FA41F32D8388
:10A88800DFED4F5A9FED4F6A01E0F0EE477AF4EEA4
:10A89800C67AF1EE10FA37EEE57AF6DCDFED4A7AA1
:10A8A800B4EEE77AF1EE10FA41F11383DFED445A82
:10A8B8009FED466A01E0B0EE677AB4EEC67AF1EE33
:10A8C80010FA77EE257AF6D49FED3B7AF4EEC77A44
:10A8D800F1EE10FA40F336859FED387A77EE677A15
:10A8E80067EEA75A9FED3A5A9FED3A6A9FED3A7A7A
:10A8F800A5EE856A27EEA55AA5EE867AE5EE077AD3
:10A9080099ED016AD9ED005A27EEC67A65EEA77A65
:10A91800A5EEA67AE6EE267A89ED007AC9ED017AE7
:10A92800002E3FF458AF089B1978099B01F00101EC
:10A93800186806F04FFB17B0BDEC028BBDE8F08F2E
:10A94800264BDB78002B3FF4A7AD254B04931B68FF
:10A958009D077FF5A3AD234DB5F800A01AF0010FB0
:10A968007FF4BFAD4AF001039A452B803FF4B9AD9F
:10A978001D4B022214211A700F20FF2259709A7061
:10A9880003F092FFB5F800A0ABE500BF54CD020874
:10A99800865B0020001D0020A41D0020AC64002060
:10A9A8001F85EB5124750020B0600020676666663D
:10A9B8009874002035FA8E3CDB0FC93FDB0F494005
:10A9C800DB0FC940E4CB1641DB0F49C0E4CB16C10D
:10A9D80092E741B99730083C15A82ABE085D0020C7
:10A9E80050520020F81C0020945E00200000000057
:10A9F8004FF4FA73A3EB0E0EA2E6A7EB0C03B3F524
:10AA0800FA7FBFF67EAE9842FFF67DAE5FED097A1B
:10AA18007EE622F480739BB29A422B807FF4AFAD1E
:10AA28007E4B1B78082B7FF4B9AD2A8822F04003AF
:10AA38009BB29A422B803FF4B4AD794B0226142185
:10AA4800FF220F201E7059709A7003F02DFFA8E5A1
:10AA5800A7EB0C03B3F5FA7FBFF639AE9842FFF6C1
:10AA680038AEDFED707A39E6B1F5FA6F80F22E83F1
:10AA7800187A8B1A03FB00F3C2F5FA6293FBF2F320
:10AA8800C3F1640307EE903AF8EEE77A9FED667A31
:10AA9800664B67EE877AC3ED007A00E6644B1B7855
:10AAA8000493002B7FF4ECADDFF8B8B1DFF8B8A160
:10AAB8001BF8030C9AF800805946ABF1030709F01C
:10AAC80091FC002800F00883049BB8F1000F53D1D3
:10AAD80007F10801787909F085FC002841F05A82CD
:10AAE8005449B87A09F07EFC002800F00983B8F1CF
:10AAF800020F41F052825049F87B09F073FC00289C
:10AB080041F04E824D49387D09F06CFC002800F078
:10AB18000983B8F1040F41F046824949787E09F06B
:10AB280061FC002841F042824649B87F09F05AFC8E
:10AB3800002800F00983B8F1060F41F02882424945
:10AB480097F8230009F04EFC002840F08A873F4917
:10AB580097F8280009F046FC002800F00983B8F1AE
:10AB6800080F40F06D873A4997F82D0009F03AFC34
:10AB780000283FF485AD09231A4600F063BF039B04
:10AB8800588B8142C0F2A082B1F5FA6FD4BFC0EBF6
:10AB98000101C0F5FA614FF47A7303FB01F1C0F5C6
:10ABA800FA60B1FBF0F1EBE5039A013BD27D34F991
:10ABB8001330002A40F07483A3F57A73B3F57A7FD3
:10ABC800A8BF4FF47A7323EAE37307EE903A9FED38
:10ABD800217AF8EEE77A67EE877A1F4AFCEEE77A81
:10ABE80017EE903A1380FFF7E1BA1D211B4802F0D7
:10ABF800B1FB00287FF4F1AA194A039BD2881B8B6A
:10AC0800B4F90670991A8F4240F3CA8613449F42DA
:10AC1800B4BF00270127FFF7E8BA00BFB03500200E
:10AC2800945E0020000000000AD7233CA41D0020E9
:10AC3800865B0020635E0020685E00206D5E002059
:10AC4800725E0020775E00207C5E0020815E00201E
:10AC5800865E0020AAF1823F503500208C640020D7
:10AC6800E03C0020595E00200A000020B34DB44BA0
:10AC78002E780393DFF8CC82002E00F02783B6B13C
:10AC8800DFF80893DFF808B3AE4FCA460024072C54
:10AC98003846E1B2D8F8043041F30782984700B249
:10ACA8000134A6422BF8020F0AF1040AEFD1A64B91
:10ACB80005931A460B99A54B12680492A3FB013E13
:10ACC80042F2010313404FEA9E1E099300F0ED8201
:10ACD8009F48A04AA04B0078A049079012781A70A4
:10ACE800079B087023B19C4B1B7883F001030793E3
:10ACF8009B4A039912780D920D9A0C8D994BB1F8D5
:10AD0800269091F822C010940C8B13941146A3FB43
:10AD180001135B0803EB4303D31ADBB295F8294010
:10AD28000F93049B98F800002E7808900F22204675
:10AD38000CF1040C03F480538B4F8C4CDFF854A2B5
:10AD4800CDF818905FFA8CFCB34685F8282011924C
:10AD58000A93002181460C95CDF8488036B9089BA6
:10AD68009C458DBF9B46E34666465E46B14280F2EF
:10AD78006983079B002B00F013837D4B069833F9FA
:10AD880011201FFA82F840454FEA410303D8109872
:10AD9800804540F252835AF82120964580F00A8374
:10ADA800E25E0998002840F02183E252013106371B
:10ADB800D4E7DFF8E4B1DFF8E4810BF15A064FF08D
:10ADC800010A59461BF8010C09F00CFBF8B19BF875
:10ADD80004009BF802309BF803E000EB400105EB10
:10ADE8008101013BD1F8B42003EB43034344934270
:10ADF8000DD095F8E02081F8B0E00AFA00F022EAD8
:10AE08000000C1F8B430C1F8B87085F8E0000BF163
:10AE1800060B5E45D5D1574B574A079319464F4BFA
:10AE2800D2F800B009681B78544E0891DA460493AA
:10AE38000027AB46736853B31D7845B3B168AAEBD6
:10AE4800010100290ADB9BF8E0100120B84021EA43
:10AE580000010AF5FA708BF8E010B060049AB2B1FC
:10AE6800317858780431C9B2002840F05982039AE1
:10AE780034F91110108B00F1C80E714540F3648548
:10AE88009BF8E0109B783941C90740F1C485013728
:10AE9800042F06F10C06CDD1FFF7F2BA95F8AB30C6
:10AEA80053B1069B1B78D80706D5039BB4F9062037
:10AEB8005B8B9A4200F3A1851121314802F04AFACE
:10AEC800002800F00F8295F8AE302BB995F8A9301C
:10AED80013B93223A5F8AC30012385F8AE30FFF75B
:10AEE80060BA1D21264802F035FA00283FF46DACFF
:10AEF800244BDB78002B7FF468ACDFED237A134911
:10AF080038EE678AC7F5FA63FDEEC87A1BB2CDED55
:10AF1800037ABDF90C20120381FB0201D217C2EBA0
:10AF2800A11203FB02F343F30F333B4407EE903ABD
:10AF3800F8EEE77AC9ED037A47E400BF5022002013
:10AF4800FC420020B860002050430020D34D62101E
:10AF5800243400206C0000206D0000202C5D0020AF
:10AF6800C4440020ABAAAAAA7C2200208071002039
:10AF78005422002020750020F062002000230020C9
:10AF88008C640020085D002000007A441C490020E1
:10AF980052220020C8440020715D0020F4B5020848
:10AFA80095F8A780B8F1F90F00F2AE8108F1010811
:10AFB8005FFA88F885F8A78085F8A630BEF1000FFB
:10AFC80000F05681B8F1140F7FF4E4A95F2B40F02C
:10AFD8006281069F3B7813F0010300F086871BF01F
:10AFE800E1FC3B7803F00103002B7FF4D3A995F82B
:10AFF800A620572A00F00087059B1B6813F004035E
:10B0080002D05A2A00F030855D2A00F055875B2A65
:10B0180000F067875E2A00F00485562A00F0DB8777
:10B0280033782BB16F2A00F0C487CD4B002119600B
:10B03800972A00F0C687A72A00F0D4840021BB2AEB
:10B04800149101F00D80B72A00F0EC87BE2A01F0B8
:10B058000A80BD2A01F00980792A01F01F807A2A26
:10B0680001F015809E2A01F00B809D2A01F00080D6
:10B07800AE2A01F07B80AD2A7FF48CA9FF21002045
:10B0880013F06FFDFFF786B90221B64802F062F9A6
:10B0980000283FF426AA2E801AF0020F7FF433AA64
:10B0A8004AF0020353452B803FF42DAAAE4B0222EF
:10B0B80014211A700F20FF2259709A7003F0F4FBC4
:10B0C800B5F800A0FFF71FBA114668E51B7AC3F16F
:10B0D800640307EE903AD7E40BF10501787909F09B
:10B0E80081F900283FF4FCACB8F1010F40F0528719
:10B0F80007F10D01B87A09F075F9002840F04D877D
:10B108009A49F87B09F06EF900283FF4FBACB8F1D6
:10B11800030F40F045879649387D09F063F9002808
:10B1280040F041879349787E09F05CF900283FF4A4
:10B13800FBACB8F1050F40F039878F49B87F09F0AB
:10B1480051F9002840F023878C4997F8230009F02B
:10B1580049F900283FF4FBACB8F1070F40F08184AF
:10B16800874997F8280009F03DF9002840F06884DD
:10B17800844997F82D0009F035F900283FF480AA92
:10B18800B8F1090F3FF47CAAF5E4D5F88C300B9A96
:10B19800D31A002BFFF60AA87B4A95F89030517C09
:10B1A8007A4A039E32F811200E98B17DC5F88C00BA
:10B1B800013303F00F0385F890302B4492B292FBD1
:10B1C800F1F283F8942095F8940095F8951095F885
:10B1D800962095F8973001440A4495F8980095F818
:10B1E80099101344184495F89A2095F89B30014417
:10B1F8000A4495F89C0095F89D101344184495F856
:10B208009E2095F89F3001440A4495F8A00095F8CF
:10B21800A1101344184495F8A23095F8A3200144CE
:10B228000B441A4442F30B12642AF17DA8BF64222E
:10B2380013B209B1C2F1640307EE903A9FED547A54
:10B24800F8EEE77AC7E42A8822F040039BB29A42D4
:10B258002B803FF477A9444B02261421FF220F20AC
:10B268001E7059709A7003F01FFBFFF76BB9F04618
:10B2780000213C4802F06EF8D8B1002385F8A830C8
:10B288001BF01AFA95F8A730142B7FF483A83378AB
:10B29800002B40F0CB87069B1B7803F00103A3E645
:10B2A800C3F53B6308331BB286E43A4B1B7807931C
:10B2B80018E5069B2A4A1B781060DB0700F17685A3
:10B2C800B8F1140F3FF493AEFFF764B893F8223047
:10B2D80098F800600433DBB2B3428EBF2E702B7037
:10B2E8001E46CCE495F8A930002B3FF45AA8069BDB
:10B2F8001B7813F001037FF454A8012285F8A930C4
:10B3080085F8AA20FFF74DB885F8A6B0BEF1000F62
:10B31800AED0FFF73FB8012185F8A410FEF7EDBFC6
:10B32800012800F07D859BF8E0100123BB40013720
:10B338000B43042F8BF8E03006F10C067FF47AAD4E
:10B34800FFF79EB89FED147AF4EEC77AF1EE10FA83
:10B3580044BF9FED127A77EE677AFFF7C1BA00BF54
:10B36800A07400208C640020945E0020685E002099
:10B378006D5E0020725E0020775E00207C5E0020FB
:10B38800815E0020865E00206862002084620020C2
:10B3980014AE23412C5D0020DB0FC9BFDB0F49C071
:10B3A800069B002B47D05AF8212096454FEA4103C7
:10B3B800FFF4F6ACBE4ABE48D25C00EB0308002A94
:10B3C80000F01082022A40F0A58198F8012002EBD3
:10B3D800820202EB820202F2EE2292B2032940F3C9
:10B3E8009B80099812B200283FF4DFAC0F9803EB5A
:10B3F800010880440C9800EB4808A8F82C20B9F103
:10B40800000F03D10D9802287FF6CFACB7F8009053
:10B418007A88B7F804804A449044A64A0FFA88F814
:10B4280082FB0802A448A2EBE87220F8038012B25B
:10B438004FF00109B9E41A464B000EF596784AF820
:10B448002180AEE411990C9D9C4BDDF8488085F86D
:10B4580000B00F294A460CBF0122002285F8299026
:10B4680085F828101A7006D11B21954801F072FF43
:10B47800002800F013859348934B82681968934B12
:10B48800C1608A1A012119704368914F9A42039A40
:10B49800397088BF002392F8227088BF80F8213065
:10B4A8000A9B98F80000B2F818C0B2F82680043752
:10B4B800FFB2002B00F0A38187427D4A40F2208230
:10B4C800844F964600210EB983460646B1421ADAE1
:10B4D80012F8113093B1022B0ED19EF8013003EB14
:10B4E800830303EB830303F2EE239BB227F8023BAB
:10B4F80001310EF1020EE6E73B88F7E7CBB2032BEA
:10B50800FAD86346F2E785F800B00D9B724A01331A
:10B5180013700A9BFEF73EBE012000FA01F811984D
:10B5280020EA080012B211903BE412B901228BF80C
:10B5380002206A4B06931E789BF8219006F00103BF
:10B548001B20049308F078FFB9F1010F089000F070
:10B558002A8206F0020307939BF82020604EDFF84A
:10B5680088A1604FDFF86081052A00F29880DFE843
:10B5780002F0887C032E3E52B9F1010F04BF052367
:10B588008BF82030049B002B00F0D880039BD8F860
:10B598000000B3F91810BAF80230002261F30F0264
:10B5A80063F31F42002361F30F0361F31F43DBF8CA
:10B5B800141062608842236040F27381032307936A
:10B5C80047F230520323CBF81C208BF820303B88FD
:10B5D80043F002033B801BF0E5F9D8F80020DBF8C4
:10B5E8001C3013440422CBF818308BF82020B9F112
:10B5F800010F40F06584D8F80030DBF818209A4233
:10B608004DD2307818B908F017FF002847D13B8889
:10B6180023F002033B80D8F80020BAF806306421F2
:10B6280001FB03234FF4806000228BF820208BF865
:10B638000320CBF8103003F031FA9BF8202093E771
:10B648001CF090F9012800F09784089B002B40F02B
:10B65800AD81B9F1010F22D0D8F80030DBF8102005
:10B668009A4259D301238BF82030B9F1010FD2D077
:10B678009AF80830012B4FD00BF0A8FF9BF8202038
:10B6880072E7049B002BDBD1089B4FF48060002BF2
:10B6980000F0F28003F01AFA0022CBF81020079B82
:10B6A800002B40F0FA80059B1B680493FEF791BDC0
:10B6B8005049002056555555C42200202D5D0020C4
:10B6C8008C640020085D0020F06200206C000020DF
:10B6D8006D00002080710020C4440020855B00209C
:10B6E800680000207A490020F43C0020E4CB164191
:10B6F800DB0F49C0DB0FC940E4CB16C1DB0FC93FE4
:10B70800DB0F494092E741B99730083C15A82ABE9B
:10B7180000000000E25A61E60BF058FF032240F6F1
:10B72800B8338BF82020CBF81C3050E743F04002A8
:10B7380093422A807FF48FADFEF704BFD8F800301B
:10B748003EE7F4EEC77AF1EE10FA40F30E845FEDAF
:10B75800175A1FED1A6A01E0F0EE476AF4EEC66A5E
:10B76800F1EE10FA36EEE57AF6DC5FED1F6AB4EE1C
:10B77800E67AF1EE10FA40F1FC835FED225A1FEDF4
:10B78800226A01E0B0EE667AB4EEC67AF1EE10FAFB
:10B7980077EE256AF6D41FED277AF4EEC76AF1EE44
:10B7A80010FA6CDD1FED2A7A77EE666A66EEA65A05
:10B7B8001FED2C5A1FED2C6A1FED2C7AA5EE856A19
:10B7C80026EEA55AA5EE867AE5EE076ABDEEE77A7B
:10B7D80017EE103A2033402B7FF64AA85FED347AF3
:10B7E800FFF78EB8CAB2022A40F2DD82032A91D14D
:10B7F800139A0A98069D002808BF2A46EEE5874254
:10B808001946B54A55D8B54896460EB9BB463E4680
:10B818008E427FF778AE12F8113093B1022B0ED119
:10B828009EF8013003EB830303EB830303F2EE235B
:10B838009BB220F8023B01310EF1020EE5E70388C6
:10B84800F7E7CBB2022B03D9032BF8D14346F0E735
:10B858006346EEE72AF0010292B252452A803FF48D
:10B868001BAC0F2086F80080777086F802B003F0D2
:10B878001BF8B5F800A00FE403F010F90CE79FEDF2
:10B88800987AF4EEC76AF1EE10FA44BF9FED957A04
:10B8980077EE666A8AE703230793079803F004F8AC
:10B8A80001E7B9F1010FF6D103239BF82020079394
:10B8B8005AE68A4F96460EB983460646B142BFF607
:10B8C80022AE12F8113093B1022B0ED19EF801303E
:10B8D80003EB830303EB830303F2EE239BB227F806
:10B8E800023B01310EF1020EE5E73B88F7E7CBB2E8
:10B8F800022B03D9032BF8D14346F0E76346EEE762
:10B908007648964600210EB9BB463E46B142BFF680
:10B91800FAAD12F8113093B1022B0ED19EF8013016
:10B9280003EB830303EB830303F2EE239BB220F8BC
:10B93800023B01310EF1020EE5E70388F7E7CBB2CF
:10B94800032BFAD86346F2E7C83881423DDA9BF800
:10B95800E0109B783941CA073FF599AAC3F100085E
:10B96800012003F083F8691E162900F21681DFE82A
:10B9780011F02A01170104014D013D017001CD00AC
:10B98800B0019B01C301F00014014D015D0170017C
:10B99800CD00B00195019801A1000402ED01D80184
:10B9A8000127FEF722BC00230793D5E59AF8043057
:10B9B800002B3FF44EAE0BF009FE03224FF47A73CE
:10B9C8008BF82020CBF81C3001E69BF8E0300121F1
:10B9D800B94023EA01030AF5FA718BF8E030B16047
:10B9E800FFF755BA4049059B0A781B6842F00402E4
:10B9F8000A7003F00403FEF7D1BC00213B4801F0B4
:10BA0800A9FC00287FF458AA322385F8AB00A5F8D2
:10BA1800AC30FFF751BA9846002B0CBF012002202A
:10BA28009FE7334B022203203249334E0B603270BA
:10BA380003F01CF8059B1B6803F00403FEF7AEBC7B
:10BA480008231A4602EB820217448AF80030B978B4
:10BA5800787815F0B1FE069B1E7806F00106FEF711
:10BA68000FBE07231A46EDE795F8A920002A40F0F3
:10BA7800918395F8AB1081F0010185F8AB1000298E
:10BA880040F048831D4A126812F4003204D01C4A60
:10BA98001279002A40F0DC8311461046194A565C98
:10BAA8000D2E01F10C0100F07D8301301528F6D12F
:10BAB800FEF774BCDBF8E4008178134B4144C829D5
:10BAC800A8BFC82121EAE17181709B78002B40F062
:10BAD800C8830FF0F1FC26E4504900208071002053
:10BAE800DB0FC9BFDB0F49C0103600208C64002073
:10BAF800925F0020F05E002028600020685D002032
:10BB0800E05E00205CD002085D600020DBF8E40005
:10BB1800B54B01799B784144C829A8BFC82121EABF
:10BB2800E1710171002B40F05E83102DD1D0417876
:10BB3800AD4B4144C829A8BFC82121EAE171417031
:10BB48009B78002BC5D013201BF03EFFDBF8E400E8
:10BB5800BFE7DBF8E400A44B017A9D784144C8298B
:10BB6800A8BFC82121EAE1710172002DB1D00B20D4
:10BB78001BF02AFFDBF8E400ABE7089A1579454487
:10BB8800642DA8BF642525EAE57515711BF036FFFD
:10BB9800954B9B78002B40F05483DBF8E40098E742
:10BBA800089A914B917841446429A8BF642121EAFD
:10BBB800E17191709B78002BEFD002201BF004FFFD
:10BBC800DBF8E40085E7089A874B11784144FA29A5
:10BBD800A8BFFA2121EAE17111709B78002BDCD013
:10BBE80001201BF0F1FEDBF8E40072E7089A7E4BB7
:10BBF800D1799878414481F30801D1710028CCD0DB
:10BC080005201BF0E1FEDBF8E40062E7089A764BBA
:10BC18009179987841446429A8BF642121EAE171A7
:10BC28009171002840F019830D2DB6D0089A6E4BFB
:10BC38005179987841446429A8BF642121EAE171C7
:10BC480051710028A9D00E201BF0BEFEDBF8E400DD
:10BC58003FE7DBF8E400644BC1789B784144C8298E
:10BC6800A8BFC82121EAE171C170002B40F0B5825C
:10BC78000F2D3FF42EAF01785B4B4144C829A8BF74
:10BC8800C82121EAE17101709B78002B3FF421AFB4
:10BC980012201BF099FEDBF8E4001AE7DBF8E40059
:10BCA800E9E7DBF8E40042E7DBF8E4004E4B817992
:10BCB8009D784144C829A8BFC82121EAE171817152
:10BCC800002D3FF406AF09201BF07EFEDBF8E400F0
:10BCD800FFE6DBF8E400444B41799B784144C829EE
:10BCE800A8BFC82121EAE1714171002B40F081828F
:10BCF800112D7FF4E1AEECE6DBF8E4003A4BC179B4
:10BD08009D784144C829A8BFC82121EAE171C171C1
:10BD1800002D3FF4DEAE0A201BF056FEDBF8E400EF
:10BD2800D7E6DBF8E400304B90F83A109D784144B0
:10BD38006429A8BF642121EAE17180F83A10002D36
:10BD48003FF4C7AE17201BF03FFE26E7DBF8E40000
:10BD5800254B90F83B109D784144FE29A8BFFE2151
:10BD680021EAE17180F83B10002D3FF4B2AE1620B5
:10BD78001BF02AFEDBF8E400ABE6089A1A4B517870
:10BD88004144B1F5967FA8BF4FF4967121EAE1715D
:10BD980051709B78002B3FF400AF15201BF014FE68
:10BDA800DBF8E40095E6139AFFF718BB0F4B1B78F6
:10BDB800002B3EF4EFAA0E4BDB78002B7EF4EAAAA8
:10BDC80095F8A8300133DBB2032B85F8A8307EF64E
:10BDD800E1AA084B5B7813B9002F7EF4DBAA1AF0AE
:10BDE800E1FDFFF74FBA00BF5D6000202C5D002029
:10BDF800085D0020D8640020CB4BCC491A684FF46A
:10BE08007A73B3FBF2F3C3EB431203EB8202059B95
:10BE18001B68D200A1F8A82003F00403FEF7BEBAFD
:10BE280034F911109878B1F5617F4FF4966393FB5C
:10BE3800F0F3C0F2928040F633008142A8BF014679
:10BE48000C2DA1F5617191FBF3F100F0D380182D51
:10BE58007FF469AAC9B2C8290B46A8BFC823DBF872
:10BE6800E400C57D5FFA83FEAE453FF45CAA5B1B28
:10BE7800AF4A80F817E048BF0733DB1092785D1CA3
:10BE8800EDB23AB9002D3FF44EAA284602F0EEFD75
:10BE9800FFF749BA18201BF097FDF3E7A549A64B11
:10BEA800CA681B688B609B1AC82B7FF62EAB0123D0
:10BEB80081F82130FFF729BBA04B00220120B3E510
:10BEC800D8F80010DBF81C200A44CBF81820FFF73C
:10BED800E6BBF0EE477AFEF7F7BCB0EE677AFEF7FE
:10BEE800DDBC974B012202209EE5964A1268970313
:10BEF80004D5954A1279002A40F04081934A1846A1
:10BF08001946175C0B2F00F10C0007D001311529D9
:10BF1800F7D1002285F8A720FFF766B88C4FD7F82D
:10BF280000C04800BCF1000F09D000EB010E02EB85
:10BF38008E0E9CF801C09EF801E0E645E9D200EBC0
:10BF4800010E8448844902EB8E024FF0000E3A60DD
:10BF5800A0F800E0C1F800E0DBE70C2D5FD0182D59
:10BF68007FF4E1A900210B4679E7B0EE667AFFF786
:10BF7800FCBBF0EE476A0EE4D8F80020BAF80630A9
:10BF8800642101FB0323CBF81030FFF75EBB0623C7
:10BF98001A4657E501231A4654E502231A4651E585
:10BFA80003231A464EE504231A464BE505231A4691
:10BFB80048E51AF081FB059B1B6803F00403FEF7B4
:10BFC800EDB9059B654A1B684FF4C871118003F0F1
:10BFD8000403FEF7E3B90AF047F800F03DFD0AF064
:10BFE8002BF817F07DFD012002F040FD95F8A62002
:10BFF800FFF716B8CDB25A4B09915B78AB423FF4C4
:10C0080092A928461AF08AFA494B09999B781BB1DC
:10C01800C9B20C201BF0D8FC0135EDB232E700257F
:10C028002946E8E70B464FF6FE714E4A9089568935
:10C0380001443344538191810AF016F800F00CFD55
:10C0480009F0FAFF17F04CFD012002F00FFD059BE7
:10C058001B68002203F0040385F8A720FEF79EB9A9
:10C068000B460221E1E70223DFE74FF6FE73DCE728
:10C078000021FF2012F075FD95F8A620FEF7F8BF05
:10C08800012012F06EFD95F8A620FEF7EEBF364AA5
:10C09800137A43F001031372FEF77CB9324A137A1C
:10C0A80023F001031372FEF775B9039A115D9847DF
:10C0B800032C1BDC40F2EE2240F6CA0C00283EF4AA
:10C0C800EFAD39F824E0BAF802104FF47A73A0EB18
:10C0D8000E0003FB00F0A1EB0E0190FBF1F01844F9
:10C0E8009042B8BF10466045A8BF604600B2FEF750
:10C0F800D7BD002F3EF4CFA895F8A5E0BEF1000FFC
:10C108003EF402A902F0B2FB96F800E085F8A5809B
:10C11800FEF7FAB80C2002F0C7FB059B1B6803F07A
:10C128000403FEF73BB900BF405200201C4A002020
:10C138005D600020085D0020F0620020FE5E0020A7
:10C14800485F0020685D0020E05E00205CD00208A7
:10C158009C1D00200E1E0020101E00203C75002093
:10C1680028600020B4640020EC5C0020012100203D
:10C1780012F0F7FC95F8A620FEF77DBF404A12782A
:10C18800002A7FF4BBAE02F071FB069B1B7803F01C
:10C198000103BEE60021012285F8A91085F8AA202E
:10C1A800FEF7FCB8374FD7F800E04100BEF1000FAA
:10C1B80008D00E1802EB86069EF801E076787645E0
:10C1C800BEF4ECA80144304E304802EB8102002155
:10C1D8003A6031800160FEF7E1B80F201BF0F4FBF4
:10C1E800DBF8E40044E510201BF0EEFBDBF8E4008C
:10C1F8009BE411201BF0E8FBDBF8E40078E53BB199
:10C208002349244A09684FF47A7000FB031313602A
:10C2180095F8A530002B3EF477A802F027FB002301
:10C2280085F8A53096F800E0FEF76EB895F8A630C8
:10C23800FEF7CCBE1AF0B6FB002385F8A530FEF752
:10C2480061B8032029461BF0BFFBDBF8E40040E49B
:10C258000B4A12785AB1084620E40D201BF0B4FBB3
:10C26800E2E414201BF0B0FBDBF8E40031E402F058
:10C27800FDFA059B1B6803F00403FEF78FB800BFA7
:10C28800423E00209C1D00200E1E0020101E002093
:10C29800F06200209C740020002870B51EDB09287D
:10C2A800044620DD012303EB83035B00B0FBF3F2BC
:10C2B800092AF8D87BB10E4EB4FBF3F00928CCBF9D
:10C2C80057223022A6FB03E5024403FB1044EB0887
:10C2D80001F8012BF0D100230B7070BD2D230B70DA
:10C2E80040420131DBE7303001F8010BF3E700BFD2
:10C2F800CDCCCCCC884230B44FF001042ED301FB16
:10C3080004F4B0FBF4F58D42F9D284B1AAB901E086
:10C31800B0FBF4F5092DCCBF572230222A4404FB88
:10C32800150003F8012BB4FBF1F4002CF0D1002226
:10C338001A7030BC7047B0FBF4F5092DCCBF37221A
:10C3480030222A4404FB150003F8012BB4FBF1F456
:10C35800002CF0D100221A7030BC70470546002A24
:10C36800EBD1D7E703685A1C02601970704700BF09
:10C378002DE9F047089C2578002B804689460CBF9C
:10C388004FF0200A4FF0300A661C35B3002A29DD29
:10C39800334601E0024698B113F8011B501E0029EC
:10C3A800F8D1971E60B13D46013D51464046C84709
:10C3B8006B1C002BF8DC257827EAE770013055B1B3
:10C3C800041B29464046C847301916F8015B002D62
:10C3D800F7D1BDE8F087BDE8F087002A04DC2846DD
:10C3E800BDE8F0870020EBE7571EDCE70A449142DE
:10C3F80051D030B441F2210411F8013B80EA032006
:10C40800430010F4004F84EA03059BB2ADB208BFA5
:10C418001D466B0015F4004F84EA03009BB280B2FE
:10C4280008BF1846430010F4004F84EA03059BB286
:10C43800ADB208BF1D466B0015F4004F84EA030037
:10C448009BB280B208BF1846430010F4004F84EA3C
:10C4580003059BB2ADB208BF1D466B0015F4004F33
:10C4680084EA03009BB280B208BF1846430010F468
:10C47800004F84EA03059BB2ADB208BF1D466B00AE
:10C4880084EA030015F4004F85B298B218BF284615
:10C498008A42B1D130BC704783684268D0ED037AD4
:10C4A80000EB83010133934281ED040A836004BFEA
:10C4B8000023836000EB830393ED047A036870EE36
:10C4C800277A9A42C0ED037A77EEC77AC0ED037AED
:10C4D8000CDA013307EE103AF8EEC76AB7EE007AC5
:10C4E80087EEA60A036030EE070A704707EE102AA7
:10C4F800B8EEC77A87EE870A704700BF90ED097AD1
:10C5080090ED004AD0ED0A6AD0ED014AD0ED047AE8
:10C5180090ED035AD0ED025AA4EE007AB0EE406ACC
:10C52800B0EE470AB0EE667AA6EE247A67EEC07AD5
:10C53800A0EE457AE6EE257A80ED097AC0ED0A7A12
:10C54800704700BFD0ED057A90ED013AD0ED003A82
:10C55800D0ED064A90ED024A90ED077A90ED035A25
:10C5680090ED086AD0ED045AC0ED067AF0EE406A04
:10C5780027EE830AC0ED056AA3EEA60A80ED087AC5
:10C58800A4EE240AA5EE470AA5EEC60A80ED070A1E
:10C59800704700BFD0ED007A90ED017A30EE670A5F
:10C5A800E7EE007AB0EE670AC0ED007A704700BF88
:10C5B800704700BF50F8043C012280F83520143839
:10C5C80003B11847704700BF037F33B1012B03D174
:10C5D8004FF400630382704770474FF4806303820F
:10C5E800704700BF90F8493013B1002280F8492005
:10C5F8001846704770B5044682B01830256D94F817
:10C608005C106B460622A847A8B19DF804009DF867
:10C6180000609DF801109DF802509DF803209DF8D8
:10C62800053041EA062143EA002342EA0522A184B3
:10C63800E2842385012002B070BD00BF70B50446B6
:10C6480082B00830256A6B4606223B21A847A8B16C
:10C658009DF804009DF800609DF801109DF80250B7
:10C668009DF803209DF8053041EA062143EA00239E
:10C6780042EA05226182A282E382012002B070BDF3
:10C6880030B490E81200057B43690222AA404A6050
:10C698002268586A996A4FF6FE752A4088422260D5
:10C6A80004D1012283F8442030BC70479C695A6B3E
:10C6B8000C44D4600DD818690024411A51609C625A
:10C6C8001168002041F0010183F8440030BC11607A
:10C6D8007047411A51609862F2E700BF70B404686D
:10C6E800037B2268022101FA03F31A4213D042693C
:10C6F8000A49582000FB02124FF6FE76506852890C
:10C70800C5680068296831402960C168D24392B27F
:10C718000A40C260636070BC704700BF943E00204E
:10C7280030B4094B1C7864B1084B002503EBC404F2
:10C738001A6899885562D06808330143A342D160CA
:10C74800F6D130BC704700BFB4420020B842002088
:10C75800F0B4334C00EB800004EB80046468002CD8
:10C768005BD0304E49004FF42040CDB23060A16913
:10C77800090444D460682C4F45F08071384041F476
:10C78800903101434FF420406160306003E0411E66
:10C79800002838D00846A1698F07F8D54FF4204003
:10C7A800A262306002E0421E68B31046A269110618
:10C7B800F9D562681C4945F0007545F480350A4092
:10C7C80015434FF420406560306002E0421ED0B14E
:10C7D8001046A2699207F9D5A362A3694FF42040D5
:10C7E8009B06306005D4431E68B11846A3699B06B2
:10C7F800F9D520233060E3610120F0BC7047411E69
:10C8080008B10846B3E7094A138801339BB24FF0D1
:10C81800FF3131601380F0BC70472046F0BC704790
:10C828008C620020B4620020009800FCB8620020EE
:10C83800B0F1FF3F09D0022810B402DC5DF8044BC8
:10C8480086E700205DF8044B70470020704700BF62
:10C858009AB170B505460C468E1801E0B4420AD06C
:10C8680014F8013B697895F900008022FFF7E0FF92
:10C878000028F3D170BD012070BD0120704700BFB2
:10C88800134600200A46682162E700BF014B18687A
:10C8980003F07EBDA874002070B5044690F84D00E2
:10C8A800002833D104F11805636D80226B212846D6
:10C8B8009847642005F00CFC636D284603226B2121
:10C8C8009847636D94F848201921284698470F2007
:10C8D80005F0FEFB636D94F8462028461A21984718
:10C8E800636D284618221B219847636D2846182235
:10C8F8001C219847636D284602223721984728460D
:10C90800636D01223821BDE87040184703F00AFF23
:10C918000546F0B1036881881B8A1940C2D12023DB
:10C92800C171837104F094F92146104B41F8143F0A
:10C93800284618F0EFFAAB88B3FA83F3C3F11F0364
:10C948005A1CAFD001229A4009490B6813430B6067
:10C95800A8E7014604F07CF92146044B41F8143F4E
:10C96800284618F0D7FA0122EEE700BFBDC5000837
:10C9780000040140084611461A4615F01FBB00BFC7
:10C98800F0B5064683B00D460024012714E00329BC
:10C998000CBF03220122C3F3011E6946C3F38103BE
:10C9A80030468DF805208DF806E08DF8073012F036
:10C9B8007FF80134102C0FD02B8807FA04F21342A9
:10C9C800F7D0AB78E9780092022903F003028DF8DA
:10C9D8000420DCD10A46DEE703B0F0BDF8B51A4DF5
:10C9E8002B789F2B2ED16B78BE2B2BD10522174984
:10C9F800A81C1EF044FB28BB072229464FF6FF70EF
:10CA0800FFF7F4FC124FEC1D22884AB1A618BE426B
:10CA180018D2052A16D92146FFF7E8FC3446F3E771
:10CA280021460222FFF7E2FC0222A118FFF7DEFCF2
:10CA38000634084B641B1C8041F60F53C31A584236
:10CA48005841F8BD0020F8BD00F00308F4D90208E9
:10CA580000000408425D00202DE9F04FDFF85491F2
:10CA68004F4F8DB00326A7EB090718220DEB0200E4
:10CA780000211EF0B9FA4B4BCDF8189007971A69A8
:10CA8800120604D5484A5A6002F188325A600122D7
:10CA98008DF82C203422DA60444B454C18689A886B
:10CAA80004909B79ADF8142004A9072206A88DF8F4
:10CAB800163004F061FC072204A94FF6FF70FFF757
:10CAC80095FCDFF8F4B080464FF0000A5C4536D399
:10CAD8000CAC002524F82C5D0222214606A804F09F
:10CAE8004BFC022221464046FFF780FC40BAC04377
:10CAF800ADF80800022202A906A804F03DFC099836
:10CB080060B108ABC0F10402294618441EF06CFA63
:10CB1800089906A804F0D6FB09950A909DF82C30D0
:10CB28000A9A23B11F490B6943F080030B61013E48
:10CB38002DD0002A99D1FFF751FF50B32CE065881A
:10CB48008DF80DA0C5F30B05AA1DADF808202288A5
:10CB5800C2F30B01120BADF80A108DF80C2002A9D4
:10CB6800062206A804F008FC062202A94046FFF7A0
:10CB78003DFC616880462A4606A804F0FDFB616812
:10CB880040462A46FFF732FC143480469EE7002AC6
:10CB9800D1D0052004F0FAFF0DB0BDE8F08F00BF3A
:10CBA8000000040800200240230167453CB6020843
:10CBB8004006030800F00308140A03080378202B32
:10CBC800024600F10100F9D0092BF7D02D2B2CD00B
:10CBD8002B2B03BF5378B7EE000A0246B7EE000AC4
:10CBE800A3F13001C8B209289FED467A10D8F2EEB9
:10CBF800046A07EE901AF8EEE77A12F8013FE7EEBA
:10CC0800267AA3F13001C8B20928B0EE677AF0D9C4
:10CC18002E2B4CD003F0DF03452B0BD0F7EE007A18
:10CC280067EE276A20EE260A70475378BFEE000A9F
:10CC38000246D5E710B451782D2959D02B290ABFBF
:10CC48009178501C901C0024A1F13003092B53D873
:10CC5800002303EB830301EB430310F8011FA1F149
:10CC68003002092AA3F13003F3D9B3F59A7F28BF1C
:10CC78004FF49A73072B42D9DFED236A1A46F7EE71
:10CC8800007A083A072A67EEA67AFAD803F007036B
:10CC98002BB1F2EE046A013B67EEA67AFBD124B30E
:10CCA800C7EE276A5DF8044B20EE260A70475378D2
:10CCB800A3F13001C8B2092802F10102AAD8F2EEA4
:10CCC800046AF0EE665A07EE901AF8EEE77A12F860
:10CCD800013F87EEA66AA3F13001C8B2092866EEC3
:10CCE800A56A37EE067AEED994E767EE276AD9E7A0
:10CCF800901C91780124A7E7F7EE007ACFE7F7EECA
:10CD0800007AC5E70000000020BCBE4CB5EEC00AA2
:10CD1800DFED317AF1EE10FACCBF30EE270A30EEB3
:10CD2800670ADFED2E7A20EE270A30B5FDEEC07ACD
:10CD380087B017EE904A054684EAE470002303A9F9
:10CD4800A0EBE4700193009302930CF007FF002C12
:10CD5800ACBF20232D2303A88DF800301BF012F957
:10CD6800012803A924D002282DD0032805BF302389
:10CD7800684668468DF801301EF05CF968461BF07D
:10CD880001F90338C4B22246694628461EF0B0F9B4
:10CD980000232B5528461BF0F5F82E22431C2A5455
:10CDA8000DEB0401E8181EF062F9284607B030BD03
:10CDB800302368468DF801308DF802308DF8033045
:10CDC8001EF038F9DAE7302368468DF801308DF81F
:10CDD80002301EF02FF9D1E76F12033A00007A44AF
:10CDE8002DE9F041064615460846B6FBF2F43CB973
:10CDF80005FB1464124B1B5D00F8013BBDE8F08194
:10CE0800B4FBF2F767B90E4B05FB174705FB146433
:10CE1800DA5D00F8012B1B5D00F8013BBDE8F081ED
:10CE2800B7FBF2F8B8F1000F02D04046FFF7D8FF81
:10CE380005FB1878024B13F8082000F8012BE3E7EC
:10CE4800FCD9020830B402681146531C036011F87B
:10CE5800024B0160D31C517803609378151D05605F
:10CE68001B0443EA0123D078234343EA006030BC23
:10CE7800704700BF0368591C1A46016012F8021B6C
:10CE88000260587841EA0020704700BF38B5044670
:10CE9800006815461EF083F822682A44226038BDCF
:10CEA800036810B40A0A5C1C04601A7003685A1CF0
:10CEB800026019705DF8044B704700BF03685A1C84
:10CEC800026010B4197003680A0A5C1C04601A70C6
:10CED80003680A0C5C1C04601A700368090E5A1C6B
:10CEE800026019705DF8044B704700BF03685A1C54
:10CEF800026019700368090A5A1C026019707047A9
:10CF08002DE9F047002488B080460F461E46A1460A
:10CF180005AD531C0393117839B3252933D1931CDC
:10CF2800CDF810900393507830284ED04FF0000A77
:10CF3800A0F13003DBB2092B42D96C2819D0642840
:10CF480000F0938024D825281CD063D9582876D09F
:10CF580063281BD131784046B847039A531C039382
:10CF68001178043601340029D7D1204608B0BDE82D
:10CF7800F087039B5A1C03921B78642B7CD02AD819
:10CF8800252B54D1252140460134B847039AC0E7E0
:10CF9800732833D044D975284FD106F1040E306870
:10CFA8002B4600220A217646FFF7A4F9049A009539
:10CFB800534639464046FFF7DBF9039A0444A8E78D
:10CFC80004AA03A90CF0A6FDB7E7D31C0393907835
:10CFD8004FF0010AACE7732B10D05BD9752B3AD010
:10CFE800782B96D1A3F15802B2FA82F2306852092E
:10CFF8002B4610210436FFF77DF9D7E73368049AEA
:10D008000093394600234046FFF7B2F9043604443A
:10D01800039A7EE70028B9D1204608B0BDE8F0871A
:10D028006E28B3D1039A336804361C6071E72AD995
:10D03800582BD7D0632B8DD06BE77828A6D1A0F1D9
:10D048005802B2FA82F2306852092B461021FFF7D3
:10D0580051F90436AAE706F1040E30682B4600227F
:10D068000A217646FFF746F9A0E7331D30682946BE
:10D078001E46FFF711F999E7331D306829461E4609
:10D08800FFF70AF992E7002B7FF443AF204608B078
:10D09800BDE8F0876E2BC6D03BE700BF0EB400B5E5
:10D0A80084B005AB019053F8042B0649039301A8FB
:10D0B800FFF726FF019B00221A7004B05DF804EB0D
:10D0C80003B070476DC300080FB430B583B006AB2A
:10D0D8000B490C4853F8042B096800680193FFF7C3
:10D0E8000FFF094C0546206803685B6998470028CC
:10D0F800F9D0284603B0BDE8304004B0704700BFFF
:10D10800BC300020C0300020A8740020DFED2B7A4E
:10D11800B4EEE70AF1EE10FA4ADDDFED296A9FED79
:10D12800297A01E0B0EE670AB4EEC70AF1EE10FA08
:10D1380070EE667AF6DC9FED247AF4EEC77AF1EEAB
:10D1480010FA38D5DFED1E6A9FED207A01E0F0EE87
:10D15800407AF4EEC77AF1EE10FA37EEA60AF6D462
:10D16800DFED1B7AB4EEE70AF1EE10FA14DDDFED1D
:10D17800137A37EEC00A60EE006A9FED166A9FEDDB
:10D18800167ADFED167AA6EE867A20EE266AE6EEA5
:10D19800877AA6EE270A7047DFED117AB4EEE70A20
:10D1A800F1EE10FA44BFDFED087A37EEC00AE2E785
:10D1B800F0EE407ABFE7B0EE670AD1E7DB0F4940EF
:10D1C800DB0FC940E4CB1641DB0F49C0E4CB16C1E5
:10D1D800DB0FC93F92E741B99730083C15A82ABE32
:10D1E800DB0FC9BF41404A0011F0800F82F0D50320
:10D1F800D2B2DBB208BF1346590013F0800F81F09A
:10D20800D502C9B2D2B208BF0A46510012F0800F47
:10D2180081F0D503C9B2DBB208BF0B46590013F041
:10D22800800F81F0D502C9B2D2B208BF0A465100B8
:10D2380012F0800F81F0D503C9B2DBB208BF0B46EC
:10D24800590013F0800F81F0D502C9B2D2B208BFDD
:10D258000A46510012F0800F81F0D503C9B2DBB243
:10D2680008BF0B465A0082F0D50013F0800FD2B2E7
:10D27800C0B208BF1046704709B909E0194690FBCB
:10D28800F1F301FB13030846002BF7D1084670475A
:10D298000146FBE710B507EE901A2DED028BB8EEAC
:10D2A800678ADFED227A28EE008A044628EE278A6C
:10D2B800B0EE480A1BF0CCFDF0EE408AB0EE480A0A
:10D2C8001BF028FDF7EE007A9FED197AF0EE675A09
:10D2D800E8EE875A0023A361B0EE676AC7EEA56A35
:10D2E80063612362E361A3626362A8EEC76ABDEC6F
:10D2F800028B77EEC07AB6EE007AF8EE005A27EE87
:10D30800877A20EE250A27EE267A26EE266A67EE29
:10D31800A67A20EE260A84ED046AC4ED017A84ED2B
:10D32800007A84ED027A84ED030A10BD27D4D23640
:10D33800F304353F10B44C09012250F8243001F0B1
:10D348001F0102FA01F10B4340F824305DF8044B49
:10D35800704700BF4B0901F01F0150F8232001233B
:10D3680003FA01F1114214BF18460020704700BFAC
:10D37800203970B501EB81010B4C4E1D2644054642
:10D388000C4414F8013B697895F900004022FFF736
:10D398004FFAB442F5D1697895F90000002340228C
:10D3A800BDE87040FFF744BA44B6020838B50C46E9
:10D3B800097839B105462846FFF7DAFF14F8011F46
:10D3C8000029F8D138BD00BF30B583B0A1F15005B0
:10D3D80010230024032201A98DF804508DF805407C
:10D3E8008DF80630FFF734FA03B030BD30B501EBE5
:10D3F8004104214683B0C1F3C3036400A2F1500580
:10D40800103304F00E04032201A98DF804508DF89E
:10D4180005408DF80630FFF71BFA03B030BD00BF9A
:10D4280038B5042208490546FFF712FA4FF480641C
:10D43800013C00234022697895F90000A4B2FFF767
:10D44800F7F9002CF4D138BDE8B8020838B58022C5
:10D4580041780446AE2390F90000FFF7E9F9054644
:10D4680088B1162209492046FFF7F2F90422084933
:10D478002046FFF7EDF92046FFF7D2FF20460322AA
:10D488000449FFF7E5F9284638BD00BFECB80208A3
:10D4980004B9020808B90208F0B5574B574A97B0C3
:10D4A8001968914200AF00F09C805549554A002305
:10D4B8004FF47000C1F888003B607B60136843F448
:10D4C8008033136003E03B68B3F5A04F09D01368BD
:10D4D80003F400337B603B6801333B607B68002BBF
:10D4E800F1D0484B1B6813F4003318BF01237B604D
:10D4F8007B68012B4BD0424D424B434AEA60434A7A
:10D50800596A11605A6A424E42F080725A625A69E8
:10D5180007F1580442F4FC0241F6FF715A6124F8FD
:10D52800501D032321464FF09040BB72FFF728FAA5
:10D538004FF6FF73214637483B81FFF721FA214612
:10D548003548FFF71DFA21463448FFF719FA2146F6
:10D558003348FFF715FA21463248FFF711FA2046FB
:10D5680011F0B2F8BB683049304AA1FB03133049C7
:10D578009B0CF02400204FF0070E5C370B605660C0
:10D5880085F823409060C2F800E0BD46F0BD294A06
:10D598001C4B122111605A685A605A685A605A68BE
:10D5A80042F480625A605A6822F47C125A605A68BF
:10D5B80042F4E8125A601A6842F080721A601A68D7
:10D5C8009201FCD559680F4A21F003015960596846
:10D5D80041F002015960536803F00C03082BFAD19B
:10D5E80089E700221A6062B6134B1B6883F3088828
:10D5F800124B1B689847FEE7FC9F0020EFBEADDE8C
:10D6080000ED00E0001002400005FA052843002064
:10D618003F1901000004004800080048000C0048B9
:10D62800001000480014004883DE1B4310E000E0AF
:10D63800F46200200020024000D8FF1F04D8FF1F1A
:10D648002DE9F04F714C54F8205083B0002D00F0B4
:10D658009A80D5F854901F46D9F804302B65A960F4
:10D668004FF4807305F15A019046064605F5AD72F0
:10D67800674828606961AA61EB602B6199F8180016
:10D6880014F096FAD9F80C40F4B162480021034628
:10D698005A68944203F11C0303D001310C29F7D1D5
:10D6A8000021C1EBC10100EB81015B480B694269B4
:10D6B8004FF00C0E1A43731C426181F818E04B7648
:10D6C8002B6D2C632433EB64D9F80810002936D06D
:10D6D8005048002403465A68914203F11C0303D0C2
:10D6E80001340C2CF7D10024C4EBC40400EB8401F2
:10D6F800494B0A695869494C104358610B20087610
:10D70800701C48765869024399F81B005A618309CE
:10D71800002291F80DE08DF805304D6101238C60F1
:10D7280001A88DF806208DF807308DF804E014F074
:10D738003FFD2B6DD9F808206A632833AB6495F850
:10D74800590002F0EFFF044695F8580002F0EAFF8E
:10D758003A07824699F819B019D5C4B117F0110FD4
:10D768004FF00B0306F1010614BF4E213E21A371B1
:10D77800E6715A46204603F099F8FB0741D52B6B12
:10D788004BB36B6B3BB3284603B0BDE8F08F17F083
:10D79800010F0CBF2E274E2718F0020F09D044B1F5
:10D7A8000B22731CA271E37120465A46394603F0D6
:10D7B8007DF818F0010FE2D0BAF1000FDFD0013682
:10D7C8000C238AF807605A4639468AF806305046CC
:10D7D80003F06CF8D3E799F81A308DF8043099F80B
:10D7E8001C3000219B09012201A88DF805308DF815
:10D7F80006108DF8072014F0DBFC284603B0BDE8BE
:10D80800F08F204603F0E0FBB9E700BFC8300020E6
:10D818000CB90208341800200010024089C600081C
:10D828000348D0F83C3113B100F59A701847704797
:10D83800341800200348D0F8203113B100F58C705B
:10D8480018477047341800200348D0F804310BB14A
:10D85800FC301847704700BF341800200348D0F840
:10D86800E8300BB1E0301847704700BF341800208B
:10D878000348D0F8CC300BB1C4301847704700BF0C
:10D88800341800200348D0F8B0300BB1A83018473E
:10D89800704700BF341800200348D0F894300BB10B
:10D8A8008C301847704700BF341800200248836F37
:10D8B8000BB1703018477047341800200248C36D08
:10D8C8000BB1543018477047341800200248036CD5
:10D8D8000BB1383018477047341800200248436AA3
:10D8E8000BB11C3018477047341800200248836871
:10D8F80003B11847704700BF341800201749184B68
:10D90800184A194810B4D1F8884044F47004C1F892
:10D9180088401C6844F001041C605C6822405A601E
:10D928001A6822F0847222F480321A601A6822F48B
:10D9380080221A605A6822F4FE025A60DA6A22F0DB
:10D948000F02DA621A6B002410404FF0006218636D
:10D958009C608A605DF8044B704700BF00ED00E0F2
:10D96800001002400CC07FF8CCFC00FF064B1B786F
:10D97800DB0700D57047054B1B68002BFAD01B68E6
:10D988001B68002BF6D01847855B0020A86500208F
:10D99800F8B53422044600211DF026FB1422234B3F
:10D9A800A27093F90260224AC4F8032001201E25C0
:10D9B8001F27002184F8225086424FF0020584F880
:10D9C8002A70C4F80B20C4F81320C4F81B20C4F82C
:10D9D8002320C4F82B20A172A0742080A5761AD029
:10D9E80093F90A10814216D093F91220824216D078
:10D9F80093F91A20824214D093F92220824212D03D
:10DA080093F92A20824205D05222642384F83220D6
:10DA18002386F8BD0521402223F83120F4E7294662
:10DA2800F9E70321F7E70421F5E700BF2C7400208C
:10DA3800050405002DE9F04F83B0484C484F01908C
:10DA4800019803685B699847002840F08380DFF8F5
:10DA580018914448D9F80430DFF810E1C3F30803FB
:10DA68004FF00A0A4FF0100C4FF47A75002B3BD197
:10DA7800EFF31183002B37D10168A26800BF036858
:10DA88009942F9D1DEF8006005FB06F39B1AB3FB57
:10DA9800F6F305FB013101260091D9F80430C3F3F0
:10DAA8000803002B3BD1EFF31183002B37D1036818
:10DAB800A16800BF02689342F9D1DEF800B005FB07
:10DAC8000BF2521AB2FBFBF205FB0323009A9B1AD6
:10DAD800B3F57A7FE1D3BAF1010AB1D0D9F80430AD
:10DAE800C3F30803002BC3D0EFF311828CF3128821
:10DAF800A6682368D90302D501233B60A66803689A
:10DB08003968D2B282F31188DEF80020194405FB87
:10DB180002F39B1BB3FBF2F305FB0131BBE7EFF309
:10DB280011888CF31288A1682368DB0344BF3E6028
:10DB3800A16803683A685FFA88F888F31188DEF804
:10DB480000801A4405FB08F35B1AB3FBF8F305FBE6
:10DB58000233BBE703B0BDE8F08F00BF10E000E080
:10DB6800EC620020F062002000ED00E0F46200208A
:10DB7800F8B5B74CB74D0E46482200210746204657
:10DB88001DF032FAB44A701CD37A927A4FF006012B
:10DB980046D012B3002B5DD0002F40F00481DFF88F
:10DBA800BCE238464FF0FF0C08E0012A03D80139DF
:10DBB800C9B287F800C00C30482849D01EF9013F87
:10DBC8002354A3F11E029E42D2B204EB0007ECD10B
:10DBD800013904F800C0C9B2EDE7002B5AD0002F74
:10DBE80040F0A980DFF874E238464FF0FF0C08E0F7
:10DBF800012A03D80139C9B287F800C00C30482877
:10DC080026D01EF9013F2354A3F11E029E42D2B230
:10DC180004EB0007ECD10139C9B204F800C0EDE704
:10DC2800002B57D0002A00F0CF80002F40F0188139
:10DC38008A4A3846FF2612F9013F23541E3BDBB2BD
:10DC4800012B02D801392654C9B20C304828F2D128
:10DC58002970F8BD002F54D1DFF800E238464FF0A4
:10DC6800FF0C08E0012A03D80139C9B287F800C0BF
:10DC78000C304828ECD01EF9013F2354A3F11E02B2
:10DC88009E42D2B204EB0007ECD10139C9B204F8C4
:10DC980000C0EDE7002F69D1DFF8C0E138464FF04A
:10DCA800FF0C08E0012A03D80139C9B287F800C07F
:10DCB8000C304828CCD01EF9013F2354A3F11E0292
:10DCC8009E42D2B204EB0007ECD1013904F800C03F
:10DCD800C9B2EDE7002A00F08980002F40F0D0801B
:10DCE8005E4A3846FF2612F9013F23541E3BDBB239
:10DCF800012B02D801392654C9B20C304828F2D178
:10DD0800A6E756484FF0FF0C07E01F2A02D18EF80D
:10DD180000C0F9B20C33482B9AD010F9012FE25405
:10DD2800964204EB030E01F1FF37EED1013904F8F6
:10DD380003C0C9B2EEE7494813464FF0FF0E09E0A9
:10DD48001E2A03D10139C9B287F800E00C33482BE9
:10DD58003FF47EAF10F9012FE254964204EB03071B
:10DD6800EED1013904F803E0C9B2EFE73B4F4FF0B9
:10DD7800FF0C09E0012803D80139C9B28EF800C0A8
:10DD88000C33482B3FF464AF17F9012FE254A2F18A
:10DD98001E00B242C0B204EB030EEBD10139C9B286
:10DDA80004F803C0ECE72D480023FF2703E00C33F9
:10DDB800482B3FF44DAF10F9012FE2549642F6D1AB
:10DDC8000139E754C9B2F2E79FBB244A3846FF2617
:10DDD80012F9013F23541E3BDBB2012B02D8013953
:10DDE8002654C9B20C304828F2D131E787B91B4A0A
:10DDF8003846FF2612F9013F23541E3BDBB2012BA4
:10DE080002D801392654C9B20C304828F2D11FE78C
:10DE180012481346FF2610F9012FE2541E3AD2B2D7
:10DE2800012A02D80139E654C9B20C33482BF2D181
:10DE38000EE70A481346FF2610F9012FE2541E2A5E
:10DE480002D10139E654C9B20C33482BF4D1FFE6AC
:10DE5800AC650020682300202C43002033B9020859
:10DE680014230027012602201E2223701F23277354
:10DE7800267684F8240084F8302084F83C30E7E6DD
:10DE88000648FF2610F9012FE2541F2A02D1013952
:10DE9800E654C9B20C33482BF4D1D9E633B9020899
:10DEA800134B5A6890420FD01A69904216D0DA691B
:10DEB800904215D09A6A904214D05A6B904213D06F
:10DEC8001A6C904212D07047002202EB420203EB18
:10DED80082030022C2621A815A6070470122F4E765
:10DEE8000222F2E70322F0E70422EEE70522ECE73C
:10DEF800AC6500202DE9F04FD14D95F9004093B065
:10DF080084429DF870909DF874801CD095F90C405F
:10DF1800844200F0B58395F91840844200F0B38339
:10DF280095F92440844200F0DC8395F9304084421E
:10DF380000F0DA8395F93C40844200F0D883002051
:10DF480013B0BDE8F08F4FF0000A4FEA4A0606EB1F
:10DF58000A0405EB84042489002CF0D11F468DE8BF
:10DF680006001F28EBD801A353F820F089E3000826
:10DF780089E3000889E3000847DF000847DF000855
:10DF880047DF000847DF000847DF000847DF0008D1
:10DF980047DF000847DF000847DF000847DF0008C1
:10DFA80047DF000847DF000847DF000847DF0008B1
:10DFB80047DF000847DF000847DF000871E2000874
:10DFC80047DF000847DF000847DF000847DF000891
:10DFD80047DF000847DF000847DF000847DF000881
:10DFE80047DF000839E10008F5DF0008954BDC7DC4
:10DFF80093F80BB0204617F0F7FB0490584617F03B
:10E00800F3FB0290204602F08DFB0590584602F083
:10E0180089FB18F008030393029B00F0EB82002BA6
:10E028008DD0894CC4F89C32C4F89802C4F8940284
:10E0380018B10B210C228171C27109F002020292FF
:10E04800DFF81CB2814984F869921846019BC4F82C
:10E0580090324FF000094FF4807201230BF5807E57
:10E06800C4F87022C4F8742284F8B434C4F87CE28A
:10E07800C4F86412C4F86C72394684F86A82C4F829
:10E0880078B2C4F88492C4F88092C4F88C92C4F828
:10E098008892C4F8B09484F8A89484F8A994019359
:10E0A80018F01CFD08F00101D4F89C0217F01EFBC3
:10E0B800029B6749674AC4F8C014C4F8BC94C4F802
:10E0C800B824D4F89C12002B00F04882D4F8A0029F
:10E0D800002800F043820A680368934200F03E82F9
:10E0E800019B84F8B534394618F0F8FC0BF5057136
:10E0F800D4F8A00217F04EFA4A460BF50771D4F887
:10E108009C0203F07BFB039B002B00F0AD82524C7A
:10E11800204618F00DFD50481F24564405EB86058F
:10E12800BDF8003004712B81686013B0BDE8F08F32
:10E13800444B9C7D93F80AB0204617F055FB049099
:10E14800584617F051FB0290204602F0EBFA059072
:10E15800584602F0E7FA18F008030393029A00F011
:10E168002D82002A3FF4EBAE374CE263A063606374
:10E1780010B10B238371C37109F002030293DFF816
:10E18800E4B0324984F809901046019A22634FF0AE
:10E1980000094FF480720BF58073E36122616261BC
:10E1A8006160E760394684F80A80C4F818B0C4F89A
:10E1B8002490C4F82090C4F82C90C4F8289084F8CF
:10E1C8005492C4F8509284F8489284F8499218F00E
:10E1D80085FC08F00101E06B17F088FA029B1C49E6
:10E1E8001C4AC4F86012C4F85C92C4F85822E16B67
:10E1F800002B00F0A981206C002800F0A58103689D
:10E208000A68934200F0A081012284F85522394619
:10E2180018F064FC0BF50571206C17F0BBF94A4641
:10E228000BF50771E06B03F0E9FA039B002B00F094
:10E2380011820A4818F07CFC1E2408486DE700BFCC
:10E24800AC6500202C4300206823002064B9020834
:10E25800F9650208996B0208CC2500206C23002080
:10E268000C260020AC230020C14FC248BB69C24C19
:10E2780043F00103BB61112102F0EAFCBD4802F042
:10E28800A3FEC82003F024FFBC4B1A6EB3F8643019
:10E2980093617B6943F400337B614FF000084FF4CE
:10E2A800C05203234FF0020B07A94FF0904007928A
:10E2B8008DF821308DF820B08DF822808DF82380DC
:10E2C80010F0F6FB4FF09043AD495A6A22F47042C1
:10E2D8005A625A6A42F460425A625A6A22F47022B6
:10E2E8005A625A6A4FF4802042F460225A624FF010
:10E2F800010908601222082304F20C50C4F80C2506
:10E3080084F8113584F8129516F092FD9D4B9E49BC
:10E31800C3F80080FB699D489D4A43F40003FB61F4
:10E328009C4F0B6801609C4982F808B03A609B4A90
:10E338000A6098479A4B9B4ADA6007A814238DF81D
:10E348001C308DF81DB08DF81E808DF81F9013F0CD
:10E358002FFF9DF81F308DF81D902A228DF81E8002
:10E368008DF81C20002B40F071818F4B4FF4806298
:10E37800C3F884208D4BC4F8C4348D481424CCE6EB
:10E38800C4B2204643464A463946FFF759F9834600
:10E3980000283FF4D4AD006D8BF805908BF806800B
:10E3A8000268019BCBF82C3022F0010200230121E6
:10E3B800CBF808708BF84410CBF82030CBF81C3021
:10E3C800CBF82830CBF82430026018F00402079705
:10E3D80000F030814FF48053089318F0020340F0A6
:10E3E8009D8109934FF48063002219F001080A9374
:10E3F8000C9240F01B81CDF82C80082319F00207FD
:10E4080007A918BF0B930FF0FFF99BF805309BF88D
:10E41800061003F00202002A15BF4FF440324FF4F1
:10E4280080324FF40030002013F0010FDBF8503039
:10E4380008BF0246586811F0010F14BF024320EAD2
:10E4480002025A609A6809074CBF42F0080222F09B
:10E4580008029A601A6842F001021A60B8F1000FC7
:10E4680037D0DBF83020002A00F04C8107A80FF0E5
:10E47800F5F8DBF84C30DBF80C20DBF81410DBF88F
:10E48800300007934FF480531093002308911193A1
:10E4980080210B930D930E9309932023ADF8282028
:10E4A8000F930C910FF008F907A9DBF830000FF073
:10E4B800E3F8DBF83020DBF85030116841F0010157
:10E4C8001160996841F040019960526892B2CBF8A6
:10E4D8004020002F32D0DBF83420002A00F01981C8
:10E4E80007A80FF0BBF8DBF84820DBF810300792DC
:10E4F8004FF480520027DBF834001092ADF8283032
:10E50800802210230C92099311970B970D970E9761
:10E518000F970FF0D1F807A9DBF834000FF0ACF82B
:10E52800DBF83420DBF85030116841F0020111604B
:10E53800576057609A6842F080029A601A6842F001
:10E54800010258461A60E8E51A4A0023084684F88A
:10E55800553202F1080103F051F966E6164A002324
:10E56800084684F8B53402F1080103F047F9CAE512
:10E57800001002402C59002068230020CC580020AD
:10E5880014040140D8004242BC190020205B00203E
:10E598004065002034650020105B00200C0000203E
:10E5A80000ED00E00005FA0500E100E03CB90208D2
:10E5B8002C280020C02500202028002019F0010E5A
:10E5C80011D0002C3FF4BBAC049B002B3FF4B7AC3C
:10E5D8005549059C4C63CB632CB14FF00C0C0B21B7
:10E5E80084F806C0E17119F0020102914ED14E4C37
:10E5F800E26BC4E519F0010E10D0002C3FF49FAC7B
:10E60800049A002A3FF49BAC4749059CC1F8944200
:10E61800C1F89C2214B10C21A171E17119F0020119
:10E62800029147D1404CD4F89C3209E504230B935E
:10E638000C23E3E618F00203089208BF09933FF49D
:10E64800D3AE4FF4005113460991CDE607A813F055
:10E65800AFFD8FE6A06B10B1012101F0ABFE0121E7
:10E66800324818F083FAE4E5D4F8980210B1012191
:10E6780001F0A0FE2E4C0121204618F077FA47E55C
:10E688004FF0010A61E44FF0020A5EE4BBF1000FAB
:10E698003FF455AC244CA063BEF1000F2AD1002AE8
:10E6A8003FF44DACE26300283FF469AD0B2383715E
:10E6B800C37164E5BBF1000F3FF441AC1A4CC4F8D8
:10E6C8009802BEF1000F18D1002B3FF438ACC4F803
:10E6D8009C3200283FF4B4AC0B210C228171C2712A
:10E6E800AEE44FF0030A30E44FF0040A2DE44FF093
:10E6F800050A2AE42264E26BD5E7C4F8A032D4F80C
:10E708009C32E6E720221A621A6842F020021A6058
:10E71800DFE61A6842F080021A600FE74FF40053F0
:10E7280009934FF480635FE6682300206C23002080
:10E73800CC25002038B1038813EA010003D08B42AE
:10E748000CBF012002207047184B19491A88104243
:10E7580011D11A89104217D11A8A10421AD11A8B6C
:10E7680010421AD11A8C10421AD11A8D10401AD19F
:10E7780006230B707047012210B400240A7003EBC3
:10E78800C4005DF8044B7047022201200A7003EBB5
:10E79800C000704703220220F8E704220320F5E7AF
:10E7A80005220420F2E706220520EFE72C7400205A
:10E7B8002874002080B3B0F5165F2ED0B0F5964FC0
:10E7C8002DD0B0F5164F2CD0B0F5614F2BD0B0F549
:10E7D800E13F2AD0B0F5613F29D01D4B984228D09F
:10E7E8001C4B984227D0B0F5E12F26D01A4B9842FF
:10E7F80025D0B0F5612F24D0184B984223D0184B60
:10E80800984222D0174B984205D0174B98420CBF1C
:10E818000F20002070470E2070470120704702200B
:10E828007047032070470420704705207047062072
:10E8380070470720704708207047092070470A2052
:10E8480070470B2070470C2070470D20704700BFA1
:10E8580090D00300801A060020A1070040420F0054
:10E8680060E3160080841E0070B0250010B50020FB
:10E8780003F0E6FC074B00241C7001F06BFB064814
:10E888000649074A074B80F814450C6014801C6041
:10E8980010BD00BF3E75002068230020101E002018
:10E8A8000E1E00209C1D002058B31C4B1B689B03A8
:10E8B8001FD41B4A012188424FF0000302F10C02C9
:10E8C80008D00133152B13D012F80C1C884202F122
:10E8D8000C02F6D130B4134C206898B15900124A92
:10E8E8004578C81802EB80004078A8420CD330BCA9
:10E8F80070470E4B1B79002BDBD00D4B1B78002B80
:10E90800D7D1B3E7084A59000B440A480A4902EB31
:10E9180083020023226003800B60E8E7685D002023
:10E9280068D002089C1D00205CD00208E05E002030
:10E93800423E00200E1E0020101E00202DE9F0414E
:10E9480005460D2005F078FD002844D13E4E336879
:10E9580023B33E4F3A68AA4220D83D4A147814F0AF
:10E96800010402D11A780A2A55D03A493A4C91F84A
:10E978001425AAB95868228810F802E0012081F805
:10E988001405BEF1000F2AD1002342F210710132A2
:10E9980001FB035522803D60BDE8F081BDE8F081B0
:10E9A8005B6822889B5C4FF0000881F81485002B77
:10E9B800EAD0404603F044FC284B83F8008001F07D
:10E9C800C9FA336822885B689B5CFE2B34D100232C
:10E9D8002380BDE8F0810A20FFF766FFB6E71B78C1
:10E9E8001F4A013B126800FA03F3134229D01B4B5C
:10E9F80001221A7001F0AEFA22883368002AE2D1A7
:10EA0800197805390129DED803F016FB154A336851
:10EA180010602288D7E7DFF8508098F80020002A95
:10EA2800A3D0E0B2032117F02FFD98F8003001348D
:10EA3800A342F6D8336898E7FF2BA6D1BDE8F0418A
:10EA480014E703F0FDFBD2E79C1D0020101E0020F8
:10EA5800855B0020682300200E1E00203E750020E4
:10EA6800685D002080640020493D00204000402867
:10EA7800094A30B4A8BF4020002302251424D554E5
:10EA88000233D118984201F8014CF8D8FF21D1542B
:10EA98000F2030BC08E700BF945E002038B5094D50
:10EAA8002B8823EA0000834228800AD0064B1421D1
:10EAB800FF220F2002241C7059709A70FFF7F4FE91
:10EAC800288838BDF81C0020945E002038B5094D10
:10EAD8002B881843834228800AD0074B1421FF2231
:10EAE8000F2002241C7059709A70FFF7DDFE2888E9
:10EAF80038BD00BFF81C0020945E0020F8B5514BCB
:10EB08005148524D524C4822002101261E701CF0DB
:10EB18006BFA5049504A002328460B60136000F0F6
:10EB2800ABFC2168CA0700F1818011F002016FD1A6
:10EB3800003118BF0121494C032000F037FD0121A5
:10EB4800052000F033FD2679454B311C1A8E454BC4
:10EB580093FBF2F318BF0121642B38BF642307200D
:10EB6800C5F8143100F022FD6779391C4FF0080010
:10EB780018BF012100F01AFD237A002B3CD03A4C33
:10EB8800002E43D1391C18BF0121092000F00EFDC9
:10EB98000121042000F00AFD344B0620197800F00A
:10EBA80005FD01210A2000F001FD21680B20C1F3B9
:10EBB800404100F0FBFC21680C20C1F3802100F0EB
:10EBC800F5FC21684B0508D5294B1B7A083B012B1E
:10EBD8009CBF4FF4FA63C5F88032C1F3C0610D20C1
:10EBE80000F0E4FC01210E2000F0E0FC01210F20E0
:10EBF800BDE8F84000F0DABC637A1B4C002BBFD1AB
:10EC0800216811F48021C0D0002EBBD00121BCE7BF
:10EC18000121022000F0CAFC164B21681B6B642BF3
:10EC280038BF642301F00201AB6781E7124B1B6810
:10EC3800642B314638BF642330466B6400F0B6FC61
:10EC4800216872E7A029002058290020B814002064
:10EC58005052002054290020A4290020E05E002002
:10EC68002C74002040420F00504300201045002023
:10EC7800FC4200206C60002040520020024B1A88A1
:10EC88009B780280837070478CB90208084B19681A
:10EC980061B130B45D68074C642202FB05F2B2FB37
:10ECA800F1F2228030BC002018605860704700BF25
:10ECB80080280020445D0020704700BF6F4B1B7800
:10ECC800002B3AD02DE9F0416D4B6E4D5B79AC6865
:10ECD800A860013B82B0041B032B00F29C80DFE894
:10ECE80003F04A02312918F03DFE002800F09B800D
:10ECF800654B66491B78B5F84A20D1ED037A6A65F9
:10ED0800DB0700F1AA8002FB04F007EE900ADFEDB2
:10ED1800606A604BB8EEE77AD5ED147A5A60E7EE90
:10ED2800267A1A60BDEEE77AC5ED147A85ED137A76
:10ED380083ED027A02B0BDE8F081564A1360536051
:10ED480093607047544B1B681801F3D5FF2009F0F6
:10ED580045FC03780A2B88BF00214E4B9CBFB0F9B5
:10ED68000420B0F90610A96588BF0A46EA655A600A
:10ED78001A609960DEE7494A494BD279DFF8308159
:10ED880033F81220B8F902304648B8F9001092B2A8
:10ED980007EE902A40F6E44707FB02F6C3EB16336A
:10EDA800B8EE670A4FF47A7606FB03F393FBF1F3A8
:10EDB800AB61FDF7A3FBD5F818E0D5ED047ADFEDDC
:10EDC800346AB8F90220334BB8F900C0C3F804E03C
:10EDD8000EFB04F007EE100AB8EEC77ABCEEC06A64
:10EDE800E7EE267A8DED016ABDF80410C5ED047AC8
:10EDF800BDEEE77A07FB01F7C2EB173706FB07F60C
:10EE080083ED027A96FBFCF685ED037A6E611E604F
:10EE180002B0BDE8F0811F4B00221A605A609A6068
:10EE280002B0BDE8F0811C4B1B68DE067FF560AFC1
:10EE3800154BB5F84A201B786A65D9077FF563AF8B
:10EE4800B5F94810184B00FB01F083FB0013C017FD
:10EE5800C0EBA31002446A6555E7FDEEE77A134E4E
:10EE680017EE900AA0F57A7101FB01F386FB030601
:10EE7800D817C0EB26100844E2E700BF423E002046
:10EE8800E05E002080280020855B0020443E0020B2
:10EE98002FE33E31BC5B0020504300206862002015
:10EEA800846200209C280020D34D62101F85EB51FE
:10EEB800A4640020F0B53E4B1B79012B83B03DD0F4
:10EEC800022B0FD03B4B00221A805A803A4B1B78FA
:10EED800022B05D1374A394B5188128819805A803C
:10EEE80003B0F0BD364B1B681B01EFD5FF2009F0BE
:10EEF80075FB03780A2B56D8B0F902203149D3178D
:10EF080081FB0212C3EBA2039BB207EE903AB8EE64
:10EF1800670A2D4C04F16400A4F86230FDF7EEFA9C
:10EF2800FCEEC07A234AB4F86230CDED017A538002
:10EF3800BDF80430A4F860301380C7E7234A244B97
:10EF48009278214D33F81240A4B207EE904A05F1A9
:10EF58009400B8EE670AFDF7D1FA1E4A15491078F1
:10EF680096785378FCEEC07A00EB4010CDED017A2C
:10EF7800BDF8042044F6FB77C3EB033300FB0272B1
:10EF880000FB0474B2FBF3F2B4FBF3F3B2FBF6F24A
:10EF9800B3FBF6F392B29BB2A5F89020A5F8923095
:10EFA8000A804B8092E79FED0C0A0023B1E700BF6F
:10EFB800E05E0020303E0020593D00205C3D0020EE
:10EFC800504300206766666680280020686200203B
:10EFD80084620020DB5E002000000000F8B5294DA7
:10EFE800294C2879294B2A4F2A4E0021032201282F
:10EFF8003A7084F8C020A4F8C210A4F8C410317084
:10F008001980598021D0022810D06979224A00231A
:10F018000129136084F8C6305360936023D0022915
:10F0280012D11E4AE36453609360F8BD302204F1A4
:10F0380060001BF0D9FF4CF250319FED190A04F122
:10F048006400FEF727F9E0E7F8BD302204F19000EC
:10F058001BF0CAFF4CF25031B7EE000A04F19400DD
:10F06800FEF718F9D1E70F4AE36053609360D36065
:10F078009FED0B0A02F110004CF25031BDE8F84048
:10F08800FEF708B9E05E002080280020303E00200E
:10F09800405D0020423E0020BC5B0020CC280020C0
:10F0A800CDCCCC3E8C2800202DE9F0432F4DD5F84F
:10F0B800C83083B01BB195F8CC30022B02D003B016
:10F0C800BDE8F0834FF020084046294C05F1D009EF
:10F0D8000126552705F0B0F9A0B199F800300BB911
:10F0E800217891B908F101085FFA88F8B8F1230F7F
:10F0F80004F1010409F10109E1D0404605F09CF949
:10F108000028EAD189F80000ECE7D5F8C80050B328
:10F118000DF1080EAA220EF8052D8DF802108DF8B3
:10F1280000708DF801608DF804306946552253400F
:10F13800082213F0800F02F1FF324FEA430318BF91
:10F1480083F0310312F0FF02DBB2F2D1714502D035
:10F1580011F8012FEBE7AA2269468DF803308DF8E4
:10F16800042015F055FA89F80060BBE780280020D4
:10F1780090B902081F4B1878002839D01E4AD38846
:10F18800FBB11E4A9FED1E6AD2ED026A07EE903A65
:10F19800F8EEE66AF8EE677A07EE103A77EEE66A76
:10F1A800B8EEC77A66EE866AC6EE877AFDEEE77A2B
:10F1B80017EE900A6428A8BF642020EAE070C0B265
:10F1C800704710B40F4B54781B88117804FB103229
:10F1D800091B642300FB01F003FB02F3B3FBF0F00F
:10F1E8006428A8BF64205DF8044B20EAE070C0B230
:10F1F800704700BF423E0020E05E0020BC5B00205C
:10F208000000C842303E00202DE9F04F794D81B012
:10F2180002F012FFD5F8D8400022C5F8D420002CFF
:10F2280000F0A580237D052B074617D9216A23699D
:10F238000B44C31A9342B8BF05F1DC010ADBD5E0E1
:10F24800137D052B0AD9136A1269FB1A9B1A002B26
:10F2580080F2CC8051F8042B002AF1D14FF0010B39
:10F268000023B9461E46C5F8D43098469A46274624
:10F2780023E07A6A39693B7DA9EB0204B4FBF1F417
:10F288000134A4B213FB04F3013301369BB2B6B2C6
:10F298003C83FB82984506D2BBF1000F01D1012CBB
:10F2A8005FD99846BA46D5F8D430013305EB8302C6
:10F2B800C5F8D430D2F8D87047B3BB68C3B1FC8A5C
:10F2C800002CD6D1396A4846A9EB01019847D0B13C
:10F2D80095F82031002B52D13B7DC7F82490013698
:10F2E80001334FF00102B6B23A83FB820124D1E721
:10F2F8003B6A3A69A9EB0304B4FBF2F4A4B23C8379
:10F3080034BBFB8AC6E73C83FB8AC3E72B686A6881
:10F318003949013316443C4685E848004F46C1F850
:10F3280000A0BAF1000F27D0DAF8203095F8202194
:10F33800AAF81640FB1ACAF81C30CAF82090002A0E
:10F3480035D1DAF80C30484601B0BDE8F04F18471F
:10F358003B7D13FB04F3013301369BB2B6B2FB824B
:10F3680098E73A7D062A04BF9846BA469BE72B6879
:10F37800214A01332B60146001B0BDE8F08F02F020
:10F388005BFE1E4B1E4A1F4C11681A68A0EB090051
:10F3980002EB000E2268C3F800E09042A1EB511185
:10F3A800014438BF1046164A2060116094E702F005
:10F3B80043FEDAF80C300446984702F03DFEDAF8CE
:10F3C8002C20DAF82830DAF83010001B9042A3EB32
:10F3D80053130344014438BF1046CAF82830CAF80A
:10F3E8003010CAF82C0001B0BDE8F08F4FF0000BC8
:10F3F80036E700BF802800203C5D0020485D0020E3
:10F408004C5D0020505D0020F0B43423184F194A99
:10F4180003FB00F3D2F82461FC58FD18002E6B683A
:10F428004B600C600DDDD2F8D8309D421DD0D8322B
:10F43800002303E052F8044FA54216D00133B3422B
:10F44800F8D10022342303FB00700A720369CB60F1
:10F45800037D4B72836AC56A046BC2690A615B09E2
:10F468004D618C61CB61F0BC70470122EAE700BFB7
:10F47800B814002080280020F8B5494ED6F8244159
:10F48800102C73DC002C40F38880D6F8D8309842D2
:10F498006CD0012C57D0D6F8DC30984266D0022CBC
:10F4A80051D0D6F8E030984260D0032C4BD0D6F833
:10F4B800E43098425AD0042C45D0D6F8E830984227
:10F4C80054D0052C3FD0D6F8EC3098424ED0062CBC
:10F4D80039D0D6F8F030984248D0072C33D0D6F837
:10F4E800F430984242D0082C2DD0D6F8F830984203
:10F4F8003CD0092C27D0D6F8FC30984236D00A2CBC
:10F5080021D0D6F80031984230D00B2C1BD0D6F839
:10F51800043198422AD00C2C15D0D6F808319842DC
:10F5280024D00D2C0FD0D6F80C3198421ED00E2CBA
:10F5380009D0D6F81031984218D0102C03D1D6F83B
:10F548001431984212D0D6F8D85095B12B7D017D50
:10F558008B420DD3134A002505E052F8043B43B112
:10F568001B7D8B4205D30135AC42F6DA0020F8BD8D
:10F5780000256B1C9B0007460B48191F621B06EBF6
:10F58800850501449200184401341BF013FDC5F8A9
:10F59800D870C6F824410120F8BDD4D0E6E700BFF2
:10F5A800802800205C29002058290020122830D00B
:10F5B800102807D8184B342202FB003019B1C36851
:10F5C8000BB159E7704770B5144DD5F82441002C9C
:10F5D8000FDDD5F8D83098420CD005F1D80633465F
:10F5E800002203E053F8041F884206D00132A242E9
:10F5F800F8D170BD002205F1D8069000011DA21AAD
:10F60800920031443044013C1BF0D4FCC5F824413D
:10F6180070BD034B1868D1E7B8140020802800207B
:10F628003C5D002010B54FF4804082B0FFF78CF8A5
:10F6380000B30022032390F90200009301924FF4D3
:10F64800E1334FF48041FEF755FC0C4BC3F8C8007A
:10F6580070B1012402221020214683F8D04083F89B
:10F66800D14083F8D24083F8CC20FFF79FFF204693
:10F6780002B010BD014BD3F8C800E9E7802800208C
:10F68800F0B50646006803681B6A85B00D4603B1ED
:10F69800984795E81800E41A0023039324238DF86B
:10F6A80008304D238DF80930B5F90A30FF2C224671
:10F6B800A8BFFF2201333FD02B7B002B0CBF3E237A
:10F6C8003C238DF80A30FE2C2B898DF80B208DF801
:10F6D8000C3033DD23128DF80D408DF80E300727DE
:10F6E8003A4602A9306800F027FE02ABDA190DF19C
:10F6F8000B010023914223D1002C8DF807300CDD3B
:10F7080022462968306800F017FE2B689DF807200C
:10F7180019198B4218D18DF80720306801220DF194
:10F72800070100F009FE306803685B6A03B1984777
:10F7380004F1090005B0F0BD2123C2E70527CFE792
:10F7480011F8010B4340D5E713F8010B4240E0E7FD
:10F75800F8B50A4E05460024A359AB4204EB060748
:10F7680007D12846FEF79CFBCC22002138461BF027
:10F778003BFCCC34B4F5197FEED1F8BDFC65002014
:10F788002DE9F3470120FEF7DFFF174EDFF85CA0F5
:10F798000024CC2708B1022C02D902B0BDE8F087BA
:10F7A80007FB04F856F8085015B10134E4B2F1E744
:10F7B800C37890F902005AF8233001950322009289
:10F7C80001212A46FEF796FB814648B104FB0760F3
:10F7D800CC2229461BF008FC013446F80890E4B214
:10F7E80016F06AF8D6E700BFFC65002054CD020881
:10F7F8002DE9F04F2DED088BCB4CCC4BC4F83C38A1
:10F8080087B00023C4F84038FDF746FE00F0B0FF8B
:10F81800FDF7E4F808B914F03FFB14F061F994F827
:10F828004438C34D43F0010384F84438C14B9A78F7
:10F83800C14B1A70C14B1B682B600AF00FF90121EC
:10F84800022001F0D1FB01F0BBFC2B6819070BD596
:10F85800BB4B1A7A0A2A07D80123934040F2034285
:10F86800134201D009F030FF6420B64E02F030FC9C
:10F8780001F030FEB44ADFF80CE30023B146995D8D
:10F8880003F10F0003F11307304437440EEB010A6C
:10F8980010F8018FB8F1000F05D09AF80CC0C445D4
:10F8A80008BF82F858C090F80480B8F1000F05D05E
:10F8B8001EF801C0C44508BF82F859C0B842E7D154
:10F8C800B2F8580040B104EB810109EB0300506520
:10F8D800C1F8482802F517722033602BCFD1286869
:10F8E8009A4F42F2010318420CBF4FF0FF31012139
:10F8F800C0F38010FEF73CF9954B3A781A7007F080
:10F9080031FD0BF061FC2A68924B059712F4805F79
:10F918001E8B18BF904A9B7818BF9688042B04D179
:10F928004FF4805001F078FD002607F08BFA8B4BDE
:10F938003046197808F0BCFF0BF002FC884B1B68B6
:10F948000BB10DF0D9FA2B68DA0740F1A2820DF05D
:10F9580067FA94F84438DFF83092DFF8308243F0E1
:10F96800040384F844380DF0CFF959F8063C0393A2
:10F97800002B3AD019F90A6C142303FB06871A46A0
:10F98800002138461BF030FBA219A9F1030A92F8AE
:10F998005C3892F85EB804931AF8011F049B9942E8
:10F9A80003D1184600F0BEFEB8609AF80310594516
:10F9B80003D1584600F0B6FEF860D145ECD11423C7
:10F9C80003FB06F108EB0102906870B1D06860B1E2
:10F9D8002644A9F10A0048F8010096F86018039B2C
:10F9E800117496F86218536051745E4B09F110094E
:10F9F8009945BAD112F062FB5B495C4B0A79501EFB
:10FA0800424242411A704A79561E724272411A7134
:10FA18002A68574EC2F3C0329A7012F045F933681B
:10FA28002BB972681AB9B268002A00F0D5801BB2E7
:10FA380008EE103ADFED4FAADFED4F8A4F4AB8EED5
:10FA4800C88A002128EE2A8A117038EE280AFDEEAD
:10FA5800C07A17EE903A2033402B00F22082FDF74F
:10FA680055FBF0EE409AFDEEC87A17EE903A203337
:10FA7800402B00F21782B0EE480AFDF747FBB0EEC4
:10FA880040AAB6F9043009EE103AB8EEC99A29EE40
:10FA98002A9A39EE280AFDEEC07A17EE903A2033FA
:10FAA800402B00F20282FDF731FBB0EE40BAFDEECA
:10FAB800C97A17EE903A2033402B00F2F981B0EE64
:10FAC800490AFDF723FBB0EE409AB6F9083008EE74
:10FAD800103AB8EEC88A28EE2A8A38EE280AFDEECF
:10FAE800C07A17EE903A2033402B00F2E481FDF7FC
:10FAF8000DFBF0EE408AFDEEC87A17EE903A2033FF
:10FB0800402B00F2DB81B0EE480AFDF7FFFA69EE00
:10FB1800806A68EE8A7AF0EE665AE7EE895A184BE0
:10FB280028EEA96A34E000BF8028002095C80008A4
:10FB38005043002028600020593D0020DC6400204C
:10FB4800FC42002094B90208A8290020B035002002
:10FB580064470020683E0020E03C0020493D00202A
:10FB6800604700201EBA0208E05E00207C62002088
:10FB7800545D002035FA8E3CDB0FC93F7C00002025
:10FB8800143600202C430020FEB902088C620020A5
:10FB980020EE0A7AC3ED035AF0EE465AE7EE495AC8
:10FBA800E6EE897AA6EE497A68EE8B8A2BEE400A51
:10FBB8002AEE4BAA69EE8B9AC3ED008A83ED010AFF
:10FBC80083ED029AC3ED045A83ED05AA83ED067A04
:10FBD800C3ED077AC3ED089A06F0F2F840B902219E
:10FBE800012002F0FFF8B74A138843F0010313809D
:10FBF80094F84438B44F012143F00203084684F8CE
:10FC0800443801F0F1F90021084601F0EDF900212E
:10FC1800022001F0E9F90A26012000F0BDFB0020CE
:10FC280000F0BAFB192002F053FA3B68DB0302D458
:10FC3800012002F005FB192002F04AFA002002F028
:10FC4800FFFA013EE8D13146304601F0CDF93146A0
:10FC5800012001F0C9F99D4B9D4F1868DFF8E88233
:10FC68000BF0DAFA0BF002FA07F026FC13F062FD4B
:10FC78004FF41972314697481BF0B6F9FFF780FD2B
:10FC8800954B1E809E700AF0E5FC944BC8F8006006
:10FC98004FF0FF39C3F800903846914BC4F86438E8
:10FCA8000FF028FB8F4A84F87268012384F87038B3
:10FCB800537884F871980D3384F86C3813781E33B0
:10FCC80084F86D38D8F80030042B464605D05A1C05
:10FCD800C8F80020844A42F823702B689F0352D545
:10FCE80094F87C38814FDFF86492C7F80090013BA4
:10FCF80084F87438C82094F87D3884F8753802F090
:10FD0800E7F93868DFF84882FDF7A0FB88F80000BB
:10FD1800C82002F0DDF93B68C4F8843809F10C0703
:10FD2800734BC4F8803838460FF092FA012384F8F0
:10FD38008C38002384F88E38FF2384F88D38082304
:10FD480084F88838152384F889386A4B1F6098F836
:10FD580000303BB13368042B04D05A1C3260624A2D
:10FD680042F82370644C1022002120461BF03CF915
:10FD780000200FF0D9FE02F05FF906460FF0EEFE04
:10FD88005E4B3344E3602B685C0501D50FF032FE0F
:10FD98002B68180101D508F0F5FB594B594A9B7897
:10FDA800003318BF01231370059B1B78052B03D163
:10FDB800554B4FF4C8721A80544B554C1A684FF47F
:10FDC8007A73B3FBF2F3C3EB431203EB8203514A9A
:10FDD800DB00A2F8A8304FF40060FEF7B5FC68B16C
:10FDE8000321182390F9020000228DE80A004FF43D
:10FDF80096534FF40061FEF77DF82060236813B135
:10FE0800454B464A1A604FF40050FEF79DFC444C9F
:10FE180068B10322082390F902004FF400518DE8DD
:10FE28000C004FF416530022FEF764F82060236894
:10FE380013B1394B3B4A1A603B4A137843F0080325
:10FE48001370FFF7CBF82B689B0306D52A4B0722C4
:10FE58005A721A7A42F001021A72344B1A68344BF9
:10FE68001A60344B344A1B689B1A344A18BF012362
:10FE78001370FEF743FEFFF7D5FB314A92F844387A
:10FE880063F07F0382F8443807B0BDEC088BBDE807
:10FE9800F08F9F047FF55DAD0CF06EFF59E5DFED47
:10FEA800299AE0E59FED27AAEBE59FED26BAFEE546
:10FEB8009FED249A09E6DFED238A1CE69FED210ACF
:10FEC80025E600BF7A490020685D0020F05E00202A
:10FED800E4300020FC650020085D0020340100208B
:10FEE80014BA0208C85B0020D4490020E45B002053
:10FEF80040BA0208FC5C0020EC5C0020404B4C003F
:10FF08005D600020686000203C75002040520020A1
:10FF1800A47100201C4A0020A865002030000020A1
:10FF2800645B00204C00002010360020DC640020B8
:10FF380050430020843E00207D5D0208F8420020E6
:10FF48008028002000000000D0490020F430002064
:10FF5800055D002008B50E4B1978012913D00DD383
:10FF6800022902D1002000F017FA02F065F8094BC7
:10FF780000F5F42000F59070186008BD00210846CF
:10FF880001F032F8F1E7002001F02EF8EDE700BFAC
:10FF98003E75002040750020436A826970B4D154D0
:10FFA800436A0469426B0133A34228BF00234362BA
:10FFB800DAB1116811F0010101D070BC7047856A8F
:10FFC80086699D422E44D6600BD3641B54608162BF
:10FFD8001368002143F0010380F8441070BC1360DB
:10FFE80070475D1B55608362F2E7026D136843F04A
:08FFF80080031360E1E700BF84
:020000040801F1
:10000000026B10B462B1036CC2684469D11A013B3F
:10001000615C5DF8044B08BF13460364C8B27047C7
:10002000016A4369C4685B5C0131A14228BF114683
:1000300001625DF8044BD8B2704700BF436B13B147
:1000400090F844007047836A406A181AB0FA80F04A
:1000500040097047416A836A99420AD3CB1A416BBF
:10006000026961B14968501E0B4483420AD2C01A2A
:10007000704702691144CB1A416B0029F2D1501E1E
:10008000C01A704700207047036B43B1026C5B6875
:1000900093422FBF981AC0689B1AC0187047C26954
:1000A000036A9A422FBFD01AC0688018C01A7047DE
:1000B0000A4B30B503F1140493F900205D78072A48
:1000C000C8BF143A811804330D7313F8025C8554C9
:1000D00013F8012C0A76A342EED130BDD8BA02083B
:1000E00003682DE9F041DF691FB13B46BDE8F041EF
:1000F0001847002A164611DD04460D460E4400E05E
:1001000023689B68204698470028F9D0236815F893
:10011000011B1B6820469847AE42F1D1BDE8F08133
:1001200000232122027043708370C370704700BFA8
:1001300030B50446006D61710368A26823F00103C5
:10014000036087B0A379009213F004023DD04FF40E
:10015000805213F00203019244D102934FF4806362
:100160000022039311F00103059237D10493082371
:100170008D07694648BF04930DF04AFB6079236DF3
:10018000A17900F00202002A15BF4FF440324FF46B
:1001900080324FF40034002410F0010F586808BF7B
:1001A0002246CC074CBF024320EA02025A609A68FA
:1001B00009074CBF42F0080222F008029A601A6850
:1001C00042F001021A6007B030BD13F00203019241
:1001D0000BD04FF4005513460295C1E70423049356
:1001E0000C23C5E74FF40053B7E70293B8E700BF0D
:1001F00010B50446006DA160036823F0010303609D
:10020000A37986B013F00402009141D04FF48052DC
:1002100013F00203019244D102934FF48063627998
:100220000393D1074FF000030493059345BF0423C4
:10023000049308230C236946920748BF04930DF0EA
:10024000E7FA6079236DA17900F00202002A15BF58
:100250004FF440324FF480324FF40034002410F059
:10026000010F586808BF2246CC074CBF024320EA62
:1002700002025A609A6809074CBF42F0080222F055
:1002800008029A601A6842F001021A6006B010BDB6
:1002900013F00203019207D04FF40051134602916C
:1002A000BDE74FF40053B7E70293B8E700232622D7
:1002B0000360027027228270012243600271837101
:1002C000704700BF1D4B70B51C68236D226BDD6944
:1002D000C2B1636B2BB12B0702D5236D08221A62C2
:1002E00070BD2A06F7D5A26A616A8A421FD0511CE6
:1002F000A069A162825C2069266D81423285EAD3C1
:10030000A362E8E7A906E4D5E26A1AB1988C80B244
:100310009047DEE7E1699B8C6069DBB24E1CE661C9
:100320004354E169E368994228BFE261D1E7226D55
:10033000136823F080031360CDE700BFC8300020AE
:1003400003682DE9F041DF691FB13B46BDE8F0418C
:100350001847002A164611DD04460D460E4400E0FB
:1003600023689B68204698470028F9D0236815F831
:10037000011B1B6820469847AE42F1D1BDE8F081D1
:1003800003689B69184700BF0368DB68184700BF14
:1003900003685B68184700BF03681B68184700BF05
:1003A000054B53F8203033B11A689B88918A0B4271
:1003B00018BF1B0493617047BC620020036803F1FF
:1003C00038422DE9F04F920A584DAA5C02F01F0501
:1003D00052090124022A04FA05F400F08C80032A51
:1003E00000F08E80012A3CD001F003077A1E012A1A
:1003F000C1F3810CC1F300188088C1F3411135D9D4
:10040000C60700F19780850700F1A380440700F13B
:10041000B180020700F1BF80C60600F1CD808506DD
:1004200000F1DB80440600F1E980020600F1F7806C
:10043000C60500F10581850500F11381440500F131
:100440002181020500F12F81C60400F13D81850460
:1004500000F14B81440400F15981020455D4BDE8F8
:10046000F08F334A55692C435461BDE7002422467E
:100470004FF0010E4FF0030904E00132102A04F19D
:100480000204ECD00EFA02F636EA0005F5D1D3F8F4
:1004900008A009FA04F5ED430AEA050AC3F808A022
:1004A000D3F808B00CFA04FA4AEA0B0AC3F808A019
:1004B000B3F804A01FFA8AFA2AEA06069E80B3F867
:1004C00004A008FA02F646EA0A06B6B29E801E6842
:1004D0002E401E60D3F800A007FA04F646EA0A068A
:1004E0001E60D3F80CA001FA04F605EA0A0A46EAEF
:1004F0000A05DD60C1E70E4A95692C43946173E7F4
:100500000B4AD5692C43D4616EE71A6822F0404249
:100510001A601A6842EA87771F60DA6822F0404260
:1005200042EA8171D960BDE8F08F00BF0CD20208A9
:10053000001002401A6822F003021A601A683A4357
:100540001A60DA6822F003020A438507DA607FF551
:100550005DAF1A6822F00C021A601A6842EA87023C
:100560001A60DA6822F00C0242EA81024407DA607B
:100570007FF54FAF1A6822F030021A601A6842EA1B
:1005800007121A60DA6822F0300242EA0112DA60D9
:1005900002077FF541AF1A6822F0C0021A601A689C
:1005A00042EA87121A60DA6822F0C00242EA811237
:1005B000C606DA607FF533AF1A6822F440721A601B
:1005C0001A6842EA07221A60DA6822F4407242EAA4
:1005D00001228506DA607FF525AF1A6822F44062B1
:1005E0001A601A6842EA87221A60DA6822F44062C6
:1005F00042EA81224406DA607FF517AF1A6822F4D6
:1006000040521A601A6842EA07321A60DA6822F425
:10061000405242EA0132DA6002067FF509AF1A68F9
:1006200022F440421A601A6842EA87321A60DA6895
:1006300022F4404242EA8132C605DA607FF5FBAE21
:100640001A6822F440321A601A6842EA07421A60B5
:10065000DA6822F4403242EA01428505DA607FF529
:10066000EDAE1A6822F440221A601A6842EA874204
:100670001A60DA6822F4402242EA81424405DA60D4
:100680007FF5DFAE1A6822F440121A601A6842EA57
:1006900007521A60DA6822F4401242EA0152DA6024
:1006A00002057FF5D1AE1A6822F440021A601A687A
:1006B00042EA87521A60DA6822F4400242EA815222
:1006C000C604DA607FF5C3AE1A6822F040721A6081
:1006D0001A6842EA07621A60DA6822F0407242EA57
:1006E00001628504DA607FF5B5AE1A6822F04062D7
:1006F0001A601A6842EA87621A60DA6822F0406279
:1007000042EA81624404DA607FF5A7AE1A6822F0FB
:1007100040521A601A6842EA07721A60DA6822F0D8
:10072000405242EA0172DA6097E600BF10B5040950
:10073000013C052C17D80D4B33F8142000F00F00A6
:1007400042FA00F313F001030DD0012303FA00F085
:100750000138104018F0C4F8054A064B125D1044E9
:1007600003EBC00010BD002010BD00BF24CC020868
:1007700030CC0208CC5800202DE9F04F4A484B4BB2
:100780004B4C4FF090414FF0010A4FF002094FF0EF
:1007900004084FF0080C4FF0100E2027402680254B
:1007A00030F8022B12F0010F03D01960A3F804A057
:1007B000083312F0020F03D01960A3F80490083335
:1007C00012F0040F03D01960A3F80480083312F06C
:1007D000080F03D01960A3F804C0083312F0100FFB
:1007E00003D01960A3F804E0083312F0200F02D000
:1007F00019609F80083312F0400F02D019609E806C
:10080000083312F0800F02D019609D80083312F473
:10081000807F05D04FF4807B1960A3F804B00833C3
:1008200012F4007F05D04FF4007B1960A3F804B0E8
:10083000083312F4806F05D04FF4806B1960A3F871
:1008400004B0083312F4006F05D04FF4006B196048
:10085000A3F804B0083312F4805F05D04FF4805B36
:100860001960A3F804B0083312F4005F05D04FF408
:10087000005B1960A3F804B0083312F4804F05D070
:100880004FF4804B1960A3F804B00833D20B04D0A6
:100890004FF4004219609A80083301F58061A1424B
:1008A0007FF47EAFBDE8F08F24CC0208CC58002046
:1008B00000180048002867D003682DE9F04F03F1C5
:1008C00038445C4EA40A0125345D04F01F06640917
:1008D000022C05FA06F558D0032C00F0A580012C57
:1008E00058D08088B0FA80F4C4F11F04A4B2E5089F
:1008F00003EB850504F007042E6AA4000F27A74028
:1009000026EA07062E622E6A01F00307A2407C1E2B
:100910003243012CC1F3810CC1F300182A62C1F3E8
:1009200041113CD9C60700F18980850700F1958007
:10093000440700F1A380020700F1B180C60600F170
:10094000BF80850600F1CD80440600F1DB80020601
:1009500000F1E980C60500F1F780850500F1058109
:10096000440500F11381020500F12181C60400F164
:100970002F81850400F13D81440400F14B81020484
:1009800000F15981BDE8F08F70472B4CA6693543C3
:10099000A561A6E7284C666935436561A1E7002497
:1009A00022464FF0010E4FF0030904E00132102AF5
:1009B00004F10204E6D00EFA02F636EA0005F5D19B
:1009C000D3F808A009FA04F5ED430AEA050AC3F8CA
:1009D00008A0D3F808B00CFA04FA4AEA0B0AC3F8E4
:1009E00008A0B3F804A01FFA8AFA2AEA06069E8035
:1009F000B3F804A008FA02F646EA0A06B6B29E80E8
:100A00001E682E401E60D3F800A007FA04F646EADE
:100A10000A061E60D3F80CA001FA04F605EA0A0AD9
:100A200046EA0A05DD60C1E7034CE6693543E56146
:100A300057E700BF0CD20208001002401A6822F0EB
:100A400003021A601A683A431A60DA6822F0030255
:100A50000A438507DA607FF56BAF1A6822F00C0253
:100A60001A601A6842EA87021A60DA6822F00C02F9
:100A700042EA81024407DA607FF55DAF1A6822F02E
:100A800030021A601A6842EA07121A60DA6822F025
:100A9000300242EA0112DA6002077FF54FAF1A68AE
:100AA00022F0C0021A601A6842EA87121A60DA68F5
:100AB00022F0C00242EA8112C606DA607FF541AF39
:100AC0001A6822F440721A601A6842EA07221A6011
:100AD000DA6822F4407242EA01228506DA607FF584
:100AE00033AF1A6822F440621A601A6842EA872219
:100AF0001A60DA6822F4406242EA81224406DA602F
:100B00007FF525AF1A6822F440521A601A6842EA4B
:100B100007321A60DA6822F4405242EA0132DA609F
:100B200002067FF517AF1A6822F440421A601A686D
:100B300042EA87321A60DA6822F4404242EA81329D
:100B4000C605DA607FF509AF1A6822F440321A60F0
:100B50001A6842EA07421A60DA6822F4403242EA2E
:100B600001428505DA607FF5FBAE1A6822F4402267
:100B70001A601A6842EA87421A60DA6822F4402250
:100B800042EA81424405DA607FF5EDAE1A6822F44C
:100B900040121A601A6842EA07521A60DA6822F4B0
:100BA000401242EA0152DA6002057FF5DFAE1A68B0
:100BB00022F440021A601A6842EA87521A60DA6820
:100BC00022F4400242EA8152C604DA607FF5D1AED7
:100BD0001A6822F040721A601A6842EA07621A60C4
:100BE000DA6822F0407242EA01628504DA607FF539
:100BF000C3AE1A6822F040621A601A6842EA87623D
:100C00001A60DA6822F0406242EA81624404DA60E3
:100C10007FF5B5AE1A6822F040521A601A6842EAAF
:100C200007721A60DA6822F0405242EA0172DA6012
:100C300002047FF5A7AE1A6822F040421A601A68D3
:100C400042EA87771F60DA6822F0404242EA817107
:100C5000D960BDE8F08F00BF002852D0036803F1CF
:100C600038422DE9F04F920A504DAA5C02F01F0560
:100C700052090124022A04FA05F443D0032A00F0A1
:100C80009080012A43D001F003077A1E012AC1F3A4
:100C9000810CC1F300188088C1F341113CD9C6070B
:100CA00000F18880850700F19480440700F1A2805C
:100CB000020700F1B080C60600F1BE80850600F193
:100CC000CC80440600F1DA80020600F1E880C60517
:100CD00000F1F680850500F10481440500F11281E0
:100CE000020500F12081C60400F12E81850400F187
:100CF0003C81440400F14A81020400F15881BDE8BE
:100D0000F08F70472A4A95692C439461BBE7284AC3
:100D100055692C435461B6E7002422464FF0010E7A
:100D20004FF0030904E00132102A04F10204E6D076
:100D30000EFA02F636EA0005F5D1D3F808A009FA52
:100D400004F5ED430AEA050AC3F808A0D3F808B091
:100D50000CFA04FA4AEA0B0AC3F808A0B3F804A094
:100D60001FFA8AFA2AEA06069E80B3F804A008FA57
:100D700002F646EA0A06B6B29E801E682E401E6043
:100D8000D3F800A007FA04F646EA0A061E60D3F874
:100D90000CA001FA04F605EA0A0A46EA0A05DD6033
:100DA000C1E7034AD5692C43D4616CE70CD2020831
:100DB000001002401A6822F003021A601A683A43CF
:100DC0001A60DA6822F003020A438507DA607FF5C9
:100DD0006CAF1A6822F00C021A601A6842EA8702A5
:100DE0001A60DA6822F00C0242EA81024407DA60F3
:100DF0007FF55EAF1A6822F030021A601A6842EA84
:100E000007121A60DA6822F0300242EA0112DA6050
:100E100002077FF550AF1A6822F0C0021A601A6804
:100E200042EA87121A60DA6822F0C00242EA8112AE
:100E3000C606DA607FF542AF1A6822F440721A6083
:100E40001A6842EA07221A60DA6822F4407242EA1B
:100E500001228506DA607FF534AF1A6822F4406219
:100E60001A601A6842EA87221A60DA6822F440623D
:100E700042EA81224406DA607FF526AF1A6822F43E
:100E800040521A601A6842EA07321A60DA6822F49D
:100E9000405242EA0132DA6002067FF518AF1A6862
:100EA00022F440421A601A6842EA87321A60DA680D
:100EB00022F4404242EA8132C605DA607FF50AAF89
:100EC0001A6822F440321A601A6842EA07421A602D
:100ED000DA6822F4403242EA01428505DA607FF5A1
:100EE000FCAE1A6822F440221A601A6842EA87426D
:100EF0001A60DA6822F4402242EA81424405DA604C
:100F00007FF5EEAE1A6822F440121A601A6842EABF
:100F100007521A60DA6822F4401242EA0152DA609B
:100F200002057FF5E0AE1A6822F440021A601A68E2
:100F300042EA87521A60DA6822F4400242EA815299
:100F4000C604DA607FF5D2AE1A6822F040721A60E9
:100F50001A6842EA07621A60DA6822F0407242EACE
:100F600001628504DA607FF5C4AE1A6822F040623F
:100F70001A601A6842EA87621A60DA6822F04062F0
:100F800042EA81624404DA607FF5B6AE1A6822F064
:100F900040521A601A6842EA07721A60DA6822F050
:100FA000405242EA0172DA6002047FF5A8AE1A6884
:100FB00022F040421A601A6842EA87771F60DA68B6
:100FC00022F0404242EA8171D960BDE8F08F00BF53
:100FD00010B1036882881A85704700BF38B10029B4
:100FE0008388026814BF002110218B4093617047F1
:100FF00010B40A4B0A4A1C7801238340234052F85C
:10100000200029B9B3FA83F149095DF8044BE5E7FB
:10101000191C18BF01215DF8044BDFE7BA620020FC
:10102000BC6200202DE9F0410B4E346873691C400E
:101030000FD0DFF828800127B4FA84F3C3F11F032F
:1010400007FA03F558F8230003689847AC43756125
:10105000F2D1BDE8F08100BF00040140A072002081
:101060002DE9F0410B4E346873691C400FD0DFF856
:1010700028800127B4FA84F3C3F11F0307FA03F5AC
:1010800058F8230003689847AC437561F2D1BDE876
:10109000F08100BF00040140A07200202DE9F04162
:1010A0000B4E346873691C400FD0DFF8288001278D
:1010B000B4FA84F3C3F11F0307FA03F558F82300C9
:1010C00003689847AC437561F2D1BDE8F08100BF79
:1010D00000040140A07200202DE9F0410B4E34685D
:1010E00073691C400FD0DFF828800127B4FA84F31D
:1010F000C3F11F0307FA03F558F823000368984764
:10110000AC437561F2D1BDE8F08100BF000401403D
:10111000A07200202DE9F0410B4E346873691C4029
:101120000FD0DFF828800127B4FA84F3C3F11F033E
:1011300007FA03F558F8230003689847AC43756134
:10114000F2D1BDE8F08100BF00040140A072002090
:101150002DE9F0410B4E346873691C400FD0DFF865
:1011600028800127B4FA84F3C3F11F0307FA03F5BB
:1011700058F8230003689847AC437561F2D1BDE885
:10118000F08100BF00040140A07200202DE9F04171
:101190000B4E346873691C400FD0DFF8288001279C
:1011A000B4FA84F3C3F11F0307FA03F558F82300D8
:1011B00003689847AC437561F2D1BDE8F08100BF88
:1011C00000040140A07200200B490C4A0C4808B5ED
:1011D0008B6943F001038B61136843F48053136000
:1011E0000021402219F004FF064B4FF0FF321A6035
:1011F000C3F8032008BD00BF0010024000000140FA
:10120000A0720020E07200202DE9F041044618464B
:101210000D461646984616F0B9FE2768E672284431
:10122000A07229467D69434632462046AC46BDE859
:10123000F0416047036810B504461B68984723686F
:1012400020469B689847A37B0133A37310BD00BF62
:10125000427A02B9704710B504460368406804F149
:101260000A0198470023637210BD00BF437A5A1CDD
:101270000344D2B242729972037A934200D802B9FF
:10128000704710B504460368406804F10A019847A6
:101290000023637210BD00BF30B40B4D002305F175
:1012A000140101E0272B0BD011F8132082424FEAE2
:1012B000430403F10103F5D12C44607D30BC704739
:1012C000002030BC704700BFD8BA02082DE9F341B6
:1012D000056906460F467DBBD0F80080C8F30A03B7
:1012E00023B30023D6F80080019308F0DBF904282B
:1012F00019D1224C236943F001032361BBB2A8F842
:10130000003008F0CFF904282ED108F10203019330
:10131000019B3F0C1F8008F0C5F92369042823F0C6
:101320000103236125D06FF0010505E008F0BAF94B
:10133000042805D04FF0FF35284602B0BDE8F08103
:101340000E4C236943F002032361C4F8148023691F
:1013500043F04003236108F0A5F92369042823F032
:1013600002032361BDD0E5E7236923F00103236174
:10137000D9E7336804333360DEE700BF0020024062
:10138000F8B504460D468E180027B54201D12069F4
:10139000F8BDE368591CE160234415F8012B1A726B
:1013A0000429F2D1A1682046FFF790FFE760206191
:1013B000EBE770B5448806460D46C4F30B0422469D
:1013C0000021284619F014FE33690A4A934209D3D2
:1013D000094A934206D2224628461946BDE8704083
:1013E00019F0E1BD23B121462846BDE870401847F9
:1013F00070BD00BF140A0308B40A0308064B07496E
:101400008B4202D30023184670471A88C2F30B029E
:101410009042F8D01433F3E740060308140A030897
:10142000024A136823EA000010607047DC64002061
:101430002DE9F0470569C3681D4028D00F460646D0
:101440004FF000484FF00009B5FA85F328FA03F28F
:10145000D2431B3B32611540042B16D8DFE803F062
:101460003129211903007B6A002B32D003F1FF3AA6
:101470001FFA8AFAC7F824903C6A34B123682046E0
:10148000514698476468002CF8D1002DDCD1BDE8A6
:10149000F0873868716B036889B29847002DD3D103
:1014A000F5E77868B16B036889B29847002DCBD116
:1014B000EDE7B868F16B036889B29847002DC3D196
:1014C000E5E7F868316C036889B29847002DBBD115
:1014D000DDE7F36A1FFA83FACEE700BF2DE9F84F84
:1014E0004FF4A07200218F488F4CDFF864928F4D2B
:1014F0008F4E904FDFF85C8219F07AFD8E488F494D
:10150000DFF854E2DFF854C200221359834200F09E
:10151000F880B3F1804F00F0F680AB4200F0F58028
:10152000B34200F0F480BB4200F0F380734500F05A
:10153000F280634500F0F180434500F0F080DFF871
:1015400020A2534500F0A7800AF5806A534508BFE2
:10155000092300F0A1801432DC2AD6D1DFF8C8813B
:10156000774F784D08F1DC064FF0030A4FF002097F
:1015700098F804301C09013C052C03F00F0300F21D
:10158000838037F8140040FA03F2D2077CD54FF07D
:10159000010B0BFA03F3013B184017F0A1F96A4B5A
:1015A0001B5D184415EBC0046ED055F83030674809
:1015B00098F8081003F13842920A825C02F01F008A
:1015C0005209022A0BFA00FB00F09480032A00F073
:1015D0008A80012A05D1594A584852694BEA0202C9
:1015E0004261B4F804E0BEFA8EF2C2F11F0292B278
:1015F000D00803EB800002F00702046A92004FF06B
:101600000F0C0CFA02FC24EA0C040462046A01FACE
:1016100002F22243002402624FF0010C224603E052
:10162000102A04F102042FD00CFA02F030EA0E0165
:1016300002F10102F4D1D3F808B00AFA04F1C94367
:101640000BEA010BC3F808B0D3F808B0C3F808B030
:10165000B3F804B01FFA8BFB2BEA0000988098883F
:1016600080B29880186808401860D3F800B009FA72
:1016700004F040EA0B001860D868102A01EA000163
:10168000D96004F10204CFD108F1140846457FF473
:101690006FAFBDE8F88F082309EBC3034FF0010BD0
:1016A00093F804A00AF01F034FEA5A1ABAF1020F86
:1016B0000BFA03F30BD0BAF1030F0ED0DA457FF427
:1016C0004AAFD1F814A043EA0A034B6143E7D1F8CB
:1016D00018A043EA0A038B613DE7D1F81CA043EA56
:1016E0000A03CB6137E7154A1448D2694BEA020274
:1016F000C26176E7114A114892694BEA020282619F
:101700006FE70023C8E70123C6E70223C4E70323EA
:10171000C2E70423C0E70523BEE70623BCE707238F
:10172000BAE700BFE872002034D602080004004087
:101730000008004000100040002C01400010024052
:1017400024CC0208CC58002030CC02080CD202086D
:101750003CBB02080040014000140040003401403E
:10176000004401400149024862E600BF00740020C5
:1017700000480140014902485AE600BFB07300200A
:10178000004001400149024852E600BF8873002032
:1017900000340140014902484AE600BF8873002036
:1017A000003401400149024842E600BF6073002056
:1017B00000080040014902483AE600BF38730020A3
:1017C0000004004001494FF0804031E610730020D2
:1017D00010B5054C05482146FFF72AFE04F1F0013B
:1017E0000348BDE8104023E6E8720020002C0140C9
:1017F00000440140014902481AE600BFE872002097
:10180000002C01402DE9F0410468574DA30AAB427A
:1018100000F085805CD9554DAB426CD078D9544DE1
:10182000AB4264D00135AB4240F09A804FF49C7ECD
:10183000072647794FEA970C00297CD0B000634611
:1018400085190227D4F80C809F400CEB4503BFB2EA
:10185000484D03F1040C47EA080745F8231045F802
:101860002C20E760EFF31181502282F31288821955
:1018700005EBC2021369002B41D0136204338219B5
:1018800005EBC202576917B11F605369043382190F
:1018900005EBC202976917B11F609369043382197F
:1018A00005EBC202D76917B11F60D3690433002763
:1018B000CAB21F6082F31188304405EBC000036A8E
:1018C00003BBE3684FF6FE721340E360BDE8F081AE
:1018D0004A3DAB422BD00135AB4204D0B3F5801F5B
:1018E00021D0BDE8F0814FF0980E0326A1E74FF418
:1018F000887E06269DE74FF0E80E052699E705EB62
:101900000E03BCE7E36843F00103E360BDE8F08148
:10191000033DAB4226D14FF0C00E042689E74FF0BD
:10192000200E002685E74FF0480E012681E74FF094
:10193000700E02267DE7BF08022306FA03F0BB40C3
:10194000DB43E7680B4D9BB23B4087190CEB470C20
:10195000E3600CF1040345F82C1045F8232081E7DF
:10196000BDE8F081BDE8F0814B0010005000100090
:1019700051001000E872002030B503685C4D1888F3
:101980005C4CB4FBF2F20139013AAB4294B283B041
:1019900089B282B266D05848834263D0B3F1804F97
:1019A00060D0A0F5983083425CD000F5806083421F
:1019B00058D0524883425BD000F5806083427CD08F
:1019C00022F4407200F58C3092B283421A80D962C0
:1019D0001C850ED0484A93420BD002F540629342D8
:1019E00007D002F58062934203D002F580629342F1
:1019F00001D100221A8601225A611A883C4992B20A
:101A000042F001028B421A8061D0B3F1804F60D066
:101A10003B4A93425FD002F5806293425DD002F56B
:101A2000006293425BD002F58062934259D002F586
:101A30009032934257D002F54062934255D002F55E
:101A4000806293421ED002F58062934208BF092251
:101A500019D002A84FF0012340F8043D10F0ACFB70
:101A600003B030BD254822F07002834292B2A3D168
:101A700001201A80D9621C8558611A8892B20243EB
:101A80001A80C5E708221F4B03EBC20301A85C794B
:101A90008DF80440012300228DF805308DF80730C1
:101AA0008DF8062010F088FB1B2CD9D1164B019322
:101AB00001A810F081FB03B030BD01201A80D9626B
:101AC0001C8558611A8892B202431A809DE7002251
:101AD000D9E70122D7E70222D5E70322D3E7042280
:101AE000D1E70522CFE70622CDE70722CBE700BFEB
:101AF000002C014000A24A040034014000100040C4
:101B0000000400403CBB0208190100011F4B984231
:101B10002CD0B0F1804F2BD0A3F59433984229D02C
:101B200003F58063984227D003F50063984225D0DF
:101B300003F58063984223D003F59033984221D077
:101B400003F5406398421FD003F58063984207D0A5
:101B500003F58063984208BF092202D00020704735
:101B600008220B4B03EBC203187970470022F8E7F9
:101B70000122F6E70222F4E70322F2E70422F0E76B
:101B80000522EEE70622ECE70722EAE7002C0140F7
:101B90003CBB02082DE9F04F013085B0C3B203937E
:101BA0008C4D8D4F8D4C8E4E0A230293DFF834926C
:101BB00012F0AEFF4FF4FA7A4FF0100C4FF47A7037
:101BC000D9F80430C3F30803002B40F0C580EFF3CD
:101BD0001183002B40F0C0802968A26800BF2B68E9
:101BE0009942F9D1D7F800E000FB0EF39B1AB3FB42
:101BF000FEF300FB01314FF0010E0191D9F80430E2
